:020000021000EC
:10F000000000012039F5010061F5010063F5010000
:10F0100065F5010067F5010069F5010000000000D9
:10F020000000000000000000000000006BF501007F
:10F030006DF50100000000006FF501004922040099
:10F04000C954020073F50100BD56020029550200A3
:10F0500075550200D16602002958020073F50100BF
:10F0600073F501008D22040073F5010073F50100B2
:10F0700073F501009161020073F5010073F5010061
:10F0800089220400952D020073F5010073F501003B
:10F090009D2E0200E9D50300911E020073F50100C8
:10F0A00073F5010073F5010073F501003169020089
:10F0B00073F5010073F5010000000000000000007E
:10F0C00073F5010073F5010073F5010073F501009C
:10F0D00073F501005D63020073F50100000000009C
:10F0E0000000000000000000000000000000000020
:10F0F0000000000000000000000000000000000010
:10F1000000000000000000000000000000000000FF
:10F1100000000000000000000000000000000000EF
:10F4000010B5054C237833B9044B13B10448AFF35E
:10F4100000800123237010BD602E0020000000003A
:10F4200030C3060008B5034B1BB103490348AFF3D3
:10F43000008008BD00000000642E002030C30600DC
:10F44000154B002B08BF134B9D46A3F5803A0021B6
:10F450008B460F461348144A121A00F063F80F4BFC
:10F46000002B00D098470E4B002B00D0984700206F
:10F47000002104000D000D48002802D00C48AFF315
:10F48000008000F02BF82000290023F0BBF800F0EA
:10F4900011F800BF0000080000000120000000007B
:10F4A00000000000602E002040E500200000000069
:10F4B0000000000008B5074B044613B10021AFF36C
:10F4C0000080054B1868836A03B19847204600F016
:10F4D00031F800BF000000001816060070B50D4D91
:10F4E0000D4C641BA4100026A64209D10B4D0C4CF8
:10F4F00042F086F8641BA4100026A64205D170BD18
:10F5000055F8043B98470136EEE755F8043B984719
:10F510000136F2E7302E0020302E0020302E002061
:10F52000342E002002440346934200D1704703F872
:10F53000011BF9E7FEE700BF0649074A074B9B1A84
:10F5400003DD043BC858D050FBDC06F0F5FFFFF7A5
:10F5500077FF00003CC30600402C0020602E0020F6
:10F56000FEE7FEE7FEE7FEE7FEE7FEE7FEE7FEE773
:10F57000FEE7FEE72DE9F04F00250646A84628469F
:10F580004FF480744FF6FF7C2E270B78B8F1000FF4
:10F5900000D1013003F0C00EBEF1C00F11D0013117
:10F5A0009BB283B3013CE41A24B2002C33DBB8F1E4
:10F5B000000F00D1184401F1FF3A02F1FF399E46D5
:10F5C00012E0B8F1000F00D1013049781B0203F4BA
:10F5D0007C530B44F1180131F35C4FF00108E0E774
:10F5E0001AF801BF09F801BF0EF1FF3E1FFA8EFEA7
:10F5F000E645F5D102EB030E194401331A448EF8A7
:10F6000000700135C1E715B92E2302F8013B002334
:10F610001370BDE8F08F4FF0FF30FAE71FB50123FC
:10F620008DF80030054B8DF8080001916846D3E94C
:10F630000012904705B05DF804FB00BF9CCB002092
:10F6400061DF704748DF704710B50388012B11D880
:10F65000094A02EB031243885189CC1A032C09D4BE
:10F66000C3F57F43FD330B44538100230380438064
:10F67000184610BD0420FCE7A0D0002010B5124AA7
:10F680000B6802EB0010426873B15888033003EB3B
:10F69000800302F580524FF6FF749A4202D918682F
:10F6A000013004D1002009E002F10803F1E7988855
:10F6B000A04204D0188810B10B60012010BD5888FA
:10F6C000033003EB8003E8E7A0D0002073B5436864
:10F6D00004460D4613B31E4A11688B421ED352686E
:10F6E00093421BD813F0030018D11A4A21891289BA
:10F6F000914213D121689A6891420FD1164A5268FB
:10F70000934201D80A2004E002F580529342F9D2D4
:10F710002880B0FA80F0400902B070BD00232B8031
:10F720001E46019601A92888FFF7A8FF30B92B884B
:10F7300001339BB22B80002BF3D0EDE7019B2268B5
:10F7400099689142EED16360024B1B892381E3E704
:10F75000382E002060CD0020A0D00020033083B2DE
:10F7600040F2FD32934230B50ED909200BE02289D8
:10F7700065892A441A4492B2B2F5806F08D2088093
:10F7800062891344638130BD024C20780028EED09A
:10F790000720F8E7A0D0002010B50A494A788C78F5
:10F7A000531CDBB29C4208BF00230C789C421FBF55
:10F7B0000370486802EB420200EBC20008BF002061
:10F7C00010BD00BF1CD00020AADF7047A9DF704722
:10F7D000A7DF704785DF70477FDF70477EDF7047A8
:10F7E000084A30B500230C2404FB03F18D5A8542EE
:10F7F00002D10A44508830BD0133082BF4D14FF6B2
:10F80000FF70F8E7CACC00206EDF704758B1CB0814
:10F8100001F00701C25C012303FA01F10A4214BF9F
:10F8200018460020704701207047000070B50A4E4E
:10F830003468054654B1706860B1FF2D08D0294680
:10F84000FFF7E4FF30B1F36803FB0544204670BDC9
:10F850000024FBE70446F9E72CD20020012804D05D
:10F86000043804288CBF0020012070478378013BB6
:10F87000072B07D8DFE803F007060606060704098A
:10F880001423038070470123FBE743689B880933F7
:10F890009B08F6E770B5054D0646002455F8043B75
:10F8A000304601349847052CF8D170BDA8170600E2
:10F8B000114BF0B5002214261D4606FB02F4E75A50
:10F8C000874212D12344142600249A788A420AD00F
:10F8D00001342246072A0BD806FB02F3EF5A87426F
:10F8E00008D1EB18F1D11846F0BD0132082AE4D155
:10F8F0000023F8E70132EDE73CD2002030B50721C4
:10F9000085B0FFF7D5FF044600283AD04568002DA2
:10F9100039D1007CFFF78AFF0721CDE902558DF828
:10F920000A1040B3E368039003EB83031B019BB20F
:10F930009B0802A8ADF80830FFF798FF9DF80A0071
:10F94000FFF78CFFD8B1114B1B789B0715D5BDF87D
:10F9500008500DF106012846FFF700FF48B9BDF831
:10F960000630A380E5800A4B185C092803D005B057
:10F9700030BD0928F7D90320F9E70220F3E708464C
:10F98000F5E70520F3E70020F1E700BF5DCD00209B
:10F990003416060038B54FF6FF73984218BF013091
:10F9A0000D4614BF84B20024FF2C03D94FF6FF7418
:10F9B000204638BD21462846FFF728FF0028F7D10A
:10F9C0000134A4B2F0E70000F8B5074D074E074632
:10F9D00000243378A34200DCF8BD55F8043B3846D8
:10F9E00098470134F5E700BF3CCD0020EDCE002064
:10F9F0007DDF704779DF70476DDF704738B5074CA2
:10FA0000051E04F1080318BF1C4623682BB11A68B1
:10FA100022605B6828469847F7E738BD74CC002021
:10FA200040DF70473FDF70470023435082B04358A8
:10FA30000193019B02B070472DE9F0470D789DF8C6
:10FA400020609DF824A004460F469946002D60D101
:10FA5000D0F8243192F800809BB14FF49271FFF7F7
:10FA6000E3FF012363613B70B04550D1D4F804310A
:10FA7000002B4CD04FF482712046FFF7D5FF0025B4
:10FA80001DE0D0F81C31FBB14FF48E71FFF7CCFFB5
:10FA9000D0F824311BB14FF492712046DFE7137880
:10FAA0009E4207D919F80330C0F81C35137801338A
:10FAB0001370D9E70123BAF1000F03D0C3612846C0
:10FAC000BDE8F0874361CFE7D0F80831002BCBD0F9
:10FAD0004FF48471FFF7A8FFD0F82431002BDAD15E
:10FAE00013789E42C0D9D0F8181509F8031013787E
:10FAF0000133DBB21370721E934205D10223C0F8AA
:10FB0000003201232362AFE79E42FAD1ACE7012520
:10FB1000D5E74FF49271FFF787FF4FF48E71FFF72F
:10FB200083FF4FF48471FFF77FFF9FE72DE9F347D1
:10FB30000C4605464FF4827120461F469046FFF75B
:10FB400073FF4FF49271FFF76FFF4FF48E71FFF761
:10FB50006BFF4FF48471FFF767FF0023012F85F8D7
:10FB6000263085F8233008BF02224FF001030CBF76
:10FB7000C4F80022C4F80032236223602E6846BB1A
:10FB800005F1260A05F12309CDE9007643465246E0
:10FB900049462046FFF750FF0028F5D195F823305D
:10FBA000EBB1D4F8C434C4F8C434C3B113F0010FBA
:10FBB00014BF4FF40240032048F2012213F0020F59
:10FBC00018BF104613F0040F48F2022318BF18465E
:10FBD00006E040F28623AB60AB68C4F80433002033
:10FBE00002B0BDE8F0872DE9F3470C4605464FF417
:10FBF000827120461F4616469DF82880FFF714FFA5
:10FC00004FF49271FFF710FF4FF48E71FFF70CFF66
:10FC10004FF48471FFF708FF0023C4F8003285F821
:10FC2000263085F8233001232362A36095F826202F
:10FC3000974232D9B35CC4F81C3595F826300133AD
:10FC400085F826302B687BBB05F1260A05F12309D0
:10FC5000CDE900783346524649462046FFF7ECFE90
:10FC60000028F5D195F8233023B3D4F8C434C4F870
:10FC7000C434FBB113F0010F14BF4FF40240032052
:10FC800048F2012213F0020F18BF104613F0040FC0
:10FC900048F2022318BF18460DE0B8F1000F01D05A
:10FCA000E361CFE76361CDE740F28623AB60AB68E9
:10FCB000C4F80433002002B0BDE8F08700234350AD
:10FCC00082B043580193019B02B0704708B50246C9
:10FCD0004FF492710068FFF7F1FF4FF484711068E0
:10FCE000FFF7ECFF136801221A6008BD10B5CB7D49
:10FCF0000A464FF4847123B9FFF7E0FFD0F81835B6
:10FD000010BDFFF7DBFF537ED168D0F81805C8544B
:10FD1000537E0133DBB25376F2E70A4610B54FF457
:10FD20008E71FFF7CBFF938A91689BB2C95C938A6F
:10FD300001339BB29382C0F81C1510BD2DE9F0472A
:10FD400093F9005090B00024013D6E46AD00274667
:10FD5000A446A0465FF0000E03E05FEA080EBEEB8B
:10FD6000050EB8EB0E0952F809A051F80E90A9FB48
:10FD70000A9A14EB090457EB0A075CF1000C1EF118
:10FD8000040EAE4501DCC645EBDD46F808403C46B6
:10FD900067465FF0000C18F10408A845DADDB8EBFF
:10FDA000450FDADD46F80840D3F8B03031469847C1
:10FDB00010B0BDE8F08713460A46FFF7BFBFF0B5A5
:10FDC000154689B01C4607460E461A46294668461F
:10FDD000FFF7F1FF23466A4639463846FFF7AEFF84
:10FDE00023462A4669466846FFF7A8FF23466A4627
:10FDF00031463046FFF7A2FF09B0F0BD00EB8101AC
:10FE00000023884200D3704751F8042D43EA52037F
:10FE10000B60D307F5E710B5013A52B2130601D5CE
:10FE2000002010BD50F8224051F822309C4205D8E5
:10FE300002F1FF32F2D24FF0FF30F2E70120F0E79B
:10FE400010B500235CB2A24200DC10BD51F8234083
:10FE500040F823400133F5E7013910B549B2041DDC
:10FE60000A06CBB204D4013954F82120002AF7D075
:10FE700001335BB273B103F18042013A50F82220A2
:10FE8000002022B9013B00EB431318B210BD520809
:10FE90000130F6E71846F9E7002310B51C465AB2C0
:10FEA000914200DC10BD40F823400133F7E7000029
:10FEB000C3F10803DB0070B50133002403A500BFC4
:10FEC0005B1920C940CAAD1B20C0184720C940CAD1
:10FED000B54120C020C940CAB54120C020C940CA90
:10FEE000B54120C020C940CAB54120C020C940CA80
:10FEF000B54120C020C940CAB54120C020C940CA70
:10FF0000B54120C06441B4FA84F0400970BD00BF1F
:10FF1000C3F10803DB0070B50133002403A500BF63
:10FF20005B1920C940CAAD1920C0184720C940CA72
:10FF3000754120C020C940CA754120C020C940CAAF
:10FF4000754120C020C940CA754120C020C940CA9F
:10FF5000754120C020C940CA754120C020C940CA8F
:10FF6000754120C06441204670BD00BFF0B5082235
:10FF700089B00C460646FFF763FFCB6A03930B6B11
:10FF800004934B6B05938B6B0693CB6B0793002706
:10FF900008236A4669466846CDE901770097FFF76E
:10FFA000B7FF082305466A4631463046FFF7B0FFE3
:10FFB000236B0393636B0493A36B0593E36B05447B
:10FFC000CDE906376A46082369466846FFF7A0FF71
:10FFD000082305446A4631463046FFF799FF236AF5
:10FFE0000093636A0193A36A0293A36B0693E36B86
:10FFF0000793054408236A4631463046CDE9047725
:020000022000DC
:100000000397FFF785FF636A0093A36AA26B0193CE
:10001000E36A02930492636BE26B0393CDE90523D9
:10002000236A0793054408236A4631463046FFF7A2
:100030006FFFE36A0093236B0193636B0293236A60
:100040000693A36A0793054408236A46314630465F
:10005000CDE904770397FFF72BFF236B0093636BC6
:100060000193A36B0293E36B0393636A0693E36AC2
:1000700007932D1A08236A4631463046CDE90477A6
:10008000FFF716FF636B0093A36B0193E36B02937F
:10009000236A0393636A0493A36ACDE90537236B4C
:1000A00007932D1A08236A4631463046FFF700FFB2
:1000B000A36B0093E36BCDE90137636A0393A36AF3
:1000C0000493E36ACDE90537636B07932D1A082380
:1000D0006A4631463046FFF7EBFE2D1A0D4C0FD421
:1000E00035B9082231462046FFF795FE01280FD08A
:1000F0000823224631463046FFF7DAFE2D1AEFE795
:100100000823224631463046FFF702FF2D18F7D468
:1001100009B0F0BD581606002DE9F04391B00F4626
:100120001C220021804609A8FFF7FCF901251C22AA
:10013000002101A80895FFF7F5F9394608AA11F939
:10014000046B009533461046FFF7E2FE314608A8DF
:10015000FFF782FE013804B2012C07DC3246694603
:100160004046FFF76DFE11B0BDE8F0833A466846A1
:100170006946FFF720FE10AB601103EB80001FFA09
:1001800084F909F01F0350F8202C05FA03F31342F9
:1001900005D03B46424669466846FFF7CFFD09F168
:1001A000FF3424B2D8E770B5036813F001050646A2
:1001B000144605D013460A460146FFF7A9FE054638
:1001C00021463046FFF71AFE45B104F18042013A5C
:1001D00056F8223043F0004346F8223070BD70B527
:1001E0009DF910401E4623460546FFF761FE38B1D3
:1001F0002346324629462846BDE87040FFF788BEB0
:1002000070BD2DE9F0438BB01446129D15F9046BB7
:1002100000961F46804689462B460246214602A884
:10022000FFF7DDFF02A9129A0846FFF7C4FD129BF3
:1002300002AA41464046FFF781FD129B02AA2146D1
:100240002046FFF77BFD2B464A4639463846009646
:10025000FFF7C5FF129A394602A8FFF7ACFD02A9C5
:100260002B46424608460096FFF7B9FF02A92B46E7
:10027000224608460096FFF7B2FF2B46424621462B
:1002800020460096FFF7ABFF129B224649464846A0
:10029000FFF754FD2B4602AA414620460096FFF781
:1002A0009EFF129B224639463846FFF747FD2B46F4
:1002B0004A46394638460096FFF791FF324602A972
:1002C0002046FFF7BDFD0BB0BDE8F08370B59DF98A
:1002D00010401E4623460546FFF71AFE30B9224657
:1002E00029463046FFF797FD012807D023463246BE
:1002F00029462846BDE87040FFF7DABD70BD2DE9FC
:10030000F0439BB01646229C14F9045B0095984676
:100310000746894623460246314612A8FFF75FFF8B
:1003200012A9229A0846FFF746FD229B12AA3946D7
:100330003846FFF703FD229B12AA31463046FFF7ED
:10034000FDFC23464A46414612A80095FFF7BEFF32
:1003500023464A46414640460095FFF740FF234664
:100360003A4631460AA80095FFF739FF229B0AAAB0
:1003700049464846FFF7E2FC2346324639460AA87A
:100380000095FFF7A3FF229A41463046FFF713FD81
:1003900023460AAA314630460095FFF720FF234640
:1003A0003246394602A80095FFF719FF229B02AAA0
:1003B00041464046FFF7C2FC23464A464146404676
:1003C0000095FFF70CFF229A12A902A8FFF7F3FC91
:1003D00002A923460AAA08460095FFF700FF234614
:1003E0003A4602A90AA80095FFF7F9FE0AA9229B3E
:1003F00012AA0846FFF7A2FC23464A460AA9484625
:100400000095FFF7ECFE2A4602A93846FFF718FDD3
:100410001BB0BDE8F0832DE9F04115468AB00446D3
:1004200088461C22002103A8FFF77CF82E1D95F9B1
:10043000007003232A46414620460293FFF7BBFC87
:10044000334602AA214620460097FFF7C8FE2B46F6
:10045000424621462046FFF771FC0097334605F1DE
:10046000840221462046FFF731FF0AB0BDE8F08143
:100470000C4B1B78062B10D10B4B1B681A070CD1A9
:100480000A4B186800F0F003302B08D000F0E000B1
:10049000A0F14003584258417047002070470120A6
:1004A000704700BFE00F00F0E40F00F0E80F00F02D
:1004B000094B1B78062B0CD1084B1B681A0708D177
:1004C000074B186800F0F000A0F130035842584183
:1004D00070470020704700BFE00F00F0E40F00F00D
:1004E000E80F00F010B9024B01221A60704700BFFC
:1004F0000050004010B50C494A6E042A044611D041
:100500000B6E1344032B02F101024A6688BF043BC1
:10051000182202FB031318460021FFF703F820609E
:10052000012010BD0020FCE740D1002010B504469A
:1005300086B01422002101A8FEF7F4FF6088ADF810
:100540000800FFF74DF92378ADF80600092B0CD809
:10055000DFE803F005051014161B1D0E1F210723ED
:100560008DF8043008238DF80C3001A8FFF72CFA21
:1005700006B010BD0D238DF80430F6E70E23FAE720
:1005800007238DF804300523EDE70F23F3E710234D
:10059000F1E70523EFE706238DF80430A368039302
:1005A000A388ADF80630E0E72DE9F041067904466E
:1005B000407B174603360023834204DB51B93E607B
:1005C0000020BDE8F081226912F833200132164480
:1005D0000133F1E73B68B34229D3237833F00308B2
:1005E00027D10B7022794A708D1C2846A16840F0F3
:1005F000B1FF2279617BA954AB180133627B42457C
:10060000DDDD226912F8382003F8012B226902EBA4
:10061000C801184612F83820496840F09BFF22694B
:1006200012F838200346134408F10108E6E70420D5
:10063000C7E70720C5E738B504461546084631B177
:1006400062682B68934206D3216840F083FF636899
:100650002B60002038BD0420FCE708B5134644F2A7
:100660000102904203BF5A681988986800221CF062
:1006700077F8000030B50B4B1B68012293F864102B
:1006800021338A4204DB405CB0FA80F0400930BD7F
:1006900013F8014B855CA54201D10132F1E700203E
:1006A000F5E700BFF0CA002003681A78302A27D186
:1006B0005A1C02605A7802F0DF024F2A03D102333B
:1006C000036008207047582A03D1023303601020CA
:1006D0007047422A04D0082013F8012F22B970472E
:1006E00002330360022070472E2A07D0A2F138019E
:1006F000012903D9303A092AEED970470A20EBE7DD
:100700000A20704770B5244B0022C3F80025234A05
:10071000516831B12249C3F8081322490420C1F8B5
:100720008000D3F80C55D3F81445D3F80815D3F846
:1007300010054FF0FF36B542C3F8146518BF05F534
:10074000E075C3F80C65C3F80865C3F810651EBFF3
:100750004FF0A043022643F82560651C1FBF4FF0F1
:10076000A04304F5E074022543F82450441C1FBF45
:1007700000F5E0704FF0A043022443F820404B1CEA
:100780001FBF4FF0A04301F5E071022043F82100A4
:100790000023D376536070BD002000409CCB002026
:1007A0008402020000E100E02DE9F04F85B08A46A6
:1007B0000390039C2578284632F0E2FE0746C8B92C
:1007C0002D2D1AD10134012303940193DDF80CB0CF
:1007D000BAF1000F01D0CAF800B003A8FFF764FF18
:1007E0008046002835D1624D00242046294605B0B8
:1007F000BDE8F08F01340394DBE72B2D04BF0134F7
:1008000003940190E2E71846029332F087FEB0F1BC
:100810000009029B20DBC8451EDD404640F01CF964
:1008200022462B4640F082F904460D46484640F0E9
:1008300013F922462B463FF0C3FF013604460D460E
:100840000396039E3378002BDDD1B8F10A0F37D120
:1008500013E000240025F4E7B8F10A0F30D12E2B65
:100860000BD10FF20419D9E9008901360396039ED2
:1008700030783038C3B2092B39D9039B1A7802F08B
:10088000DF02452A1CD15A1C03925A782D2A01D026
:100890002B2A05D12D3A574203F102035741039306
:1008A0004FF000080A20039A1378303BD9B2092987
:1008B00036D9002F39D12F4F0026B8F1000F46D17D
:1008C000039BBAF1000F01D0CAF800309B458AD0D3
:1008D0009BF800202E2A03D10BF1010B5B4582D03F
:1008E000019B002B81D005F100431D467DE740F0C0
:1008F000B3F842464B4640F019F902460B462046F3
:1009000029463FF05DFF002204460D464046494619
:10091000184B40F035FA0136804689460396A6E723
:10092000013200FB08380392BDE7124FC8F10008FE
:100930000026B8F1000FC3D02046294632463B4678
:1009400040F01EFA08F1010804460D46F1E7204682
:10095000294632463B4640F0E9F808F1FF380446A4
:100960000D46AAE7AFF300809A9999999999B93FF2
:100970000000F87F0000244070B58AB00C460146A4
:1009800068461D4637F050FA0022214605A837F088
:100990004BFA684636F059FF044605A836F055FF75
:1009A0008442064621D0039850B1C389A3F5007351
:1009B0009BB2C381C38903F4F0530BB937F000FF36
:1009C000089850B1C389A3F500739BB2C381C38952
:1009D00003F4F0530BB937F0F3FE002C01DB002ECB
:1009E00000DAF5B9A01B0AB070BD002C1BDA039821
:1009F00050B1C389A3F500739BB2C381C38903F4CB
:100A0000F0530BB937F0DCFE089850B1C389A3F559
:100A100000739BB2C381C48914F4F05401D137F040
:100A2000CFFE0020DFE7684636F0F4FF05A836F079
:100A3000F1FFAEE7044A138A9BB223F0410343F06F
:100A400040031382704700BF8C2E00202DE9F04137
:100A5000114B04460F46186810499046002239F0A1
:100A600001FD064637F0AAFB054680B1214600226B
:100A7000304639F0F7FC044660B1014643463A4639
:100A800030462EF0B3F93146204639F06BF928464E
:100A9000BDE8F0810546F6E78C2E00202E530600B7
:100AA00030B587B00A46014601A837F0BDF90025E8
:100AB000DDE90132934205F1010401D2013514D17F
:100AC000049850B1C389A3F500739BB2C381C38955
:100AD00003F4F0530BB937F073FE20202DF01CFA0D
:100AE00014F1FF340DD207B030BD059810B1C05CD1
:100AF0000A28E5D02DF010FA01A8254636F08AFF25
:100B0000D6E70820EAE7000070B50F202BF0CCFFF5
:100B10000028264B46DB264C1871A17D01229A70D5
:100B200000293DD1234DA18204334FF48E71284614
:100B3000A360A275FFF7C2F82146AA60FFF7EDF89F
:100B4000636893B92646A27DA38A9A420ED8A38AE7
:100B50009BB2B3F5807F1BD0164BD3F81C21002A23
:100B6000FBD00122DA600023A37570BDD5F81C31DB
:100B700023B9A38A9BB2B3F5807FF7D1A38A9BB236
:100B8000B3F5807FE0D031462846FFF7C6F8DAE7B4
:100B90000023A3750F210848BDE8704032F06EBBFA
:100BA0001121F8E700229A70DFE700BF01D300208F
:100BB0009CCB0020002000407A18060030B58BB096
:100BC0000D46019009B100230B602022002102A8EC
:100BD000FEF7A8FC002202A901983BF00FFCD0B15F
:100BE0000024029B039A23F07F43033323F0030383
:100BF000203352B11C44032202A901A83BF02CFC73
:100C00000028EED120460BB030BD002DF3D02A686D
:100C100013442B60EFE70446F4E730B58BB04FF494
:100C2000DA242022002102A80194FEF77BFC002296
:100C300002A920463BF0E2FB70B1032202A901A801
:100C4000DDE901543BF008FC0028F6D124F07F4494
:100C500023352C4424F00304C4F5EC200BB030BD44
:100C600084B02DE9F0438BB012AC199F1B9D84E832
:100C70000F00FC1C002324F0030420340193984649
:100C8000019E002E36D030463BF0BCFB80460198DA
:100C90003BF0D2FB064680B1019BC21A94420CD9AC
:100CA000FB1A0344984508D9B4F5007F05D2002209
:100CB00002A93BF0A3FB00B901969DF8683012AE83
:100CC00047EA03670FCE03AC0FC496E8070084E839
:100CD000070020220199029702A820F08DFC35B16F
:100CE00002AC0FCC0FC594E80F0085E80F00019E01
:100CF00020363CE04FF4DA230193B146012202A9E9
:100D000001983BF07BFB88B1039A129B9A4207D172
:100D10001C2212A903A840F00FFC08B9DDF80490CA
:100D2000002202A901A83BF097FBECE701983BF0F9
:100D300069FB844221D901983BF07EFB012301909D
:100D40000198E0B9B9F1000F0CD0012202A9484680
:100D50003BF054FB0422002309EB020103A8039398
:100D600020F04AFC019888B9B8F1000F13D0304642
:100D70000BB0BDE8F04304B070470023E0E7002B60
:100D8000BCD13BF03FFB8442B8D8DBE73BF03AFBF9
:100D90008742E9D874E73BF0A6FD80460028E6D0FC
:100DA000002301936CE7000070B5044637F006FAA3
:100DB0000546B0B120460022184939F053FB0446DD
:100DC00036F0CCFF78B900255CB1E389A3F5007358
:100DD0009BB2E381E38903F4F05313B9204637F063
:100DE000EFFC284670BD00220D49204639F03AFB41
:100DF00006460028E7D00B492FF06EF9F389A3F5DA
:100E000000739BB2F381F38903F4F0530546002B82
:100E1000DAD1304637F0D4FCD6E700BF8C17060095
:100E200032620600961706000C4A002330B41146C1
:100E3000184640F6C41401EB03151032E8819D1CDE
:100E40000133A34222F80C5CF5D149F63443012268
:100E5000C852034B1A8030BC37F036B8AC2E002095
:100E6000AA2E002070B586B015460C460022014619
:100E700001A836F0D9FF2E46DDE901239A4210D3AE
:100E8000049850B1C389A3F500739BB2C381C38991
:100E900003F4F0530BB937F093FC00232370AD1B20
:100EA0000DE07EB9049850B1C389A3F500739BB2DD
:100EB000C381C38903F4F0530BB937F081FC284692
:100EC00006B070BD059B03B19B5C04F8013B01A813
:100ED00036F0A0FD013ECFE737B501230093002394
:100EE0001A460A49044637F06DFF05465CB1E389AE
:100EF000A3F500739BB2E381E38903F4F05313B9C4
:100F0000204637F05DFC284603B030BD9D17060033
:100F1000F8B5858907460C4695B31A4B013D03EB9E
:100F200005152846EB8903F500739BB2EB8139F078
:100F30002DF8EB89A3F500739BB2EB81EB8903F4E9
:100F4000F053461C13B9284637F03AFC304637F0C8
:100F50000EFC214638F02EFC044680B1014638468E
:100F600039F08AF8E389A3F500739BB2E381E38942
:100F700003F4F05313B9204637F022FC701CF8BD7F
:100F80000126E3E7AC2E002038B5074C2578002376
:100F9000EDB20246194623703AF0D6FD257003489B
:100FA000BDE838402BF0B0BEA82E00206BB4060080
:100FB000002370B50B6005460E4637F0D3FA0446A1
:100FC00010B90025284670BD294638F08FFA05462D
:100FD00068B9E389A3F500739BB2E381E38903F465
:100FE000F053002BEDD1204637F0EAFBEAE720462C
:100FF00036F012FF3060E389A3F500739BB2E38102
:10100000E38903F4F053002BDCD1ECE7F8B5044698
:101010000E46174640F0D8FA0146204637F07EFBD0
:10102000054650B3164B1C88A4B224B100221146C9
:101030002DF094FE0446EB89A3F500739BB2EB817F
:10104000EB8903F4F05313B9284637F0B9FB3B465C
:101050003246002120462DF04BFE05465CB1E38967
:10106000A3F500739BB2E381E38903F4F05313B952
:10107000204637F0A5FB2846F8BD0446E7E700BF49
:10108000AA2E00202DE9F843394F03791C2202FBD8
:1010900003720646506820B132684FF40174C2F8FA
:1010A00008431C2202FB0373DA7D52B11A7E002A28
:1010B00041D020B133684FF40172C3F804231120EA
:1010C00037E00120D875D9605A761A7635791C2315
:1010D00003FB05739B7E1BB912B93046FEF7F6FD84
:1010E0004FF01C0808FB05783068D8F80430002B56
:1010F00035D14FF4A271FEF7E1FDC5EBC50907EB51
:1011000089093068D0F82431D0F80821D0F844415A
:10111000A2B90CB9002BF4D01C2202FB05750022E9
:10112000EA750BBB14BBA97E33680122A9B11A6012
:101130000020BDE8F88319610122C6E7002BEBD13E
:10114000002CE9D14946FEF7D1FD98F8193098F8FE
:1011500017209A42D5D82346DEE75A60E8E74FF4D5
:101160000173C0F80433E3E70320E2E70F20E0E770
:101170009CCB00200A490B4808B5FFF783FF0146C6
:1011800010B1094832F07AF808490648FFF77AFFAB
:10119000014620B10648BDE8084032F06FB808BDEE
:1011A00001D300204C1606003418060002D300209C
:1011B0005718060038B50022054639F053F90446A1
:1011C00098B100231A46014628462DF00FFEE38908
:1011D000A3F500739BB2E381E38903F4F05323B9D1
:1011E0002046BDE8384037F0EBBA38BDF0B54FF0D7
:1011F00080530220D3F85014D3F85424284BC3F85A
:1012000004032848C3F80403274B93F800E093F83D
:1012100001C09F78DE781D795C7998794EEA0C03DD
:101220003B4333432B4323430343204B2AD083F8D0
:1012300000E083F801C09F701E715D719C71D871D0
:101240001D789C785A785E79586885EA0401514087
:1012500081F08801D970197971409E797140DE79E9
:101260007140197212020321597242EA05420C4B75
:101270002243C3F8942500BA4422C3F89005C3F86A
:10128000A025F0BD080A1970090C9970110A1A718D
:101290005971110C120E58709971DA71D0E700BFB4
:1012A000005000408000080014D00020FFCF002034
:1012B0002DE9F0471546814615F8014B884644F460
:1012C00080740F2701F1510A464612E0220606D526
:1012D000D9F80C303A463146484626F0C0FD640045
:1012E000E30348BF15F8014B06F1010648BF44F47B
:1012F00080745645EAD10137312FE5D1BDE8F0873A
:1013000038B50B4C0B4D2B785BB130F0DDFF40B99D
:1013100014F1FF34F7D208490420BDE8384031F019
:1013200059BC002CF7D030F0CFFF0028F3D138BDE6
:1013300080841E00F3D200201517060070B5EFF36D
:10134000108672B60D4A94680123A4B993600C4BC1
:101350000C4DD3F8801029401160C3F88050D3F8A9
:10136000841051604FF0FF32C3F88420047006B936
:1013700062B6002070BD0370F9E700BFE4D2002020
:1013800000E100E0FC06FFBC10B588B012788DF8D3
:101390000C20CDE90001FF22002102918DF80D20E3
:1013A00001214FF6FF72104C8DF81C10ADF80E2085
:1013B0008DF810302BF018F870B130F085FF58B967
:1013C00014F1FF34F6D20949042031F003FC6846D9
:1013D0002BF01AF808B010BD002CF4D030F074FFD8
:1013E0000028F0D1F3E700BF80841E0073170600C9
:1013F00073B52F4C637E0546002B56D123680BB185
:101400000123637695E80F002A4E86E80F00A27E3E
:10141000637FFF2A23F0030363771FBF01239340F9
:101420004FF0A042C2F80C352A6822B102F06043A6
:10143000B3F1005F06D1AB684BB103F06043B3F189
:10144000005F04D000236376102002B070BD1A4BF9
:101450002979C3F84425C3F848152A7BA968C3F83D
:101460003415C3F83825154A00201060126801921F
:10147000019AC3F850050122C3F840051A6121689A
:101480001A4671B9D2F81831002BFBD0A27EFF2A80
:1014900005D0012393404FF0A042C2F80835002048
:1014A000D3E74022C3F80423CFE71120CDE700BFE4
:1014B000E0CB0020E8CB0020003000401831004095
:1014C00037B50B015BB249B2044643EA01008DF81F
:1014D00004001A4D50B20343120152B28DF8053088
:1014E0002B78114302438DF806108DF8072013B3B3
:1014F00002AB03EB941302AA13F8040CC4F3011318
:10150000134413F8043C43EA00201FF0D1FF2B786A
:101510008BB102AAC4F3810304F0030413441444FE
:1015200013F8040C14F8043C43EA002003B0BDE8AF
:1015300030401FF0BDBF03B030BD00BFF2D200206D
:10154000C30914BF13020B0270B510F0400F0D4613
:101550000CBF29461146194306461320144620F0B5
:1015600033F9B1064CBF23022B0216F0100F14BF43
:10157000214629461943132020F026F932074CBF93
:1015800023022B0216F0040F14BF214629461943EB
:10159000132020F019F9B3074CBF2102290216F0DD
:1015A000010F08BF2C4621431320BDE8704020F0F6
:1015B0000BB900002DE9F047FF2705463C460426FD
:1015C0004FF6FF78296911B9002E61D051E02868E3
:1015D00028F0B7FD064600284BD168690378002B38
:1015E0005ED0C27AE52B02F03F0247D022F0200104
:1015F000082943D00F2A46D159063DD503F0BF0430
:10160000EB88477B2B84437BBB4237D10378EE6961
:10161000DFF890E003F03F03013B0D2253434FF00E
:10162000010C00211EF8019B00EB090292F801A0B9
:1016300010F8092042EA0A22BCF1000F20D03E2B0C
:101640001CD826F813209446013301310D29E9D125
:101650000278520604D53E2B10D8002226F813201B
:10166000013CE4B20021284628F020FF064600286D
:10167000A8D000232B610CE0A342C4D0FF24F1E7E3
:101680004245E2D0FAE73CB927F026F9B84203D147
:1016900000263046BDE8F0874FF6FF732B84F8E74D
:1016A0000426E6E73E1606002DE9F047ADF5127D6B
:1016B00080460CA80D4622F0BDFF30F00DFEC0F3B1
:1016C0000E02002302F5FA620221404622F0F6FEE5
:1016D0004045F2D1AA4A1388013312AC9BB2138061
:1016E0005BBA238001234FF480722946638052A89D
:1016F0000023C4E901233FF06FFF52A83FF064FFCD
:1017000015AB1FFA80FA0DF5A4791D4649460A78F3
:101710000F4601312AB12E2AF9D1A7EB0906B6B23C
:1017200001E05646174603F8016B5EB11846324693
:1017300049463FF051FF03463344002F40F0938069
:1017400003F8017B01225A70DA7000211A1D19700A
:101750009970121B3523009392B20DF1420321467A
:10176000404622F0F7FA20F0CDF910F580130293ED
:1017700041F100030393404622F0A2F906460028F7
:1017800000F0EF80B0F5807F28BF4FF480760DF138
:101790001603B2B221460093404606AB22F0EAFBA4
:1017A000404622F0ADFB0023ADF81E30227863786E
:1017B000E07894F8058003EB0223ADF81C30A378A1
:1017C00000EB032080B2020444BF01238DF81E30D9
:1017D000C0F3C3238DF81F30430544BF01238DF8A8
:1017E0002030870544BF01238DF82130C60544BF52
:1017F00001238DF82230010644BF01238DF82330E8
:101800002379E779227A08EB0328A37907EB0327EA
:10181000637A03EB0223ADF82A30A27AE37A00F070
:101820000F061FFA88F8BFB203EB02238DF824607D
:10183000ADF82680ADF82870ADF82C304FF00009D7
:101840001FFA89F3434515D3DFF838814FF00009BB
:101850001FFA89F39F421AD8B6FA86F040090DF5AF
:10186000127DBDE8F087721CF643B24491441FFA22
:101870008AFA4BE7294652AA2046FDF77BFE421C16
:101880001ABF2D180435002509F10109D8E752AA1D
:1018900029462046FDF76EFE431C03D1002509F1C1
:1018A0000109D5E729182A5C4B7803EB02239BB288
:1018B000013B01F10A050E2BF1D801A252F823F0E9
:1018C000FD1802002F1902009F1802009F18020045
:1018D0002F1902003F1902002F1902002F190200D0
:1018E0002F1902009F1802009F1802002F190200F2
:1018F0001B1902009F1802002B1902008B7A88F82E
:101900000030CB7A88F801300B7B88F802304B7BB3
:1019100088F8033001F10E05C1E701F10B028B7A63
:10192000D05CD51801300544B9E701F10C05294612
:1019300052AA2046FDF71EFE411CF4D1AEE752AA82
:1019400029462046FDF716FE421CA7D0054452AAA0
:1019500029462046FDF70EFE431C9FD00544143552
:101960009DE74FF47A701AF015FC20F0CBF8DDE912
:10197000022382428B41BFF6FEAE30466FE700BFC6
:10198000A42C00207C2E002010B5074A002332F83A
:10199000024B8C4203D1184100F0010010BD01330D
:1019A000082BF4D10020F9E7F8CA0020F0B5224B4B
:1019B0009F7C1C4600221D46D6B2B7420ED895F831
:1019C00078701D4C0022D6B2B74216D895F8DE507A
:1019D0000022D4B2A54220D800200DE0B4F814C0F3
:1019E000844502F1010204F10A04E5D142F64D23D7
:1019F00001200B808870CE70F0BDB4F87AC06045CD
:101A000002F1010204F10A04DDD142F64D230B80FC
:101A100002238B70CE700120EEE7B3F8E060B04295
:101A200002F1010203F10A03D3D142F64D230B80E8
:101A300003238B70CC70EEE76CCD002010B50C4CFE
:101A4000226886B0034682B104208DF8040008683D
:101A5000D989ADF80C10123333F8021C0290ADF89E
:101A60000E10049301A92046904706B010BD00BF98
:101A70006CCD00207FB54B89022B0FD1094A13682A
:101A800063B1097B0068029011F0010F14BF0221BD
:101A900003218DF80410104601A9984707B05DF89E
:101AA00004FB00BF6CCD002070B50D4D002435F84F
:101AB000026B964210D10122A240D2B2D543EDB2C0
:101AC000014410F8014B2BB11443884200F8014C3B
:101AD000F7D170BD2C40F8E70134082CE7D1F8E7C6
:101AE000F8CA002070B50023084C1A4641FA02F5E6
:101AF000ED0706D504EB420600EB4305B688AE8041
:101B000001330132082AF1D1036070BDF4CA00200C
:101B100010B586B004460022684619F0DFFF204663
:101B2000009919F087FD204606B010BD38B5012395
:101B30000B7004460D4636F011F988B100220B49AE
:101B4000204638F08FFC10B139F013FC2870204685
:101B50000022074938F086FCBDE8384039F0A2BAC7
:101B60002046BDE8384038F011BA00BF081706001B
:101B70000D170600084B5A6E013A5A6622B90749FA
:101B80000A7822F002020A701A6E0132042A08BF93
:101B900000221A66704700BF40D100205ECD0020B1
:101BA00030B5044685B00D46102200216846FDF789
:101BB000B9FC237A012B0AD0022B0ED06368019363
:101BC000236829469B686846984705B030BD23695D
:101BD0000293A38AADF80C30F0E70123A2898DF8B7
:101BE0000030E389ADF80A20D31AADF80830E5E7F4
:101BF00028DF704729DF704738B51C4B5A6E1946ED
:101C00005AB31C6E182202FB04331A7A012A07D039
:101C1000022A23D018460921BDE83840FFF7C0BF8B
:101C20001825D88A9A8A05FB0414D4E90314121AD9
:101C3000B2F5806F4FEA80000144B4BF92B24FF416
:101C400080622044FFF7D6FF11280BD1084A137891
:101C500023F0020343F00403137038BD9889FFF7A3
:101C6000C7FFF1E70028F8D0D4E700BF40D100203B
:101C70005ECD0020054A137813F0060F04D143F01F
:101C800002031370FFF7B8BF704700BF5ECD00209E
:101C90002DE9F3411F4B1B781746DA0706468846A5
:101CA0002BD51D4D1D4B9D4229D31D4B9D4226D248
:101CB00039B330B341EA00039B0724D12B68984223
:101CC00023D36A6800EB87039A421ED3FFB101A8B1
:101CD000FEF710FC78B1019B0024C3E90054019B7E
:101CE00001221A72C3E903869F82FFF7C3FF2046D1
:101CF00002B0BDE8F0810720FAE70120F8E70220F2
:101D0000F6E70320F4E70620F2E70520F0E70420D9
:101D1000EEE700BF5ECD0020382E0020382E0020D8
:101D2000482E002038B5074B074A59689488106838
:101D30004A880332032592B200EB84001D70FFF73E
:101D4000A7FF38BD60CD0020E4D1002010B50122EE
:101D50000C460649FFF79CFF28B9054901EB041121
:101D600001238B7310BD0E20FCE700BFBC170600DB
:101D7000A0D0002008B502220149FFF789FF08BD65
:101D8000C017060008B5034B034918680222FFF785
:101D90007FFF08BDE4D10020C817060073B51B4BB8
:101DA0001B78DB0705462BD5194E1A4B9E4229D3CB
:101DB000194B9E4226D238B3C0F30B04D4B9336812
:101DC000984219D3726800F580539A4214D301A83F
:101DD000FEF790FB90B1019BC3E90064019B0222D6
:101DE0001A722D0B01229D811A82FFF743FF2046B4
:101DF00002B070BD0620FBE70520F9E70720F7E7F2
:101E00000120F5E70220F3E70320F1E75ECD002093
:101E1000382E0020382E0020482E002010B50B4C04
:101E20000B4B628803EB02139A892AB95868FFF7B3
:101E3000B5FF0423237010BD05232370054B022238
:101E400018689A80FFF7AAFFF5E700BF60CD002071
:101E5000A0D00020E4D1002008B5074B191D5888F8
:101E6000FDF70CFC18B1BDE80840FFF75BBFBDE80B
:101E70000840FFF7D3BF00BF60CD002060DF704790
:101E800010DF7047002208B511461AF069FC000007
:101E90002DE9F347254B1B681BB1984730B3FFF77B
:101EA000F1FF234B1B7803F0FF07FBB1214D224EBE
:101EB0002C68DFF88C90B4FA84F46409B046337867
:101EC000A3B901A8FDF7BEFB052812D00028E6D172
:101ED000019B0BB9FDF792FD184B1B680BB10198E4
:101EE00098474CB10124EAE7002CFBD002B0BDE8D2
:101EF000F087002CFAD13C46DFF848A098F8003073
:101F0000002BF3D1B9F80030ADF80430DAF8003026
:101F100001A91846FDF794FB0528E5D00028BED19D
:101F20002A6818469047002CE8D1C8E74CCD00201D
:101F3000E1D100202CCB0020E2D10020ECD1002008
:101F400028CB0020DCD2002010B5084B9A685AB18B
:101F500050B9EFF3108172B6054A1C6814605C68D2
:101F60005460986001B962B6002010BDE4D2002030
:101F700000E100E02DE9F3411D4F7B6806460D4668
:101F80009BB304292FD943697BB3437C0024012BE5
:101F90000DF107000CBF8846A0468DF80740FFF7FB
:101FA000CDF90DF10600FDF7F7FBD0B10123037069
:101FB000104B4660D3F80435C0E90484C0E902350B
:101FC0009DF806307B709DF80700FFF7BDFF24B930
:101FD000094B4FF48012C3F80021204602B0BDE83F
:101FE000F0810424EFE70724F7E70824F5E700BFB2
:101FF0001CD000200010014000E100E02DE9F34179
:10200000CE0801F007044FF0010808FA04F4855DDA
:10201000E4B22540074613D10DF107008DF80750B3
:10202000FFF78CF9BB5D9DF807001C4202BF1C4303
:10203000BC554546FFF788FF284602B0BDE8F08151
:102040000025F9E72DE9F3478146002701261FFA0D
:1020500087F84FEAD80A08F0070406FA04F419F8DA
:102060000A50E4B2254008D00137B7F5807FEED1A1
:10207000B846404602B0BDE8F0870DF107008DF884
:102080000750FFF75BF919F80A309DF807001C426A
:1020900002BF1C4309F80A400125FFF755FF002D38
:1020A000E2D0E6E773B50546B8B1C1F3C70401F065
:1020B000070301269E40035D33420ED000230DF13D
:1020C00007008DF80730FFF739F92B5D9DF8070001
:1020D00023EA06062E55FFF737FF02B070BD000059
:1020E00038B50A4B1A687AB15D686DB1FF280BD01C
:1020F00084B221462846FDF789FB28B121462846AF
:10210000BDE83840FFF7CEBF38BD00BF2CD200205D
:102110002DE9F74F9846531E072B81460F4615466B
:1021200000F2BB80FF2800F2B88001465E48FDF750
:102130006DFB0646002800F0B08039464846FDF7A2
:10214000B7FB044600283ED0C3689D4247D805D25D
:102150005FFA85F9E368207C994543D394F81090A1
:10216000B9F1FF0F40F09780504B1A689B46002A48
:1021700041D14FF6FF732380A3700023C4E90133DC
:10218000E360238A03F4784343F0FF0323821120A2
:1021900084E0237C1844C0B2FFF7A2FFE3685FFA33
:1021A0008AF083420AF1010AF3D84FF6FF732380C5
:1021B000A3700023C4E90133E360238A03F4784366
:1021C00043F0FF032382FF214FF6FF70FDF770FB02
:1021D00004460028DBD0A0F800908770BEE74FF0DF
:1021E000000ADBE74844C0B209F10109FFF778FFB4
:1021F0005FFA89F9AEE75B68002BBAD00023DBF801
:1022000008205FFA83FA924502D34FF0FF0912E0EB
:10221000DBF8040060B351460193FFF7EFFE019B2A
:1022200030B3B9F1FF0F08BFD146AAEB090A0AF192
:10223000010AAA4521D1B9F1FF0F84F8109098D076
:10224000E560207CFDF7F2FA58B305EB85052D011A
:10225000ADB2AD0888F80270C8F80400A8F80050C4
:1022600026B1082F02D1AD00063D8580002015E083
:10227000B9F1FF0F0CD14FF0FF090133BFE748461A
:10228000019309F10109FFF72BFF019B5FFA89F91F
:10229000D145F4D3EFE70026D2E7072003B0BDE82D
:1022A000F08F0320FAE700BFF8D000202CD20020E6
:1022B00038B504460025E368AB420ED84FF6FF73ED
:1022C0002380A3700023C4E90133E360238A03F46D
:1022D000784343F0FF03238238BD207C2844C0B2FA
:1022E000FFF7FEFE0135E6E737B5FDF7E1FA0546F3
:1022F000A0B144682CB10A4B01941B789B0706D40B
:1023000003242846FFF7D4FF204603B030BD01A8C0
:10231000FDF79AF904460028F3D0F1E70524F3E726
:102320005DCD0020FF2810B5044609D801460548B8
:10233000FFF7B8FE21460448BDE81040FFF7B2BEE3
:1023400010BD00BFF8D0002018D1002013B50DF14A
:1023500006010446FDF7BAF970B1BDF80620084B36
:1023600003EB02139A894AB1A17A39B1013A0020EC
:102370009A81A07202B010BD0A20FBE70620F9E79F
:10238000A0D0002037B50D460DF106010446FDF73B
:102390009DF988B1BDF80620084B616803EB021374
:1023A00000209A8901329A81296063680C336B603E
:1023B0000123A37203B030BD0A20FBE7A0D00020A8
:1023C0002DE9F043DFF88480D8F874E0BEF1030F04
:1023D0000F46944635D81C4E756CC1F108039D42DA
:1023E0002FD8D8F8704074441C2304F003048146AD
:1023F00003FB0484B9E80F000FC499E807000EF14D
:10240000010384E80700C8F87430C7B1336C2B446B
:1024100003F0070306EBC303002206F138040CEBBC
:10242000C20103C9A34202F1010283E8030014BF01
:102430000833054B9742F2D1736C1F447764012037
:1024400000E00020BDE8F08324CC002024D0002050
:102450002DE9F0411C46184B1B789B0706460F469A
:10246000154627D5DFF85880A3880BB10A201FE056
:1024700098F800302BB92146A088FDF7FFF820B965
:102480002060A3880133A380EEE723681EB19988FA
:1024900032889142EFD11FB119883A889142EAD12E
:1024A0009B682B6023686B60044B1B892B81002089
:1024B000BDE8F0810220FBE75DCD002060CD00206B
:1024C000A0D0002030B587B04CF2070305460C467B
:1024D000ADF8043003AA0F4B01A90020FFF7B8FFA5
:1024E00010B1002007B030BD01A903A8FFF74AFFD3
:1024F0000028F6D10723A370019B5A882280029AF4
:1025000062609B8803F580432B8003A8FFF71EFFC2
:102510000120E7E750CD00201FB50023A0F5804043
:10252000A1F58041CDE90233ADF80400ADF8061005
:1025300002AB0DF1060101A8FFF78AFF002818BFC2
:10254000052005B05DF804FB2DE9F04102230B8066
:10255000164B00251C6800F5805E2F4608304FF6AC
:10256000FF7870450AD305B11C6002B11770BDE851
:10257000F08101270EE0344601250BE006680136A4
:10258000F1D086884645F4D00688002EF1D08668C2
:10259000A642F0D8468806F1030C00EB8C00B1F897
:1025A00000C00CF1030C66440E80DAE7E8CE002090
:1025B00070B5064D0646002455F8043B0BB1304675
:1025C00098470134082CF7D170BD00BF00CC002023
:1025D0002DE9F047AA4C266F1C2707FB06F586B0AD
:1025E000635D013B8046052B00F22A81DFE813F092
:1025F0000600640064001D011D017E0130B1A14A86
:10260000137823F00103137001201FE025442B7978
:10261000032B15D8DFE803F002072C34FFF7B2FBD9
:1026200001232B7109E0984D2B78022B40F03C825E
:102630006868FFF79FFB00232B70002800F0F080F4
:10264000904A137823F0010313700E201C23734368
:10265000E218E35C0290023B012B00F232818B4BCB
:10266000907D196C5A6C0144121A19645A6428E15D
:10267000874F3868FFF792FB0223BB800023D0E727
:10268000834FDFF804823868FFF774FB814BD7F87B
:1026900000E05B88B7F804C01B0108EB0302516837
:1026A000A2F808C0C2F804E00222BA800022396011
:1026B00008F803202A71C0E707FB0647724BB7F8FA
:1026C00012A04FEA0A1A03EB0A029946118960B177
:1026D000FB8803F103088844C3F57F435189A2F8BE
:1026E0000880FD330B4453818EE7536803EB810868
:1026F0003B7C062B00F29780DFE803F02D733C4D06
:102700001F84040041F61D501C2303FB0643D144E3
:10271000DB88B9F80810DA1C0A44A9F80820C3F5C8
:102720007F43B9F80A20FD331344A9F80A3041F673
:102730001D53984200F0C38088E75748574900234B
:1027400043601C2303FB06439B690360FCF7BEFF49
:10275000002800F04C81291D012221444046FFF74A
:1027600097FA1C2303FB064302221A74002857D051
:102770000E20C9E705F10C010122214408F10800EF
:10278000FFF786FA1C2303FB06439A7D002A14BF39
:1027900003220122E9E73D4B5A6C002A00F08C81AC
:1027A000196C1C2505FB0645481C00F0070003EBCF
:1027B000C1071864A88A53F83110013A5A6408EB2B
:1027C0008000BA88FFF764FAAB8ABA881344AB82F8
:1027D000AB7D013BDBB2AB75002BC7D101232B7462
:1027E000C4E705F108010122214408F10400FFF7C4
:1027F0004FFA1C237343E25C032A0CBF0522062216
:102800002344B2E7254B1988234B5868FFF79EFAFB
:102810001C2303FB064306221A7400287FF474AFBE
:1028200006B0BDE8F0870F206EE700287FF4ECAE1D
:1028300007FB06473B79012B32D01BB1022B3ED060
:102840000F2003E7CDE90200FB6801930DF10201BF
:1028500001A8FCF73BFF80B10298BDF80210838805
:10286000FB8003883B81FFF771FA1C2303FB0643BF
:1028700002221A710028D3D059E70A20F5E700BFD9
:1028800024D000205DCD0020A0D0002024CC00204A
:10289000E4D1002060CD0020802E0020F0D2002066
:1028A000864FA81D3B4601AA41462044FFF7D0FDB4
:1028B000B8B9B9880298FFF749FA0A28DAD1002393
:1028C00002931C2303FB06F2A25C013A052A00F2E4
:1028D000B580DFE812F08E009200A000CB00D5009A
:1028E000E1000A28C7E90088E9D020E700287FF442
:1028F0008BAE734BDA7AAAB1D8721A78013A062AEB
:102900009ED801A151F822F0B9290200B329020092
:10291000C9290200CF29020041280200D52902005E
:10292000E52902001A78072AE7D801A151F822F018
:1029300051290200FB280200FB2802006D29020039
:10294000812902009F2902009F29020069290200B3
:102950001A8901321A8100225A80DA72594A127891
:10296000B2FA82F252099A72012207E05649586877
:102970008A884088033202448A8002221A70BCE7A7
:102980005D88504A504902EB05120868556850604E
:102990008888108102228A800D600622EEE70722D5
:1029A000ECE7484900229A728A8942B9897B31B1A1
:1029B0005A80FFF751FA5DE79A7A002AF1D1002296
:1029C0001A705A805A607AE7FFF7ACF952E7FFF7BE
:1029D00025FA4FE75A883B4B03EB02135868FFF781
:1029E000C9F947E700225A60FFF7CCF942E70A200D
:1029F0002CE600238DF8043020E003FB064301227F
:102A00008DF804201A89ADF810209A88ADF81220AC
:102A1000DB68039312E003FB064302228DF80420D7
:102A20001A89ADF810209A88ADF81220DA681B7C5C
:102A300003929A1F534253418DF8143001A8FFF7B7
:102A4000B7FD206F1C22002102FB0040FCF76AFD4D
:102A5000636F1BB3226F013202F00302013B226756
:102A60006367DBB10020FFF7B3FDD9E603FB064344
:102A700003228DF80420DA88ADF810201A89C5E702
:102A800003FB06430422DB88ADF8103000238DF8E9
:102A90000420ADF81230D1E70523ABE70B4A1378D9
:102AA00023F004031370BBE6084A137843F00203D3
:102AB00023F00103137002E71368FFDEF8D2002051
:102AC00060CD0020A0D00020E4D100205DCD00200A
:102AD0000846FFF77DBD0000054A137813F0040097
:102AE00004D143F004031370FFF772BD704700BFB9
:102AF0005DCD0020F0B51C463D4B1B789E0789B08C
:102B000007460D466FD509884FF6FF7399426CD082
:102B10006B88002B69D06968B5F808C000239C4514
:102B200003D8BAB9164604310AE051F833008007D9
:102B300057D10133F3E731F83200304486B2013225
:102B40009445F8D80DF102013046FCF707FE28B194
:102B500009B0F0BD13885688ADF8023000238DF817
:102B60001430BDF80230ADF816300323ADF818303C
:102B7000204B8DF804401A6829898DF81A1001320B
:102B80001A602B88ADF80C30032C6B88ADF8083038
:102B900004BF04238DF81430049208BF3B686A68B0
:102BA00008BF0793002401A8ADF80A60ADF80E40F5
:102BB000FFF706FC50B9BDF802200F4B03EB0213E0
:102BC00058890338801B58810820C1E7049B3B606B
:102BD0000A4B7C601B89BC723B81FFF77DFF20465E
:102BE000B6E70320B4E70220B2E70420B0E700BF55
:102BF0005DCD0020E8CE0020A0D0002060CD0020D8
:102C000030B58BB0FF28044601921D4645D88B781D
:102C10001846FCF723FE00283FD04A6802920A8833
:102C2000ADF80C20A4F58042ADF81C20A3F580423D
:102C3000ADF81E2002AA08920122ADF82420194600
:102C400004AA2046FFF768FC0528019A0ED102234A
:102C500052B907A904A8FFF74DFF07281FD010D8C5
:102C6000B0B103200BB030BD01AAF2E732B10E4B78
:102C70001B789B0702D501A8FCF7E6FC0323002282
:102C8000E7E708280DD00E280CBF11200320E9E744
:102C9000002DE7D0049B2B60E4E70720E2E78620C5
:102CA000E0E71120DEE700BF5DCD00201F4B204A8A
:102CB0001B6800BF00BF00BF00BF00BF00BF00BF58
:102CC00000BF93422FD000BF00BF00BF00BF00BFB6
:102CD00000BF00BF00BF00BF00BF00BF00BF00BFFC
:102CE00000BF00BF00BF00BF00BF00BF00BF00BFEC
:102CF00000BF00BF00BF00BF00BF00BF00BF00BFDC
:102D000000BF00BF00BF00BF00BF00BF00BF00BFCB
:102D100000BF00BF00BF00BF00BF00BF00BF00BFBB
:102D200000BF00BF00BF0138C3D17047A82C0020EE
:102D30000024F40073B5154E736805461BB3436950
:102D40000BB3002404740DF107008DF80740FEF763
:102D5000F5FA0DF10600FCF71FFD90B10223037098
:102D60009DF80630456073709DF80700FFF7ECF89A
:102D700024B9074B4FF48012C3F80021204602B05B
:102D800070BD0424F0E70824F8E700BF1CD0002041
:102D900000E100E02DE9F8432649274B0025C1F862
:102DA0004051C1F84451C1F84851C1F84C51C1F8E3
:102DB0000051C1F804511B68002B39D0D1F80445EB
:102DC0001E49DFF88C800968641A24F07F442F467E
:102DD0001A68A24217D8A41A15441A7CDE6982B177
:102DE000D8F800901F74D3E90521B9F1000F06D07F
:102DF0001046C84728B1FFF745F83346E8E70846CC
:102E00009047002EF9D10E4A0E4B11781B788B4259
:102E100005D10133DBB2022B08BF002313701278F7
:102E2000094B43F82250094B4FF48012C3F800219C
:102E3000BDE8F88300100140E0D20020FCD1002062
:102E4000F9D10020F8D10020F0D1002000E100E00D
:102E500048CD00200D4B0E494FF4003210B5C3F899
:102E6000802001244FF48033C1F848332F20C1F86B
:102E700008334C60FFF71AFF064B8C602F200021AF
:102E80001960FFF713FF044B197010BD00E100E05B
:102E900000100140FCD10020D9D100202DE9F04FD5
:102EA000B64AB74913780978B64D85B09942D5F836
:102EB0000080019500F095800133DBB2022B08BF42
:102EC000002313701278B04B53F82260019A08EB7C
:102ED000060323F07F4313600127AC4BAC4A18680C
:102EE0000290AC48117890F800904FF0000CE24648
:102EF0005078884278D1BCF1000F02D0A54981F802
:102F00000090002F40F0BB801F6802997F1A18BF05
:102F100001270020196802919E49039191F800E071
:102F200000244FF00108002840F0AD8092F8019095
:102F3000D2F804C092F802A01178494540F0C1804F
:102F40001B68029A9A4201D1002F44D0002B00F056
:102F50001281D3F80090904C019BD4F80465196855
:102F60008E4F751A3B7825F07F450335A3B94FF492
:102F70008033C4F84433C4F80433894B4FF400322F
:102F80004FF00108C3F880212F201A60C4F8008098
:102F9000FFF78CFE87F80080A9452CBF49444919EA
:102FA00021F07F41C4F84015D4F804359B1B23F071
:102FB0007F43891B033321F07F418B420BD9D4F827
:102FC0000435C4F840352F20FFF770FE744B4FF4E2
:102FD0000032C3F80021039A0023137005B0BDE846
:102FE000F08F0026374678E701EB4104506892F8ED
:102FF00002B000EBC40E013110F834401868C9B2B9
:103000008B4508BF0021022C04D0032C7FF470AF45
:10301000002410E0DEF804B004468646002C3FF49D
:1030200067AFA34500F0C080A646E469F6E780F8E4
:1030300010A0C06901240028F9D1002C3FF458AF3A
:10304000186055E7D4F80C90C4F800E0761A8C4468
:10305000E1691960B9F1000F07D008EB0C0121F00C
:103060007F41C4E90119E06120461C68002C3FF44F
:1030700051AF2168B142E5D98E1B26604AE7002096
:1030800084468646F1E70146C069019DD1F804A057
:103090002E68444DD1F80890AAEB060C2CF07F4C1A
:1030A000AC4535D80CEB09060E60D3F800C081F8AA
:1030B0001080C1E90144CC61BCF1000F33D119602B
:1030C00031E701EB410B0131C9B2514514BF117019
:1030D00014701CF83B1001290CEBCB067FF42CAFCD
:1030E000716891F810B0BBF1000F7FF425AFD6F8EE
:1030F00008C0C1F804C0F5688D603569CD60766997
:103100008E61BEF1000F0CBF66465E464E60BCE7A6
:10311000A6EB0A0626F07F464E4502D2A9EB06062C
:10312000C2E70C60C1E7D1F80090DCF80060B1455F
:103130001FD8A6EB0906CCF80060C1F81CC0BEE79A
:10314000A9EB0A09D6F81CA0B446BAF1000F0AD0C0
:103150005646D6F800A0CA45F2D3AAEB090AC6F82B
:1031600000A0B2466646C1F80090C1F81CA0F1610B
:10317000D9E66646EDE7FFF76DFE2CE7F8D10020B3
:10318000F9D10020FCD10020F0D10020E0D20020B5
:103190001CD00020D8D1002000100140D9D100203F
:1031A00000E100E0FEFF7F0074450FD1D0F81CB0B5
:1031B000C3F800B0BBF1000F08D10A4D0120A86090
:1031C00001984FF0010CC0F800B0E1462068E469B6
:1031D000CEF81C40002C3FF48BAE256828442060BC
:1031E00086E600BF0010014037B5074B054693E85F
:1031F00003006C46002384E803001A462146284653
:10320000FFF7FEFC03B030BD1C160600FDF78EB9BB
:1032100010B54FF6FF7304469C42084609D1FEF7ED
:1032200011FFB0F5807F044601D14FF6FF742046B0
:1032300010BDFF2CF9D82146FEF7E0FE0028F6D19C
:10324000F3E710B5044601F0EFFC2046BDE810405E
:1032500000F02EBF1FB5037893B90279072A0FD16A
:10326000448803932046CDE901338DF80420FCF710
:10327000B7FAADF8060001A8ADF80840FFF7E1FF86
:1032800004B010BD1FB50023CDE901330393ADF8A1
:103290000600022301A88DF804308DF80810FFF70E
:1032A000D0FF05B05DF804FB86DF704738B50488B1
:1032B0004CB9821C00F10A0512F8013B1BB995427A
:1032C000FAD100200AE00B88A342FAD10822023189
:1032D00002303EF031F9B0FA80F0400938BD08B54F
:1032E00070B171B103780A78534013F0FE0F08D122
:1032F0000622013101303EF01FF9B0FA80F040099A
:1033000008BD0020FCE710B5044600F0BDFF2046D4
:10331000BDE8104000F04ABF43DF70476FDF7047E1
:10332000024B0022C3E90022704700BF50CD0020AD
:10333000F0B5FF2887B004460E4615461F4629D82B
:103340000846FCF78BFA28B303AA2046FFF7E4F8F7
:1033500018B10524204607B0F0BD01A903A8FFF766
:1033600011F804460028F4D1019BAE705A882A80D7
:103370005FB13B6892009A420AD3029968683EF0B6
:10338000E9F803A8FEF7E2FFE4E7029B6B60F8E7C9
:103390000424DFE70724DDE72DE9F041CEB020AEBD
:1033A000502380460CADB82200213046019303958E
:1033B000FCF7B8F80DF1970305930DF1AE030693F2
:1033C0000DF1C503079337AB08930DF1F303099390
:1033D0000DF585730A931C4F04960DF221130B9380
:1033E0000024444507D1E2B2002104A8FFF796FF6C
:1033F0004EB0BDE8F081502200212846FCF792F83B
:1034000001AB02AA072137F8020BFFF791FF20F06A
:1034100002000528ECD06B7C032B12D817230DF18A
:10342000310203FB04630DF1450152F8040B43F82C
:10343000040B8A42F9D11188198092789A7001346C
:10344000CFE743F20220D3E70AD200202DE9F04172
:1034500010220546A6B000212D48FCF763F835B9C7
:1034600029462846FCF7D0F926B0BDE8F0816A006D
:1034700028492748DFF89C8004AE3EF06BF83822DC
:1034800000213046FCF74EF800245023CDE90134EA
:1034900012AF0397502200213846FCF743F801ABE6
:1034A00002AA072138F8020BFFF742FF20F00200C2
:1034B0000528D9D09DF85930032B26D8C4EBC40277
:1034C000B318DDF85910B1500134BDF85D209A8071
:1034D000A5429DF85F209A71DCD10DF1170313937B
:1034E0000DF11E0314930DF1250315930BAB1693E9
:1034F0000DF1330317930DF13A0318930DF14103C6
:1035000012961993E9B23846ACE743F20220ABE7D2
:103510001AD200200AD200202DE9F043037889B0A6
:103520000546002B3FD1017907293CD104AA4088E8
:10353000FFF7FEFEB8BBFFF7F3FE02A90DF1060090
:10354000FEF7C0FF78B36E88BDF80670BE42F4D0B7
:10355000059C631C1846113413F8012B12B9A342C1
:10356000FAD1EAE7DDF80C80102208F101013DF004
:10357000E3FF08F1110181462046FFF7B0FEB9F1E3
:10358000000F01D00028D8D03046FCF729F90023DD
:10359000ADF81A0006A88DF81830ADF81C60ADF82B
:1035A0001E70FFF7B0FE09B0BDE8F083CA1F012A04
:1035B00073B5064654D80025CDE900558DF80210A4
:1035C000FCF776F9044600284CD0437CDB074BD44B
:1035D000007CFCF72BF910B9032002B070BDE36842
:1035E000019003EB83031B019BB29B086846ADF877
:1035F0000030FCF73BF9626804F108036946304685
:10360000FFF7FEFA637C03F00603062B01BF174A9F
:10361000136803F1FF33136030B9637C23F00703B1
:1036200043F001036374D8E711280BD10F4A1368E4
:1036300001331360637C23F0060343F004036374D7
:103640000020CAE7862809D1084A136801331360AD
:10365000637C23F0060343F00203E3E70728BBD1B2
:103660000720BAE70520B8E72846B6E7F0CE0020E5
:103670002DE9FF410546102200216846FBF752FF65
:1036800068882979ADF802008DF80410FCF710F96C
:103690002B78454E092B5ED8DFE803F00505684D11
:1036A0004D6C7173757D00283FD0437CDC073CD5A1
:1036B000FEF7FEFD2B78581E434243410024684626
:1036C0008DF800408DF80830FCF7E4F833684BB310
:1036D000364E002537464FF0140808FB05735B7C17
:1036E0005A0703D49B0759D5002C57D0B17830889E
:1036F000FFF75CFF002851D014235D437B19862817
:103700009B788DF804307A5B16BF0290082309235A
:103710006846ADF802200CBF8DF800308DF80030FF
:10372000FCF7B8F804B0BDE8F08101238DF8003053
:10373000AB68029316E080B18268AB689A420CD104
:10374000437CD90709D5326823F00503013243F0E1
:103750000403326043740024B8E702238DF800307C
:10376000EB6803936846FCF795F8F4E703238DF8BC
:103770000030F7E704238DF80030EB68D9E7052324
:10378000F5E70623F7E7072368468DF800300124A4
:10379000FCF780F89AE7EB680293DCE70135082D27
:1037A00006F1140699D1BDE7F0CE00203CD20020EE
:1037B00070B500238CB02D492C4E4FF6FF70CDE92B
:1037C0000033FCF7E7F84FF6FF750446AC420BD028
:1037D000A4F58043ADF8143002AA6B46002105A879
:1037E000FEF736FE0A2822D0214B1A781846E2B995
:1037F0004FF6FF718C4218D01E4E367801251D7091
:10380000B607A4F580439BB21DD58B422CD0052171
:103810008DF8141005A811468DF81850ADF81A301F
:10382000FEF7CEFD60B1FFF757F90CB070BD204632
:10383000FEF778FD20463146FCF7ACF80446C5E7B4
:103840000D4B1D70F1E702230022092102708DF853
:10385000141005A8FF21ADF816408DF81810CDE919
:103860000723FFF705FFE0E70423EDE718D1002069
:10387000B1D000205DCD0020B2D00020F0B542686C
:1038800005783D4C85B0B2FA82F149090391691E71
:103890000346042924D8DFE801F0030330496A0015
:1038A0009989DE8901F5804189B243F6FE77B942F4
:1038B00004D906F5804080B2B84211D8012DADF888
:1038C00002108DF8046013D1002A14BF03210021D7
:1038D0008DF8001003929B6802936846FFF7C8FEBC
:1038E00023781BB100232370FFF762FF05B0F0BD02
:1038F000002A14BF04210121EAE79989DD8901F535
:10390000804189B243F6FE76B14204D905F5804084
:1039100080B2B042E4D8002A0CBF02220522ADF8E2
:1039200002108DF804508DF80020D4E7988900F536
:10393000804080B243F6FE718842D1D8DB89002BEB
:10394000CED1FF23ADF802008DF804305AB906231A
:103950008DF80030FEF7E6FC084A00232370137050
:10396000FFF726FFB9E707238DF80030F4E70823B7
:103970008DF80030B1E700BFB2D00020B1D00020F8
:10398000F8B50D490D4DFCF705F84FF6FF760446E6
:10399000A5F12007B44201D12046F8BDFF2CFBD889
:1039A00021462846FBF732FF0028F5D0204639464D
:1039B000FBF7F0FF0446EDE7F8D0002018D1002017
:1039C00073B5104B104C93E803006D46002385E857
:1039D00003001A4629462088FFF712F94FF6FF76B2
:1039E0002388B34201D0112801D102B070BD18461E
:1039F000FFF7C6FF00231A4629462080FFF700F98B
:103A0000EEE700BF2416060038CD00201FB503786E
:103A1000012B044615D10179012912D1002302AAF4
:103A20004088FFF785FC60B902238DF80030638879
:103A3000ADF80230039B68461B788DF8043000F027
:103A4000B5FD054B1A884FF6FF739A4201D0FFF778
:103A5000B7FF04B010BD00BF38CD002070B50446DC
:103A60008AB0142200216846FBF75CFD6588ADF83A
:103A700004502846FBF7B4FE2378ADF80200092B6A
:103A800015D8DFE803F005163048525E8614A1A56C
:103A900007238DF8003023798DF808309DF80A301F
:103AA00043F001038DF80A306846FBF78DFF0AB03A
:103AB00070BD07238DF8003023798DF808309DF80C
:103AC0000A30444AA168039143F001038DF80A309B
:103AD0001368002BE8D09942E6D1002313603E4AD8
:103AE00003931580E0E708238DF8003023798DF8E3
:103AF0000830E3680493374BA1681A680391002AE1
:103B0000D2D09142D0D1354900221A600B6803927D
:103B1000013B0B60C8E707238DF8003023798DF84F
:103B2000083001238DF80930BEE708238DF80030F6
:103B300023798DF8083001238DF80930A3680493A8
:103B4000B2E7274D09238DF800302B78002BABD03E
:103B50004FF6FF70FFF714FF4FF6FF7398420646CB
:103B6000A2D12049FBF716FFB04204469CD1142293
:103B700000210DEB02002970FBF7D4FC0B238DF81C
:103B80001430ADF81840ADF8164005A8FBF71CFF3F
:103B90008AE70A238DF80030114BA4681A78029442
:103BA000002A81D0142200210DEB02001970FBF7CE
:103BB000B9FC0C238DF814304FF6FF73ADF81830B4
:103BC000ADF816300794E0E705238DF800306BE779
:103BD0000623FAE7F4D00020E4CE002034CD002004
:103BE0003ACD002018D100202DE9F047474B1B7833
:103BF0008AB00546002B00F08780454B454F93E87F
:103C000003003C7803AE86E80300BCB94FF6FF70B2
:103C1000FFF7B6FE0123ADF8143001AB0693042381
:103C2000029305AA02AB062180460194ADF8164026
:103C3000FFF77EFB07284AD101233B70364B1C68F7
:103C40009846002C5AD1354A354F12883B68AA4213
:103C500041D1002B3FD0142221460DEB0200FBF78F
:103C600061FC072328468DF81430FBF7B9FD0623C5
:103C7000ADF8160005A8ADF818508DF81C30FBF70C
:103C8000A3FE20460AB0BDE8F087CDF804A0019B52
:103C90004046A34224BFC1461C46FFF771FEBDF853
:103CA00014309B00029305AA02AB06218046FFF761
:103CB0003FFB0028EBD00528E7D04FF6FF7398456F
:103CC0001CD1164BA3F80090154B1C60B4E74FF6BF
:103CD000FF79A246EDE701333B6000220E4B3146EF
:103CE0002846FEF78DFF0028CCD00023C8F800300E
:103CF0003B68112803F1FF333B6001D11120C1E77C
:103D0000862818BF0320BDE70820BBE7ECCE0020C3
:103D10002C160600F3D00020F4D00020E4CE0020C2
:103D200034CD002063DF7047A6DF7047A2DF704705
:103D30002DE9F04391B0984611238DF804301378A3
:103D40008DF805300024164601254FF0000365F379
:103D50004203074689461C22214609A88DF80630F1
:103D6000FBF7E0FBB3788DF80930C3F30302A242FE
:103D700014BF1A2212228DF8242001AA0E9203AB3E
:103D800072788DF808200493224602AB65F3420254
:103D9000059308238DF80A20CDE9064404AAADF85E
:103DA0001C3009A9434638888DF80E50ADF80C90A8
:103DB0000894FFF7BBFF11B0BDE8F083A0DF7047A8
:103DC000044A0123116883400B401ABF1218507E29
:103DD00018467047F4CA002070B4094D13460126F6
:103DE0002A6806FA01F4144207D001F119040246C8
:103DF0003146281970BCFDF757BE70BC704700BF34
:103E0000F4CA00201FB50023CDE9013303938DF8D8
:103E10000A201A46074BADF8081006241978ADF8A9
:103E200006008DF80440FFF7D7FF01A8FFF709FA55
:103E300004B010BDB32C002010B4084A012314684C
:103E40008B40234006D00A445DF8044B0146507E67
:103E5000FDF79ABD18465DF8044B7047F4CA002080
:103E600010B50A4B19780446FFF7E6FF58B1084B26
:103E700000205A88A24201D1C0B210BD01300828EA
:103E800003F10C03F5D1FF20F7E700BFC8CC0020F9
:103E9000CACC00202DE9F8430546FBF7A1FC234BD3
:103EA000074600221420984600FB02F1CC5AAC428F
:103EB0002AD10B44002634464FF014095BB199789F
:103EC0002846FEF711FA10B1052818BF0324013661
:103ED0003246072A1DD9A4B9FF2D24D814492846F3
:103EE0004FF6FF75FFF794F9FFF762FCAF4208D079
:103EF0003846FFF7B5FFFF2803D00C2343430D4A94
:103F0000D5522046BDE8F8830132082ACCD10023DF
:103F1000D0E709FB02F338F80310A94201D143446A
:103F2000CCE70132D5E70724EBE700BF3CD2002005
:103F300018D10020CACC00202DE9F0411F46154BB6
:103F40009DF818400E46904619780546FFF744FF45
:103F5000B8F1000F17D0104B3A4619782846FFF7F2
:103F60003BFF0E4B224619782846FFF735FF44B138
:103F70002846FFF775FFFF2803D00C234343084A68
:103F8000D652BDE8F081002CFBD03046BDE8F041B0
:103F9000FFF780BFB32C0020B52C0020B42C0020EC
:103FA000CACC002008B5FFF75BFFFF281DBF0C231C
:103FB0004343034A4FF6FF7018BFD05A08BD00BFF5
:103FC000CACC00202DE9F04385B00546FFF7EAFF93
:103FD0004FF6FF739842074641D001224FF0030984
:103FE00001AB0821384602F10108FEF791F81FFAEB
:103FF00088F8064648BB02990A46032342F8049B08
:1040000006312846FBF7E0FB044660B90821384634
:10401000FFF7CCFA0446112C3FD01AD80CB30C2C65
:104020002FD107231EE00C280DD0052800D13446DF
:1040300008213846FEF758F9002818BF03244246E5
:10404000002ECDD1E7E70126F2E70728E9D00446A4
:10405000E1E7862C13D043F202039C4211D10022E7
:104060001CE0012328468DF80430ADF80850FFF716
:1040700099FFADF8060001A8FFF7C8F8EFE708239D
:10408000F0E7092328468DF80430FFF78BFFADF8E1
:104090000850ADF806000394EDE70122034B2846D3
:1040A0001978FFF799FE05B0BDE8F0835ACD0020DE
:1040B0000378072B02D14088FFF784BF70470000C8
:1040C0002DE9F0434FF6FF75A84285B0044668D04D
:1040D000FFF768FFA84227D100260327B0464FF01C
:1040E00001093B46324641462046FBF76FFB042858
:1040F00005464DD0082847D00B282DD117F00203D4
:104100001FD1B8F1000F20D11EBB032320468DF82C
:104110000430FFF747FFADF80840ADF8060001A8EE
:10412000FFF774F8002237E0002301AA0821FFF707
:10413000FFF80028D0D1029B03F106089E881F6873
:10414000CDE701274FF00009CBE703271E4698462D
:10415000F8E703274646F5E7B9F1000FD5D0112857
:1041600019D043F202039842DCD008B90223CDE70C
:10417000092320468DF80430FFF714FFADF80840FE
:10418000ADF806000395CAE7B9F1000FEED1BCE720
:10419000B9F1000FB9D00122034B20461978FFF77F
:1041A0001BFE05B0BDE8F08359CD002037B505787A
:1041B000012D044614D14088FFF782FF6088FFF785
:1041C000F1FE00236A462946FFF7B2F840B9019B89
:1041D0001B782BB1034B608819782A46FFF7FCFD4A
:1041E00003B030BD5BCD0020F0B587B004460E466D
:1041F0001746FFF7D7FE4FF6FF739842054624D0C7
:104200001E4B20461978FFF717FE80B30023CDE937
:104210000033029304238DF80030194BADF80240AF
:104220001978ADF8046020468DF80670FFF704FE9B
:1042300068B12846FFF72EFE124B2046002219785F
:10424000FFF7CAFD6846FEF7FCFF07B0F0BD072187
:104250002846FEF749F80528EED10923049003A863
:104260008DF80C30ADF80E40FEF7EBFFE4E73A4670
:1042700031462046FFF7C6FDE7E700BFB52C00201A
:10428000B42C0020B32C002010B5027886B0044670
:104290001AB1012A09D006B010BD0E4B1B78002BB5
:1042A000F9D0C088FFF7F6FDF5E70B4B4088197889
:1042B000FFF792FD1422002101A8FBF733F9608873
:1042C000ADF80600FFF76EFEADF8080001A8FBF799
:1042D0007BFBE0E7ECCE002030CB002070B504463D
:1042E00086B01422002101A8FBF71CF9237860880E
:1042F000ADF80600013B0B2B00F29080DFE803F0E5
:104300002106233A4E585C68747A7C8C2679444B9B
:10431000321C19784FF0010518BF01228DF80450A6
:10432000FFF75AFD731B5A425A413E4B6088197879
:10433000FFF752FD6088FFF735FEADF80800002D4D
:1043400042D106B070BD02238DF804302379002BD2
:1043500014BF012302238DF80C30314B0122197850
:10436000FFF73AFD2F4B227919786088FFF734FD6B
:104370000125DFE703238DF804302A4B1978FFF776
:104380005BFD002814BF012302238DF80C30A379B4
:104390008DF81030A388ADF80E30E9E7204B19787E
:1043A000FFF74AFD0028CCD102238DF80430DFE767
:1043B00003238DF80430EAE70723A2888DF8043040
:1043C000ADF808208DF80C3001A8FBF7FDFAB8E72E
:1043D00008238DF80430A388ADF8083007238DF842
:1043E0000C30A3680593EFE706238DF8043063686B
:1043F0000393BDE70523D8E703238DF80430094B69
:104400001978FFF719FD002814BF012302238DF846
:104410000C3041F20113BEE70423C6E7002589E70B
:10442000B0D0002030CB00201FB50D294FF0000385
:1044300001930393ADF80600029108D10B2301A864
:104440008DF80430FFF74AFF05B05DF804FB8629BC
:104450000CBF0A230923F2E730B508490A68002394
:10446000012505FA03F42242D8B202D122430A60A0
:1044700030BD0133182BF4D11846F9E7F4CA0020F7
:1044800010B50378182B044602D1FFF7E5FF207022
:1044900010BD000010B5024B197DFDF723FB10BDC8
:1044A000F4CA00202DE9F04F3D4D89B02878FFF780
:1044B00087FC60B103A8FFF7EDFFDFF8E8A0DFF8A5
:1044C000E8B00DF110090027039B9F4202D309B009
:1044D000BDE8F08F39F8024B29782046FFF7ACFC95
:1044E000064678B39AF800102046FFF7A5FC8046F0
:1044F00040BBBBF800304FF6FF7219462046FBF771
:1045000067F943F20302904229D10133ABF800303E
:10451000EFE7052320468DF80030FFF743FDADF8A7
:1045200002006846ADF80440FEF770FEB046324621
:1045300029782046FFF750FC42469AF800102046A2
:10454000FFF74AFC0137BFE72046FFF72BFDFEF7D8
:104550004BFE0026EBE72046FFF7B2FDE7E7082811
:10456000F2D012D80028D4D00628EDD0092302902A
:1045700020468DF80030ADF80440FFF713FDADF88C
:1045800002006846FEF742FED1E743F2020398427A
:10459000CDD043F201439842DDD01128E6D1C6E7E1
:1045A0005BCD00205CCD0020F4D200201FB5044676
:1045B00040882378ADF80600012B10D05AB21AB10A
:1045C000022B15D004B010BD01A88DF80420FEF711
:1045D0001DFE6088FBF704F9FFF772FDF2E78DF826
:1045E000043001A8A388ADF80830FEF70FFEE9E714
:1045F0002379002BE6D0FBF7F3F84FF6FF739842D0
:10460000E0D0044B01221978FFF7E6FBFFF74AFFE1
:10461000D8E700BF5BCD002038B5074C0146207DB0
:10462000FDF7B2F930B1A07DFDF7AEF9002814BF57
:104630000220012038BD00BFF4CA00202DE9F04758
:104640008CB0894616468046FFF7E6FF2022824658
:10465000002104A8FAF766FFBAF1000F46D0B9F1BD
:10466000000F17D099F8005015F001054FF6FF74B0
:1046700015D04046FFF796FCA042074639D1404886
:10468000FDF7E0FCB0F5807F01D0B84275D1002580
:10469000032470E04D4685264FF6FF775FE02E46F7
:1046A00027465CE04A4631464046FBF795F804460B
:1046B000B9F1000F5DD000285DD199F8003013F0FA
:1046C000010F14BF012102214046FEF7DBFDB6F1C8
:1046D000850218BF01220024009501233946404677
:1046E000FFF72AFC20460CB0BDE8F08743F2020435
:1046F000F8E7002502AB012207213846FDF708FD47
:104700000446002837D1214650220398FAF70AFFC1
:10471000039B83F800A0039C079604F134030493E1
:1047200004F118030893631C09934046154B0B933F
:10473000FFF796FBFF280CD0134A0C2101FB002049
:1047400050F8042FC4F811208288A4F8152082792B
:10475000E2753846FBF7D2F8044660B90646BAF16E
:10476000020F04AB9ED1002231464046FBF734F8DD
:104770000446002CABD00022AEE707460125B9E77E
:10478000F8D00020B3D00020CACC0020F0B585B00E
:104790000446FFF741FF324F012806463D7831D1EC
:1047A0002046FFF7FFFB4FF6FF7398422AD02046C2
:1047B00032462946FFF710FB0023CDE9013303936E
:1047C00001A80C238DF80430ADF80640FFF786FDF4
:1047D000244B1B78E3B139782046FFF72DFBB8B99D
:1047E000214B22491A682046FFF728FF86280546F4
:1047F00032D011280FD070B129462046FFF714FEA1
:1048000005B0F0BD002229462046FFF7E5FADFE7B4
:1048100000221146E7E7A5F111035E425E41002246
:10482000134B20461978FFF7D7FA124B3246197806
:104830002046FFF7D1FA104B002219782046FFF7E7
:10484000CBFA0E4B002219782046FFF7C5FA002D4F
:10485000D6D0112DD4D0CFE700260122E0E700BF4B
:10486000B22C0020DFD100209CD00020DAD1002023
:10487000B12C0020B02C0020AF2C0020AE2C00204A
:10488000F0B587B0074601A8FFF704FE02AD00248B
:10489000019B9C4201D307B0F0BD35F8026B39464D
:1048A0003046FFF7C9FA10B13046FFF76FFF013409
:1048B000EEE700002DE9F04F054687B09046994697
:1048C0000F4639B9A14B1B78F3B90524204607B030
:1048D000BDE8F08FFFF7A0FE0138C0B2012800F25A
:1048E0002D8100212846FAF779FF0446862C00F036
:1048F000B080112C00F09980002C00F09680B9F166
:10490000000F00F0BF80B9E0FFF786FE012800F03D
:104910009E80022840F012818D490B78284613F0C2
:1049200001048B4614BF4FF0010A4FF0020AFFF753
:1049300039FB4FF6FF739842064659463AD03B463C
:1049400002AA0721FEF7F4FC0446F0B9039B93F892
:104950004420D10740F1C780B8F1000F40F0D68065
:1049600003F1340202F112012846FAF733FF4FF047
:10497000000A044600230093BAEB030318BF012387
:10498000B4FA84F25209314645E00528F2D1BDE07F
:1049900004AB012207213046FDF7BAFB044600288C
:1049A00040F0C1803046FAF7A9FF0446002800F025
:1049B000B280B8E0002C41D06648FDF743FBB0F56B
:1049C000807F834637D0B04236D004AB0122072126
:1049D000FDF79EFB044650B95846FAF78FFF044690
:1049E00028B95B492846FAF7F9FE044638B1072191
:1049F0005846FDF779FC10B1052818BF03244FF67F
:104A0000FF73BBEB030318BF0123B4FA84F20093D6
:104A10005209012359462846FFF78EFA002C7FF4ED
:104A200065AF51462846FEF72DFCA4F111035E4206
:104A30005E4100220FE0B3460324E0E72846FAF780
:104A4000CDFE009704460123B0FA80F29AE7404970
:104A500048E700260122404B28461978FFF7BCF9A9
:104A60003E4B324619782846FFF7B6F9B9F1000FE8
:104A700008D0002C3FF42AAF112C17D0214628462D
:104A8000FFF7D2FC0D2C3FF421AF06D8002C3FF4E9
:104A90001DAF082C18BF032418E7862C14D043F24E
:104AA00002039C423FF412AF112C1AD12C4B3A4610
:104AB00019782846FFF790F92A4B4246197828467C
:104AC000FFF78AF9002401E7254B3A461978284672
:104AD000FFF782F9234B424619782846FFF77CF905
:104AE000F4E60324F2E6B8F1000F0FD1598D03F17B
:104AF000180200297FF436AF03F12C01343311F88A
:104B0000010B00287FF42EAF8B42F8D19BF80030C8
:104B1000DA073FF53DAF0E492846FAF75FFE044637
:104B200000283FF427AF07213046FDF7DDFB0028C2
:104B30003FF420AF052818BF03241BE743F202040B
:104B4000B9F1000F3FF4C2AE98E700BFDFD10020FB
:104B5000DAD10020F8D00020AF2C0020AE2C0020AD
:104B6000AD2C0020AC2C00202DE9F04786B0074684
:104B7000FFF726F958B101A8FFF78CFCDFF8488051
:104B8000DFF8489002AE0025019B9D4202D306B09B
:104B9000BDE8F08736F8024B39462046FFF74CF95E
:104BA00080B198F800102046FFF746F999F80010F8
:104BB00082462046FFF740F901230146524620462F
:104BC000FFF778FE0135DFE7AC2C0020AD2C00208C
:104BD00010B50378062B0ED9072B1BD10E4B1C7872
:104BE0002046FFF7EDF810B12046FFF749FE0B4BCA
:104BF0001878FFF7B9FF0A4B1C782046FFF7E0F85A
:104C000010B12046FFF73CFE064BBDE81040187877
:104C1000FFF7AABF10BD00BFB12C0020AF2C0020B1
:104C2000B02C0020AE2C00201FB503780446092BC1
:104C300009D8DFE803F0050A2020202020202020CA
:104C40004088FFF7A3FD04B010BD144B197819B3C9
:104C5000134B00791B7803F00102904206D861796A
:104C6000C3F34003994294BF002101210123002294
:104C70006088FFF71FFE23788DF80430043434F881
:104C8000023CADF8063094E8030004AB03E90300EE
:104C900001A8FFF723FBD6E70121E7E7DFD10020DA
:104CA000DAD1002037B5174B174A5B881188174CAB
:104CB000174D994208D852889A4205D36369FBB9C7
:104CC00000232B7003B030BD2B783BB16369002B00
:104CD000F6D000228DF8042001A80FE00D490E48FF
:104CE0000978D4E9012300290CBF11461946FDF7C4
:104CF00041F90028E4D0A369002BE1D09847DFE711
:104D00000122E7E72ACD002038D100208CCC0020FA
:104D100020CC002008D20020A8CC00207BDF7047E8
:104D20007ADF704776DF704775DF704737B5164B0F
:104D300018884FF6FF73984210D0144A144D137818
:104D4000297B0133DBB2994213702C4608D31149F9
:104D5000FFF7EAFF10B1AB6903B1984703B030BD6C
:104D6000002313702B7C33B13B21FFF7DBFF10B125
:104D7000AB6903B198476369002BEFD000228DF82F
:104D8000042001A8E9E700BF88CC002008D2002059
:104D90008CCC002038D1002065DF70472DE9F74F1B
:104DA0000C9CBDF834B02788002580468A46914681
:104DB0002E46B8F80020B2420BDC35B12288013A09
:104DC000D21B92B2FF2A39D8DA55002003B0BDE8D1
:104DD000F08FD8F8042052F82600019000220DF13F
:104DE000030101A8FFF7D8FF0028EFD19DF80320A9
:104DF0004A4521D12288002D14BF0020022002EB59
:104E000009010144594519DC3DB9013292B22280B1
:104E100003F802A022880132228022880DF10301CA
:104E20001A4401A8FFF7B8FF0028CFD121889DF8C8
:104E300003200A44228001250136BAE70C20C5E789
:104E40002DE9F341089CBDF824501746CDE90045F3
:104E500002220646FFF7A2FF48B910223946304623
:104E6000CDE9084502B0BDE8F041FFF797BF02B0B9
:104E7000BDE8F0812DE9F04F00231688138090F8EB
:104E80002D3085B007460D4614465BB3082E01D879
:104E90000C2008E102A8FAF7AFFD002840F00381DA
:104EA00013880822CA54238801339BB21B22238013
:104EB000CA54238801339BB2CA18DDF80910238035
:104EC000E950BDF80D30938023889DF80820063303
:104ED0009BB212F0FE0218BF01222380EA542388FD
:104EE00001332380BB78FBB123880433B342CFD88E
:104EF00002A8FAF77FFD002840F0D580238803221E
:104F0000EA54238801339BB219222380EA54238870
:104F1000BDF8082001339BB2E9182380EA54120A35
:104F20004A70238802332380FA789AB12388D91CE7
:104F3000B142ADD80221E954238801339BB201214B
:104F40002380E95423880B449BB22380EA542388AE
:104F50000B4423807A68AAB12388D91CB14297D820
:104F6000022192F90020E954238801339BB20A21DF
:104F70002380E954238801339BB22380EA54238899
:104F8000013323803B89002B40F081803B8A53B161
:104F9000CDE900462B460722032107F11000FFF759
:104FA0004FFF00287FD13B8B53B1CDE900462B4604
:104FB0001522142107F11800FFF742FF002872D1D3
:104FC0003A6A002A72D1D7F82480B8F1000F30D0A5
:104FD000B8F804302188981C8A1C0244B2423FF67B
:104FE00057AFFE283FF654AF03336B542388013389
:104FF0009BB2FF222380EA54238801339BB2238093
:10500000B8F80020EA54E918120A4A7020880230E1
:1050100080B22080B8F804205AB1D8F808100029CE
:105020004ED028443CF096FA2388B8F80420134464
:10503000238097F82C30002B7DD1387898B33B88AB
:10504000012B3DD0228802F1020CB4453FF620AF7F
:10505000012805D17B78023313449E42FFF418AF38
:10506000023EB61AB6B202A905EB0C00ADF8086014
:10507000FAF7BEFCB8B93B78022B40F09F80BDF830
:105080000830B34240F2B580ADF808609FE0CDE94A
:1050900000462B460622022107F10800FFF7D0FE4A
:1050A00000283FF473AF05B0BDE8F08FB4F800C03E
:1050B0000CF10603B3423FF6EBAE1188052901D887
:1050C0000720F0E76FF4486E01EB0E039BB24FF23E
:1050D0007D3E7345F4D95388052BF1D96FF44860B0
:1050E000181880B27045EBD94FF6FF70814203D09B
:1050F000834201D09942E3D8052305F80C30238878
:1051000001339BB212212380E954238801339BB2DF
:1051100023801188E954E818090A41702388023372
:105120009BB223805288EA54E918120A4A702388F5
:105130000233238047E7BB6A002BC1D04FF0000940
:105140004FF00C0A4FF0160B97F82C305FFA89F2EB
:1051500093427FF672AFB96A0AFB02F201EB0208D2
:10516000B8F80430981CFE283FF692AE208803332E
:105170002B54238801339BB2238005F803B0238886
:1051800001339BB223808A5AEA54E918120A4A7002
:105190002088023080B22080B8F804205AB1D8F8B4
:1051A000081000298CD028443CF0D4F92388B8F8A2
:1051B00004201344238009F10109C5E7012B7FF482
:1051C00063AF7B789E42FFF45FAFADF808300821F3
:1051D000BDF80830FE2B3FF65BAE22880133AB549E
:1051E0002288013292B22280A9542288134423805B
:1051F00059E70921ECE700002DE9F0430646B2F833
:10520000009007460D4690460FCE9FB06C460FC4E7
:105210000FCE0FC40FCE0FC496E8070084E8070036
:105220003C2200210DEB0200CDE90C118DF82E106F
:105230008DF82D1000910E91FAF774F93C22694611
:105240000DEB02003CF078F9002840F0C9807C6B3F
:10525000002C34D1BB6B23B104F12400002D3ED1CE
:1052600084B23B6B23B104F11201002D62D18CB2E8
:1052700097F82E30002B00F0A980E11C002D7CD186
:105280008CB297F82D300BB10934A4B2BB780BB1B6
:105290000434A4B2FB780BB10334A4B238780028EC
:1052A00000F08F80012840F094807B78ADF83C308E
:1052B0000020BDF83C3002331C44A4B281E065B14B
:1052C000B9F1020F03D80C201FB0BDE8F083022211
:1052D00023782A7011226A70AB700324BAE748451C
:1052E000F1D811222A55621C92B22221A954A21C83
:1052F00003F1170115FA82F203F1270C0E4651F85B
:1053000004EB42F804EB6145F9D104F1120292B2C8
:105310001121A95404F1130292B223211434A95487
:10532000073315FA84F453F8042B44F8042BB342E2
:10533000F9D195E74945C6D811222A55621C92B287
:105340001020A854274A1668023415FA84F456B17E
:10535000107992F805C0844540D900F1010C82F81B
:1053600004C046F820405A1E013C0F3312F8010FCA
:1053700004F8010F9342F9D179E74945A3D8601C9D
:10538000022280B22A551C261444013B2E54A4B29A
:10539000032B25D8DFE803F00205071800232B555F
:1053A00002E00123FBE72A558CB2A9EB0409291975
:1053B0000FAA3846ADF83C90FFF75CFDBDF83C30D5
:1053C0001C44A8F800407FE70323E8E7002DECD158
:1053D00057E70FA90020FAF70BFB6AE7042073E7F1
:1053E000072071E700D20020F0B590F82D3085B08D
:1053F0000C461546002B44D190F82E30002B40D19E
:10540000436B002B3DD0C3780BB15B0739D584B318
:105410002B68072B33D9083BB3F5803F28BF4FF6E5
:10542000FF7304F10806ADF806300DF106023146AF
:10543000FFF7E2FE0346F8B9BDF80620083292B243
:10544000ACB1110AA71C6170F11B89B20529029049
:105450002270CDF80B0012D902A8FAF7CDFA50B994
:10546000DDF80910C4F80210BDF80D10E1802A60C3
:1054700002E02646D9E70346184605B0F0BD0423EE
:10548000FAE70723F8E713B590F82D301446CBB1AF
:1054900090F82E30B3B1436BA3B9C3780BB15B075F
:1054A00010D52368B3F5803F28BF4FF6FF730DF189
:1054B0000602ADF80630FFF79FFEBDF80630236008
:1054C00002B010BD0720FBE707B5144B1A686AB19C
:1054D000002018601B6800934FF08042009B01235E
:1054E000C2F808330E4A5370FAF788FA0D4B1A685F
:1054F0008AB100221A601B680193019B4FF0804320
:105500000222C3F80823064B0120987003B05DF80F
:1055100004EBFAF773BA03B05DF804FB0001004036
:105520006CCC0020040100400E4BD3F8183182B03F
:10553000B3B10D4B0D4800221A601B680193019B0B
:105540000B4B997EFF291FBF01228A404FF0A041DB
:10555000C1F8082500225A761A711B6802B0184754
:1055600002B070470030004018310040E4CB00200A
:10557000E0CB002070B52D4C86B094F8213001931B
:1055800094F820300093E36904F1260204F123012A
:105590004FF04020FAF750FA2346E0B994F8236020
:1055A000A56906BB217B8A1E012A1CD8E0692269F5
:1055B000904218D16269E37BE261C5F3401503298B
:1055C00084F8203084F8215007D100954FF0402115
:1055D0002046FAF708FB06B070BD4FF04021204688
:1055E000FAF7A4FAF7E7124A07CA06AC04E907007B
:1055F000C6B14FF04021D1F8C424C1F8C4249007AB
:105600000CD501228DF80820002283F824206A0797
:10561000E1D4D3E9002102A89047DCE75107F3D594
:105620000222EFE78DF80860EEE700BFB8CB00205C
:10563000C4CB0020F7B515464FF0FF32C1F8082360
:1056400090F8242004460F4602F0FF0E2AB183682A
:10565000C1F80433112003B0F0BD012680F82460A6
:10566000836100F10C0C95E807008CE80700AA782C
:1056700084F820206A68E2616A78C7F888252A7869
:10568000B24212D012B91E1C18BF012684F8216044
:105690000096AB786A6839462046FAF7A4FA236880
:1056A000002BD8D184F82430D5E784F821E0AB78FA
:1056B0006A6839462046FAF739FAF0E730B54A4ABF
:1056C000D2F8043313F4007F85B015464AD0D2F8DF
:1056D0002431002B46D04FF492711046FAF7EEFABF
:1056E0004FF40173C2F80833404B997E09B9012188
:1056F00051603D4902228DF80020D1F88024C1F884
:1057000080240392DA7D8DF80820DA680192002265
:10571000DA751A766846D3E9001290473248D0F815
:105720001C313BB1314A938A917D994247D9114648
:10573000FAF7F3FA2C4AD2F844318BB14FF4A27144
:105740001046FAF7BBFA294B997E09B10121116085
:10575000DA7D2AB10022DA75587ED968F9F75EFF42
:1057600005B030BDD5F804335B07D7D5D5F808317F
:10577000002BD3D01D4C1C482146FAF7B7FA637EA4
:10578000E27D9A422346C9D1227E52B12369E16863
:10579000E3600023607EE27523766376F9F73EFFCF
:1057A000BCE7A27E0AB901226A600F4A4FF4017178
:1057B000C2F808130022DA75587ED968EEE74FF474
:1057C0008E71FAF77BFA917D0029B3D000238DF812
:1057D000081091688DF80030019193756846D2E900
:1057E00000139847A6E700BF002000409CCB002094
:1057F000800000F1A040D0F8003723F44033C0F817
:105800000037D0F8003743EA0141C0F8001770476D
:1058100000F1804000F5C040002382B003600368BF
:105820000193019B02B070472DE9F04F85B0002431
:10583000594D01944FF48072012102F1804303F528
:10584000C04390B21B68012B06D1D5F804330B423C
:1058500002D0FFF7DDFF0C430432B2F5907F4FEA30
:105860004101EAD14D4B1B68012B0AD14FF4BE70A8
:10587000FFF7CEFF4FF0A04344F00044D3F81035BB
:10588000019314F0FF0F1AD0454F01260025344232
:1058900010D0AB0003F1804303F5C043D3F81005EB
:1058A000D3F8101557F8253023B1C1F30141C0F3E7
:1058B000042098470135082D4FEA4606E7D1002C11
:1058C00063DA4FF0FF330022CDE90232344D354E1A
:1058D0000024A24601274FF0A04816F9012B531CC3
:1058E00046D0D2B222F0C0094FEAD90104A8084438
:1058F00002F0070310F808CC07FA03F31CEA030FC1
:1059000036D005EB090C92099CF930C055F82CB043
:10591000BBF1000F0AD1032A2AD10DF10C0E1EF89B
:1059200001C04CEA030C0EF801C001E0032AF4D0D8
:1059300009F5E07110F80C0C58F821101842C1F369
:10594000014105D0022913D1032A0BD1114604E0ED
:1059500003290DD1032A05D102214846FFF748FF4C
:105960000134E4B2BBF1000F02D011464846D847DB
:105970000AF1010ABAF1040FAFD134B14FF0A043DC
:10598000019AD3F81035934202D105B0BDE8F08FEB
:105990000193039B02939AE7006000407C61004002
:1059A00044CB002094CB00200028C3B2A8BF00F154
:1059B00060424FEA501010B5BABF0D4A03F00F0411
:1059C00002F561424FEA41114FEA8000C9B200F18D
:1059D0006040B4BF115582F8001300F5614003F038
:1059E0001F0201239340C0F88031036010BD00BF47
:1059F00014ED00E02DE9F8430446C279C17A0F2086
:105A000027F004FB237B644A0BB3937843F0100325
:105A100093702568EB175906604B41EAD51168066B
:105A20004FF0FF328B4208BF82420AD35C4A002308
:105A30003BF0C4FB00F5006020F47F6727F00F0700
:105A40004FB929465748BDE8F8432DF037BC937845
:105A500003F0EF03DCE7207927F0C8FA40B960795A
:105A600027F0C4FA20B95048BDE8F8432DF026BC11
:105A70004E4EF3781BB10023F370FAF743FE2579FD
:105A800000232846F37027F0B1FA20B14FF440719B
:105A900028461CF0A3F96579284627F0A7FA20B11B
:105AA0004FF4985128461CF099F9637A2579002B18
:105AB000284614BF4FF00E094FF0000927F096FA60
:105AC00000285BD03A4B05EB45051D4495F8018055
:105AD0006479204627F08AFA002852D0344B04EB30
:105AE00044041C446378334CE27E002A4CD15A1C97
:105AF0000AD04FF0A04101229A40C1F8082503F5D1
:105B0000E072032041F82200B8F1FF3F2A4D1FBF89
:105B10004FF0A04108F5E072002041F82200C5F8DE
:105B20002475C5F86C950027C5F81485C5F80C35A3
:105B3000224B636028464FF48E712760FAF7BEF857
:105B40004FF4A271FAF7BAF81D4BC5F804330221DD
:105B50000846FFF729FF0423C5F80035B8F1FF3FD9
:105B60004FF48073E7822776638311D01548FAF7E4
:105B7000ADF80123A376FBF7FDFA09E04FF0FF38FB
:105B8000A6E74FF0FF33AEE708210F482DF076FB74
:105B90000123F370BDE8F883ECCA002047E8010058
:105BA00048E80100251706003A17060001D3002037
:105BB000D01706009CCB002000200040810F04007D
:105BC000800002004C1606005017060010B50D4C60
:105BD00000226260A2602261E2600B4A106810F04D
:105BE000010002D10621FFF7DFFE084B1B7823B925
:105BF0004FF080430122C3F81825012323700020B1
:105C000010BD00BF6CCC002000E100E0E1D100201D
:105C1000F8B50E46D11C48BF911D144641F38701CB
:105C20000546671EFAF738F900214AB2A24201F18F
:105C3000010100DBF8BDBB1A23F00300B25C03F0E6
:105C40000303DB0002FA03F32A581A432A50ECE755
:105C5000F0B500254F1E6CB28C4205F1010500DB4A
:105C6000F0BD3B1B23F0030603F003039659DB0052
:105C700026FA03F30355EEE72DE9F041B3F90240AC
:105C800014F11F0548BF04F13E050F4603F1240639
:105C900045F34715904601462B4632463846FAF7FB
:105CA00037F9B8B9B4EB451F16DA6211012304F0D5
:105CB0001F0403FA04F457F822301C4214BF0124D5
:105CC00000242B46324639464046FAF721F9204651
:105CD000BDE8F0810124F4E70446F2E710B50023A3
:105CE0001A465CB2A14203DCB2FA82F0400910BD50
:105CF00050F8234001332243F3E700002DE9F04F31
:105D00008A46234F8BB00646114650461446FAF792
:105D1000A3F83B68FBB10425C0EB441014FB05FB62
:105D200000B205FB04654FF0FF38043D28FA00F887
:105D30004FF040093B6859463046984758B12B68A8
:105D400003EA08032B6021463046FFF7C7FF20B166
:105D5000B9F10109EED1002017E023463246514641
:105D600002A8FAF7A5F82146019002A8FFF7B6FFAE
:105D7000019B003318BF01235B00002814BF584269
:105D8000C3F10100C0B20128E2D10BB0BDE8F08F31
:105D9000A42E00202DE9F04FD1B0CDE905015B9D87
:105DA00095F9004048A8914622461F46FAF748F860
:105DB000A3000793069BA20013441946224638A865
:105DC0000293FAF73DF895F90060002F00F08C80FF
:105DD0003246394628A8FAF733F80DF5807A32466C
:105DE00030AF48A95046FAF72BF838A93846FAF7E9
:105DF00027F82B4628AA38A948A8F9F7E0FF2B4630
:105E000028AA38A948A8D5F8A460B0472B4628AAE4
:105E100039465046F9F7D3FFBDF968310497023B84
:105E20001BB2002B67DCD9F80030009503F00108A5
:105E30004FEA481840AADB4302EB080A03F00103CB
:105E400030AA90445B0140AA1A44039230AAD318A6
:105E50004146039A0493504605F10409FAF74FFAB4
:105E60004B4640AA48A908A80094FAF7B8F908A92F
:105E700008462B464246F9F761FF08A908462B461B
:105E8000069AF9F75BFF214608A8FFF727FF0028CD
:105E90005DD008A8FAF700F808A92B46029A084630
:105EA000F9F74CFF08A92B4652460846F9F746FF7A
:105EB000DDE90301434652460095FAF7A2F92B4665
:105EC00008AA30A940A8F9F77AFF224640A9059808
:105ED000F9F7B6FF059B079C234430A91846F9F74C
:105EE000AFFF51B0BDE8F08F314628A8F9F7D4FFD5
:105EF0000123289371E71FFA83F85B1108F01F0252
:105F000059F823300095012101FA02F21A42049B4C
:105F100013BF20270027202600260AEB070B1F446B
:105F20000AEB06030393049B039A1E443346394647
:105F30005846FAF7E4F908F1FF383B4600955A460F
:105F400031460398FAF75DF90FFA88F369E710AF65
:105F5000224608A938460DF1600BF9F771FF20AE13
:105F600049465846F9F76CFF30462146F9F794FF49
:105F7000012328A82093F9F78FFF22465946384677
:105F8000F9F749FF28B9224620A908A8F9F758FFD0
:105F900082E73B68DA0709D421463846F9F72EFF35
:105FA000224649463046FAF7FEF8E6E7189BDB073B
:105FB00007D421465846F9F721FF2246494628A82A
:105FC000F1E7002823461CDD5A4639463846F9F7E2
:105FD0006FFF21463846F9F711FF224628A93046BF
:105FE000F9F719FF002805DA23464A4631463046BC
:105FF000F9F78EFF234628AA31463046F9F758FFB5
:10600000CEE73A4659465846F9F752FF21465846D8
:10601000F9F7F4FE2246314628A8F9F7FCFE0028DD
:1060200005DA28A923464A460846F9F771FF28A948
:10603000234632460846F9F73BFFBEE72DE9F04715
:1060400093F9006092B004468946104631461546E1
:106050009846FFF743FE002840F0918042464946AB
:106060000AA8F9F7A8FE43460AAA214602A8F9F7AA
:1060700065FE0AA908464246F9F79DFE43462A46B0
:1060800049464846F9F75AFE08F1040742462946B0
:106090002846F9F790FE3B462A46214620460096C0
:1060A000FAF714F93B462A46294628460096FAF79D
:1060B0000DF93B462A46214628460096FAF78FF806
:1060C00043462A4621462046F9F738FE3B462246FB
:1060D000214628460096FAF7F9F83B4600962A46EC
:1060E00021462046FAF7F2F82368DB074AD5334603
:1060F0003A4621462046F9F70BFF314682462046B4
:10610000F9F77CFE06F18043013B54F8230040EA96
:10611000CA7044F82300424621462846F9F74BFE50
:106120003B4602AA294628460096FAF758F83B460D
:1061300002AA294628460096FAF751F802A908460D
:106140003B462A460096FAF74AF8434602AA2146F9
:106150002046F9F7F3FD0AAA3B4610462146009671
:10616000FAF73DF8324629462046F9F769FE4946D6
:106170002846F9F765FE0AA94846F9F761FE12B00C
:10618000BDE8F08731462046F9F738FEC3E7000046
:1061900073B500230DF102008DF80230FBF7CEF845
:1061A000264B1B7803F0FF04002B41D1244B1A68C7
:1061B000002A3DD0234AD2F80813C90738D51C60FD
:1061C0001B68214D01930DF10300019BD2F8086576
:1061D0008DF80340FBF7B2F86A6829681F2A98BF58
:1061E000541CA142F6B26C6004D1202C14BF611C77
:1061F0000021296015499DF803008E542A689442B5
:106200003ABFC2F121021319A31AAA689A4238BFF1
:10621000AB60FBF799FE6B682A681F2B94BF0133B4
:1062200000239A4201BF074A0123C2F80833536092
:106230009DF80200FBF788FE02B070BDE1D100209E
:1062400000D1004000D00040CCD10020A8D10020D7
:1062500030DF70472DE9F74F3B4F06468846B8F1CF
:10626000000F03D1012003B0BDE8F08F4546202D7B
:1062700028BF20255FFA85FB002400230DF10200D2
:106280008DF80230FBF75AF8304B1B7803F0FF090A
:1062900093BB0DF103008DF80390FBF74FF8D7E99E
:1062A00000148C4204D3641AA54207D9052414E0D3
:1062B0002134641AA542F9D8C1F12104244BA54226
:1062C000194431D82A4630463BF044F93B682B4408
:1062D000212B28BF00233B6000249DF80300FBF71F
:1062E00033FE1C4B00221A601B680193019B1A4B62
:1062F0000122C3F804231A609DF80200FBF724FE74
:10630000B9F1000F08D059463046FFF7A1FF42F21D
:10631000070398420446ADD0022CAED0002CA9D180
:10632000A8EB05082E449AE7224630463BF012F9C6
:10633000074BA5EB040A5246194630193BF00AF9FF
:10634000C7F800A0C8E700BFCCD10020E1D10020F1
:10635000A8D1002000D1004000D0004017B4314A3D
:10636000314B116889B90021304A106820BB0020E8
:106370005A79D40740D408B9002949D01C68DA8872
:10638000234603B05DF8044B1847002111601268E2
:10639000D9680092009A0029E5D0254AD2F8400534
:1063A000814204BFD88801EB8001C2F840155A79B8
:1063B00042F004025A71D7E7002010601268986812
:1063C0000192019A0028D2D0194AD2F83845A04249
:1063D00004BFDC8800EB8400C2F838055A7942F02B
:1063E000020214075A71C3D512F0010402BF64F30C
:1063F000C3025A712046BBE702F00601062907D105
:1064000022F0060211075A7106D56FF3C3025A71C2
:1064100003B05DF8044B7047054AD2F83805D2F84E
:106420004015ABE71451024034CB00200451024028
:1064300000500240A5DF7047A4DF7047A3DF70471C
:106440002DE9F0470E4690B016F0100581469246B1
:106450009846189C0CD011238DF8083023788DF8BD
:10646000093001224FF0000362F342038DF80A3035
:106470001C22002109A8F9F755F88DF8246005B110
:1064800002AD42F64D23ADF80C3063789DF86410F0
:106490008DF804300022A3788DF80530134661F39F
:1064A000C303DBB243F00303CDE906220E950127B7
:1064B00001AD8DF80630089203AE1A9BB9F80000C2
:1064C0008DF80E7004AA09A9CDE90465ADF81CA0E9
:1064D000FDF72CFC58BB42F60813ADF80C3063787E
:1064E0008DF80430A3788DF80530034667F3420336
:1064F0008DF806301A9A98F800308DF8003098F828
:106500000130CDF81A00ADF81E008DF8013032F8D8
:10651000080B8DF80E70022304A9CDE90465ADF8CF
:106520001830ADF81C30CDF820D0FFF787FF10B041
:10653000BDE8F087A1DF704708B5F9F7B9FF10B1E2
:106540004F4B504A1A60F9F793FF28B14E4B4F4A10
:106550001B68C3F342331360F9F7AAFF20B14C4A1A
:10656000D36823F08073D360F9F782FF40B14FF016
:1065700080430022C3F80C21C3F81021C3F838254A
:10658000F9F796FF10B1434B03221A60F9F790FF19
:1065900040B1414B05221A6001229A6700229A609D
:1065A0003F225A603D4B1B78062B50D13C4B1B6859
:1065B0001B074CD13B4B1B6803F0F003502B46D11B
:1065C0004FF08052384BD2F80414C3F82015D2F89B
:1065D0000814C3F82415D2F80C14C3F82815D2F8FF
:1065E0001014C3F82C15D2F81414C3F83015D2F8CF
:1065F0001814C3F83415D2F81C14C3F84015D2F897
:106600002014C3F84415D2F82414C3F84815D2F85E
:106610002814C3F84C15D2F82C14C3F85015D2F82E
:106620003014C3F85415D2F83414C3F86015D2F8F6
:106630003814C3F86415D2F83C14C3F86815D2F8BE
:106640004014C3F86C15D2F84424C3F87025F9F748
:106650000FFF28B1154B164A1B6803F04F03136058
:10666000144AD2F8883043F47003C2F88830BFF37C
:106670004F8FBFF36F8F104B104A1A6008BD00BFD9
:1066800074C007400DF0ADBA440200103C05004054
:10669000F0ED00E0A005004010560040E00F00F0D3
:1066A000E40F00F0E80F00F000C0004058020010B6
:1066B000E40E004000ED00E0A82C00200090D00384
:1066C000002382B0036003680193019B02B070470E
:1066D0002DE9F341844BD3F8042162B3D3F800339E
:1066E0009F0728D5814D8248FFF7EAFF2B7803F0FA
:1066F000FF08F3B97F4F804E7B783C4603F0FF02E2
:10670000002B00F0AF8073684046984701A88DF8D1
:106710000480FAF713FE7B689DF8040001337B6068
:10672000FBF712FC754B0122DA601A60744B0022F1
:106730001A6001232B706C4BD3F81821D2B1D3F817
:106740000023560616D5D3F824356E48DB08C3F36C
:10675000080113F4FF7F18BF0239FFF7B1FF624B46
:106760004FF48052C3F808254A1EFE2A40F2A48046
:106770000122DA615C4AD2F81031D3B1D2F8003389
:10678000DD0616D56048FFF79BFF1023C2F80833DB
:106790005E4BC2F81035FF23C2F814350123D361D4
:1067A0005B4B1C682CB15B4800231A460321006830
:1067B000A0474D4AD2F84C3133B3D2F800331C0312
:1067C00022D55548FFF77CFF4E48FFF779FF534825
:1067D000FFF776FF4D4BC2F81035FF23C2F8143592
:1067E0000123D3614FF48863C2F804330D23C2F848
:1067F0000C34C2F80434464B1C682CB145480023C5
:106800001A4619460068A047374AD2F828315BB1CA
:10681000D2F80033580507D54048D2F80C34FFF7BA
:106820004FFF0D23C2F80C342F4AD2F81C31B3B1FC
:10683000D2F80033190612D53948D2F80414FFF7FC
:106840003FFFCB0707D5374B197821B10121C2F89B
:10685000041400221A70244B0D22C3F8042402B041
:10686000BDE8F0810DF103008DF80320FAF766FD15
:10687000BA68134683B93260A660636833B92A4B9D
:106880001B7803F0FF025BB1F9F7CCF863689DF861
:1068900003000133636043E7B342EED01B68E9E7CE
:1068A000224B1A601B680193019B4FF08043012229
:1068B000C3F804231A60E9E7144A1078502803D17A
:1068C000184901220A7054E711480468002C3FF46B
:1068D00051AF4FF6FF70C3F808050E480B4600682D
:1068E0000221A04746E700BF0050004058CD0020DD
:1068F000045100406CCC002080CC002000B001404E
:10690000A02E0020185100401051004000CF002060
:106910000CD0002010D000204C51004028510040E5
:106920001C510040E0D10020E1D1002000010040D6
:1069300013B5284B2849D3F83C3413F0030345D151
:106940000A680132072A0A602CD9244A01241461FA
:106950000DF107008DF80730FAF7F0FC204B5A686C
:10696000013A5A605A6822B91E4A127802B3F9F7FE
:1069700057F89DF80700FBF7E7FABFF35F8F1A4A55
:1069800000231360BFF35F8F01211160174A146861
:106990001CB117481A460068A047164B00221A700F
:1069A000FAF724FC0D4B0022C3F8402102B010BDC1
:1069B000114A4FF080411460D1F80C2402F001120A
:1069C000B2F1011FF8D000225A70D2E700230B6009
:1069D000E8E700BF00500040A02E002000B00140BA
:1069E0006CCC0020E1D10020FC5F00400CD00020E6
:1069F00010D0002058CD002004000040D0E9012331
:106A000093423FBF026842F82310836801333ABFC4
:106A100083600020042070472DE9F04F87B00D46B9
:106A200093460190C8B1C2B103680393ABB14FF074
:106A30000009C846019B9B68434503D8CBF80090EA
:106A4000002022E0B8F1000F09D1012B0CBFC023B8
:106A50008023039A52F8284044B90E2015E008F12B
:106A6000010293420CBF40230023F2E76178227AAF
:106A7000571869B9971D002D44D0DBF80020A2EB10
:106A80000902BA42029205D2042007B0BDE8F08F95
:106A90000737F0E72B702278AA4613430AF8023B27
:106AA000227A6A7062783ABBAE1D227AE16830467B
:106AB0003AF050FD237A62781E442AB1304661686C
:106AC0003AF048FD63781E44029BDB1B0593236963
:106AD000002BC2D005AA3146606998470028D4D15E
:106AE000059B16B11ABACAF800201F44B94405B173
:106AF0003D4408F101089DE743F00803EE1DAA712B
:106B00002B70D2E7AA462E46E1E710B5144661B1D4
:106B100013689BB14378027803F00F0343EA021332
:106B200001F8013B2368013B236022464068FFF7E0
:106B300073FF10B923680133236010BD0420FCE704
:106B40008DDF704777DF70472DE9F04F89B00E4633
:106B500000AF0023044607F1140130467B6132F098
:106B60007FFC054618BB304633F0D6FD8046786181
:106B70002BF0CEFB08F5807383420CD9A649012087
:106B80002CF028F83246A54901202CF023F82437B0
:106B9000BD46BDE8F08F08F1070323F00703ADEB16
:106BA000030D6D4642462946304633F023FF7E6989
:106BB00026B99B4901202CF00DF8E8E74FF00308B7
:106BC000B6FBF8F303EB43039E4201D09549F1E78E
:106BD000204626F00BFA08B99349EBE7934BC7F828
:106BE00008D004EB44041C446178914C20790028BF
:106BF00040F009818F4A0123C2F80405FF29C2F839
:106C00002405C2F82005C2F81C35C2F82805C2F8D0
:106C100018054FF0C050C2F81405C2F8103518BF5F
:106C200001F5E0704FF0A04308BF4FF0FF31C3F80B
:106C30003887C3F8FC8A18BF43F820800E23C2F8B7
:106C40006435FF23C2F868354FF0FF33C2F8603572
:106C50002520C2F87015C2F86C350221764B2360EE
:106C6000FEF7A2FE012323710323B6FBF3F39BB2CD
:106C700003EB430808F1010828F001029100ADEB95
:106C8000010D6846FA606D4A3A6041184FF0000CF9
:106C9000796082F800C0E91C4FF0EE09851C4FF0C6
:106CA000880A4FF08E0B63455FDC0C2202FB030366
:106CB00000227968994200F29E802679012E40F0E8
:106CC000A28000F06043B3F1005F40F0A280FB6857
:106CD000C3F34E02574B0021C3F85025C3F83815B3
:106CE000C3F80815C3F84005C3F80C656579E28060
:106CF00025F0090545F008056571C4E90210C3F8DF
:106D00000065022323710D46002977D04FF6FE72ED
:106D100008EA0202F8F706FC494B00221A601B68D9
:106D2000FB61FB69474B1A601B68BB61BB69414B48
:106D30002222C3F8042301221A603A681278042A36
:106D4000FBD94149002222250120C3F808530860DD
:106D5000C3F80025C3F808530860C3F800253B4B6F
:106D60002021C3F88410227150E011F8026C11F850
:106D7000032C360246EA024611F8012C05F10C0EEE
:106D8000164306F44012B2F5001F1ED0B2F5401FA4
:106D900020D0B2F5801F20D105F802BC06F44002D5
:106DA000B2F5000F1CD0B2F5400F1ED0B2F5800F27
:106DB0001ED105F801BC0235AE454FEA0616E0D1FA
:106DC0000CF1010C033175466DE76FF0170205F801
:106DD000022CE3E705F8029CE0E705F802ACDDE7EA
:106DE0006FF0170205F8012CE5E705F8019CE2E7D2
:106DF00005F801ACDFE703F8012B5AE701462368E9
:106E00002846984788E70820FBF73CF8D7F808D0D1
:106E1000BDE61020F8E700BFFF220600262306008B
:106E200052230600722306009D230600D017060099
:106E300034CB002000500240458D030080D5002057
:106E400004510240145102400450024000E100E0AD
:106E500070B500221649054633F004FB34F022F9E0
:106E6000144B154906460322586833F0FBFA0446D2
:106E700078B10022B1B233F027FAE389A3F50073A9
:106E80009BB2E381E38903F4F05313B9204631F058
:106E900097FC0A4B1C6824B1E38903F500739BB28D
:106EA000E3812846002115F0F5F9204670BD00BFAA
:106EB000991906008C2E0020A619060058D500202E
:106EC00010B5838AC3F30C0413F4604301D1204648
:106ED00010BDB3F5005F02D106206043F8E7B3F5BB
:106EE000C04F07D100220449006833F0BBFA34F0E8
:106EF000D9F8F2E70020EBE7D721060008B540B249
:106F0000FFF720FEBDE8084015F04CBC38B505463B
:106F100008460C4630F03AFF002808BF00242246FD
:106F20000E49284633F044FA0D4B4FF6FF7219888C
:106F300074B18A4204D10020BDE8384015F032BC5B
:106F40000022188811461AF095FA0828F4D1F2E7C1
:106F50008A42F0D018881AF08BFAF6E77419060006
:106F60008C2D0020014B188815F0FCBE8C2D0020C4
:106F7000014B188815F0F6BE8E2D002008B5074B82
:106F80001A884FF6FF71914207D018881321FDF738
:106F9000C9FEBDE8084015F005BC08BD8E2D0020D7
:106FA00007B500230846072269460093CDF8033051
:106FB00034F014FC094B1A884FF6FF71914209D046
:106FC00018886A4601211AF059FA15F0EBFB03B054
:106FD0005DF804FB43F20200F7E700BF8C2D0020B0
:106FE00038B500220E49054633F03CFA0446A8B9EC
:106FF0000C4929F0C9F80A4904460246284633F0EC
:10700000D7F92A460849204633F0D2F9002031F05A
:10701000A6FB06490246204633F0EBF9204638BD70
:107020004E190600531906006D1906008F19060047
:1070300010B5044630F092FE224630B92CB1074913
:107040000320BDE810402BF0C5BD054B054958682D
:1070500034F014F9BDE8104016F00EB9211E0600F8
:107060008C2E00204A1E0600F8B5044628B9214A95
:10707000136823F480431360F8BD1F4931F038FFD3
:107080000028F4D1204630F0A5FE054690B1194AFB
:107090001368204643F48043136034F033FC53EC10
:1070A000102B10EE100A19461EF0CAFDBDE8F8407C
:1070B00015F078BB204630F051FE0028DCD00D4A98
:1070C0000E49136843F48043136020462A4633F088
:1070D000C9F934F0EDFE2A4606460F462046084917
:1070E00033F0C0F934F0E4FE02460B463046394630
:1070F000DAE700BF5CD50020161D06001B1D060048
:10710000271D0600084B1A6818B142F400521A6095
:10711000704722F400521A60044B1860044B01229D
:107120001A7015F07BB800BF5CD500208CD500200C
:1071300089D50020F0B583B0044600AF28B90146D8
:1071400015F0B2F90C37BD46F0BD30F0F0FF28B1B4
:10715000204632F01BFF0421C0B2F1E77860391DF0
:10716000204632F07DF90546F0B9204633F0D4FAD6
:10717000064678602BF0CCF806F58073834208D978
:107180000D4901202BF026FD0C4901202BF022FD9A
:10719000D8E7F31D23F00703ADEB030D6D46324630
:1071A0002946204633F026FC79680029ECD0284691
:1071B00015F0ACF9C6E700BFFF2206004325060024
:1071C00008B5044B0449586834F03EF8BDE808405F
:1071D00015F0D4B98C2E002083250600F0B583B0BD
:1071E000044600AF15F0CAF9002C69D00023391D00
:1071F00020467B6032F034F9054610BB204633F060
:107200008BFA064678602BF083F806F5807383428C
:107210000CD93A4901202BF0DDFC394901202BF033
:10722000D9FC002420460C37BD46F0BDF31D23F0E9
:107230000703ADEB030D6D4632462946204633F079
:10724000D9FB78680028E8D031F08CF9044608B9F9
:107250002C49E3E72C4B2D490246586833F0A8F837
:10726000E389A3F500739BB2E381E38903F4F05350
:1072700013B9204631F0A4FA204630F0CDFD7A68EB
:1072800029463AF067F9204630F0C6FD054620460B
:1072900032F0BDF80146284615F080F90023391D6B
:1072A0000A207B60F9F784FE7B680446002BB9D086
:1072B000174A116819605168596012891A81B1E73B
:1072C000204631F04FF9044620B90E4901202BF039
:1072D00081FCA7E70C4B0D490246586833F068F86B
:1072E000E389A3F500739BB2E381E38903F4F053D0
:1072F000002BC8D1204631F063FAC4E7FF22060014
:10730000432506005A2506008C2E00208325060002
:10731000FFCF0020F0B583B0054600AF48B9424B1F
:107320004249586833F090FFFFF74AFF0C37BD46DB
:10733000F0BD0023391D7B6032F092F80646F0B9AB
:10734000284633F0E9F9044678602AF0E1FF04F5B5
:107350008073834208D9364901202BF03BFC354924
:1073600001202BF037FCE1E7E31D23F00703ADEB31
:10737000030D6E4622463146284633F03BFB7868C3
:107380000028ECD0133031F0EDF8054608B92A4951
:10739000E6E7254B25490246586833F009F82846A8
:1073A00030F03AFDEB89A3F500739BB2EB81EB89DA
:1073B00003F4F053044613B9284631F001FA1F4B89
:1073C000224603F1100153F8040B42F8040B8B42E0
:1073D000F9D11B8813807D6831462A4604F11200DA
:1073E0003AF0B8F865742544FE23AB740020FFF72B
:1073F000F5FE3946054632F033F828B103682360BC
:107400004368636003892381002D8FD0EB89A3F546
:1074100000739BB2EB81EB8903F4F053002B85D111
:10742000284631F0CDF981E78C2E00203B2506005F
:10743000FF220600432506005A2506009B18060079
:10744000F0B5ADF5037D064600AF50B9374B38496E
:10745000586833F0F9FEFFF7B3FE07F50377BD4632
:10746000F0BD0023391D7B6031F0FAFF0446F0B90E
:10747000304633F051F9054678602AF049FF05F5AA
:107480008073834208D92B4901202BF0A3FB2A49A2
:1074900001202BF09FFBE0E7EB1D23F00703ADEB92
:1074A000030D6C462A462146304633F0A3FA7B682A
:1074B000002BECD04FF40072204D3A600022AA60FD
:1074C0001F4A20491460DBB228465360FFF796FA42
:1074D00038B9AB6883B13A4607F108012846FFF78F
:1074E0009BFA15F05FF90028B7D1386831F03AF807
:1074F000044618B91449CBE70720F2E730F08CFCBA
:107500003A6807F108013AF025F82046FFF702FF34
:10751000E389A3F500739BB2E381E38903F4F0539D
:10752000002B9AD1204631F04BF996E78C2E0020A3
:107530003B250600FF220600C5240600A82D0020DA
:1075400050D50020382D0020DC2406002DE9F04322
:10755000E1B0054600AF58B9634B6449586833F051
:1075600073FEFFF72DFE07F5C277BD46BDE8F08339
:107570000023391D7B6031F073FF0646F0B92846C1
:1075800033F0CAF8044678602AF0C2FE04F580732E
:10759000834208D9564901202BF01CFB5549012094
:1075A0002BF018FBDFE7E31D23F00703ADEB030D22
:1075B0006E4622463146284633F01CFA7B68102B73
:1075C000ECD107F108044FF480733C2200212046DF
:1075D00007F144054FF001083B604FF00209F7F74F
:1075E000A1FF40F201433C2200212846BE637B817B
:1075F00087F8089087F8358087F83680F7F792FF8C
:107600007E673D4E3D4BBB6773693D495B6887F8BC
:10761000468000229A60736987F844905868FFF7A3
:10762000EDF900283AD1736936495868FFF7E6F951
:10763000002833D1344B354A1B781370DFF8E480CF
:10764000334AC8F81440003318BF012388F80130CA
:10765000304B314C1B78DFF8D0901370003318BFDB
:107660000123A06031462046C9F8145089F8013042
:10767000FFF7C4F990B941462046FFF7BFF968B952
:1076800049462046FFF7BAF940B9244B3A461860FC
:10769000988007F180012046FFF7BEF915F082F8C7
:1076A00000287FF460AF386830F05CFF044608B90A
:1076B0001B4974E730F0B0FB3A6807F1800139F0FC
:1076C00049FF2046FFF726FEE389A3F500739BB22E
:1076D000E381E38903F4F053002B7FF444AF2046A9
:1076E00031F06EF83FE700BF8C2E00203B250600EE
:1076F000FF22060009250600602D00206F260600E7
:107700000C2D0020E02C0020532D0020A8D50020B7
:10771000A9D50020522D0020542D002000D2002099
:10772000DC240600B42D0020902D00202DE9F0412E
:1077300082B0054600AF50B9594B5A49586833F0EA
:1077400083FDFFF73DFD0837BD46BDE8F08130F011
:107750001EFC28B92A46544903202BF03BFAF2E7D5
:107760000023391D28467B6031F07AFE0446F0B9CB
:10777000284632F0D1FF064678602AF0C9FD06F5AA
:107780008073834208D9494901202BF023FA4849E4
:1077900001202BF01FFAD6E7F31D23F00703ADEB12
:1077A000030D6C4632462146284633F023F97D68A6
:1077B000002DECD007223F49204639F0BDFE60B9CC
:1077C000073D07347D604FF0030878681B3030F0C8
:1077D000C9FE064680B93849DAE70822374920460B
:1077E00039F0AAFE28B9083D08347D604FF004083E
:1077F000EBE74FF00008E8E7294B2A4902465868B2
:1078000032F0D6FD304630F007FBF389A3F5007364
:107810009BB2F381F38903F4F053054613B9304664
:1078200030F0CEFF264B2A4603F1180153F8040B23
:1078300042F8040B8B42F9D11B8813807E6885F8CF
:1078400019802146324605F11A0039F083FEF3B261
:1078500003F108022E440133EB75FE236A74002005
:10786000B376FFF7BBFC3946044631F0F9FD28B189
:1078700003682B6043686B6003892B81002C3FF405
:1078800062AFE389A3F500739BB2E381E38903F45C
:10789000F053002B7FF457AF204630F091FF52E7B2
:1078A0008C2E00203B25060059240600FF220600EE
:1078B000742406008B2406009C24060093240600F2
:1078C0009B18060010B5044630F060FA084B0949D1
:1078D000002808BF00242246186832F069FD201CE9
:1078E00018BF012014F0DAFEBDE8104014F05ABFB2
:1078F0008C2E0020741906002DE9F74F504B51498A
:1079000005460322586832F0ADFD0646002845D0F2
:1079100000224D49DFF83081284632F0A3FD314680
:10792000814668462CF038FA009CECB1204632F0D3
:10793000F5FA00224146074632F094FD0123002269
:1079400049468246F9F718F858BBFB8903F50073DE
:107950009BB2FB813C465046394632F003FA6846FA
:107960002CF0DEF9002CDFD0009850B1C389A3F5CC
:1079700000739BB2C381C38903F4F0530BB930F099
:107980001FFF2946002C57D001A82CF005FA019DB5
:107990004DB932464946204632F0B8F903B0BDE849
:1079A000F08F0024D7E7EB8903F500739BB2EB81DE
:1079B000284632F0B3FA012229460746204633F022
:1079C0007FF922498046284631F092FA20498246C2
:1079D000284631F08DFABAF1000F00D1D0B14046FF
:1079E00032F09CFA834610B3BAF1000F1BD001228B
:1079F000394635F053FDBBF80E20A2F5007292B265
:107A0000ABF80E20BBF80E2002F4F05212B9584623
:107A100030F0D6FE40463A46294632F077F901A8C2
:107A20002CF07EF9B3E7394633F0A7F9E3E739469E
:107A3000404632F09DF8EDE7304632F0CBFBA8E748
:107A40008C2E0020CA1A0600241C0600D11A06003B
:107A5000DA1A0600F8B5064608460C4630F07EF9FC
:107A6000074620B300223949204632F0FBFC33F0B0
:107A700080FC002207463649204632F0F3FC0446DB
:107A8000E0B130F063F9C8B9E389A3F500739BB2A4
:107A9000E381E38903F4F05313B9204630F090FEFC
:107AA00022462C490320BDE8F8402BF093B82CB1B6
:107AB0002246294903202BF08DF83C46304630F011
:107AC00065F900283AD0002E38D048F24801234802
:107AD00030F02EFE0546D0B12246002133F016FAD2
:107AE00032461F49284632F063FC1E4B1E49186877
:107AF0002A4632F05DFCEB89A3F500739BB2EB8163
:107B0000EB8903F4F05313B9284630F059FE301CCA
:107B100018BF0120394614F0EBFD14F043FEA4B168
:107B2000E389A3F500739BB2E381E38903F4F05387
:107B30005BB92046BDE8F84030F042BE094B0A4927
:107B4000186833F081FB0026E1E7F8BD3D1D060013
:107B5000E61B0600441D0600781D0600D1800200C9
:107B6000911D06008C2E0020961D06002DE9F8437D
:107B700080460C4630F00AF930B9394942460120B6
:107B8000BDE8F8432BF026B8204630F023F905462F
:107B90002046C5B133F0B6FE57EC106B00243246D8
:107BA0003B463046394639F05BFA30B900222D4B5E
:107BB0003046394639F02CFAC8B12B490120BDE8CE
:107BC000F8432BF007B830F0C9F850B12A462749DE
:107BD000204632F047FC40B134F06AF906460F46C1
:107BE000DDE714B122462249C9E7224F0026224D83
:107BF000D5F8049030F0A6FD20490246484632F000
:107C0000F8FB42461E49686832F0D2FB08211D4845
:107C100030F08EFD054670B12146FFF71BFFEB8962
:107C2000A3F500739BB2EB81EB8903F4F05313B916
:107C3000284630F0C5FD32463B46134824F0B6FFD7
:107C400060B1C389A3F500739BB2C381C38903F4F8
:107C5000F0531BB9BDE8F84330F0B2BDBDE8F8837E
:107C6000601A060000002440B11A0600B91A060086
:107C70008E1A060000409F408C2E0020CA1A060073
:107C8000C11A0600F97802008D7C020037B5144C49
:107C900000210846FFF7DEFE03221249606832F039
:107CA000E1FB002201901049606832F0DBFB0D49D6
:107CB0000546606833F0C8FA0B49606833F0C4FACF
:107CC000019B33B12DB1012301AA2946002024F0E4
:107CD0008FFF2946019832F045F803B030BD00BF50
:107CE0008C2E0020CA1A0600C11A06001FB54FF0DC
:107CF0008052D2F8A430D2F8A820D8B20290C3F3B0
:107D000007200190C2F30721C3F3074000901B0E28
:107D1000D2B241F0C001034831F02AFA05B05DF853
:107D200004FB00BFE61A06002DE9F04786B00E46B8
:107D3000014601A82CF030F8019888B90446019852
:107D400050B1C389A3F500739BB2C381C38903F407
:107D5000F0530BB930F034FD204606B0BDE8F08793
:107D600032F0DCF80022B349054632F07BFB0746CF
:107D7000002800F003810022AE49304632F072FB49
:107D80003946804602A82CF007F801240298002802
:107D900040F0C3804146384631F0E4FF0022A64956
:107DA000284632F05FFB0746E0B10022A249304688
:107DB00032F058FB8046384630F030F9002800F0A9
:107DC000DF80404630F02AF9002800F0D980414693
:107DD000384631F04DFC00284146384608BF0024A3
:107DE00031F0C0FF00229549284632F03BFB0746A0
:107DF00010B300229049304632F034FB80463846BA
:107E000030F0C5F898B1404630F0C1F878B1384646
:107E100031F0C9FA8146404631F0C5FA814506D8AD
:107E20000123002241463846F8F7A6FD00B10024A0
:107E30004146384631F096FF00228149284632F00B
:107E400011FB074680B100227D49304632F00AFB23
:107E500001468046384631F00BFC41460028384642
:107E600008BF002431F07EFF00227649284632F018
:107E7000F9FA0746D0B12FF071FF58B1394605A87D
:107E80002BF08AFFDFF8BCA1DDF81480B8F1000FF9
:107E900040F08980FB89A3F500739BB2FB81FB89CD
:107EA00003F4F05313B9384630F08AFC00226649D7
:107EB000284632F0D7FA0746D0B12FF04FFF58B11D
:107EC000394605A82BF068FFDFF88491DDF81480AF
:107ED000B8F1000F40F09180FB89A3F500739BB2CD
:107EE000FB81FB8903F4F05313B9384630F068FC8A
:107EF0005DB1EB89A3F500739BB2EB81EB8903F4D1
:107F0000F05313B9284630F05BFC01A82BF008FFB2
:107F1000002C3FF411AF012411E7B8F1000F10D08D
:107F200031F0FCFF014603A81AF090FE414604A878
:107F30002BF032FF4FF00009049838B9B9F1000F67
:107F400000D1002402A82BF0EBFE1FE731F0E6FF82
:107F5000014605A81AF07AFE9DF80E209DF816300D
:107F60009A4207D1BDF81420BDF80C309A4208BFE0
:107F70004FF0010904A82BF0D3FEDDE701240DE743
:107F8000324BF81A0011013082B2B8F1000F08D05C
:107F9000A8EB03000011013080B2131A5842584177
:107FA00019E74046F9E7B8F80E3003F500739BB2C5
:107FB000A8F80E3000225146304632F053FA81467E
:107FC00040B900244046494631F0CCFE05A82BF0CC
:107FD000A7FE59E70022414632F072FE0028F0D099
:107FE000C389A3F500739BB2C381C38903F4F05323
:107FF000002BE7D130F0E4FBE4E7B8F80E3003F5EE
:1080000000739BB2A8F80E3000224946304632F089
:1080100029FA82460146404631F02AFB51460028A3
:10802000404608BF002431F09DFE05A82BF078FEE5
:108030004CE700BFD11A0600D7240600371A060005
:10804000241C0600DA1A0600421A0600AC2E002094
:10805000531A060073B504460E462FF077FE38B962
:108060001A4903202AF0B6FD0025284602B070BD4B
:1080700030462FF06BFE0028F2D030F063FB05464F
:108080000028F2D0214601A82BF086FE0198002896
:10809000EBD031F043FF044601463046FFF744FE83
:1080A00018B12146284632F095F85CB1E389A3F572
:1080B00000739BB2E381E38903F4F05313B92046C4
:1080C00030F07EFB01A82BF02BFEDFE7111A060033
:1080D0002DE9F04F87B000AFC7E902011446002A2E
:1080E00076D09549002028F04FF8002205463861E7
:1080F0009249204632F0B6F990490246284632F0BD
:1081000078F900228E493D69204632F0ABF98C495E
:108110000246284632F06DF930F014FB804605F037
:1081200003FD002283468749204632F09BF98146B1
:10813000E8B102468349386932F03AF9002307F181
:10814000140148467B6131F08BF9044600284ED17A
:10815000484632F0E1FA054678612AF0D9F805F58B
:108160008073834238D9784901202AF033FDB8F171
:10817000000F07D0D8F8003023B142467349386960
:1081800032F016F9584631F042F920B15A4670499A
:10819000386932F00DF95A464146484631F0B6FD8D
:1081A000FB68002B40F0C08007F110030122002182
:1081B000B86826F09DFD386950B1C389A3F50073F6
:1081C0009BB2C381C38903F4F0530BB930F0F8FAC2
:1081D0001C37BD46BDE8F08FEB1D23F00703ADEB68
:1081E000030D6C462A462146484632F003FC7B6963
:1081F000002BBCD0B8F1000FC4D0BBF1000FB6D03B
:10820000002514E0092A09D1A91C2144701ED7F8C1
:1082100010A031F0DBFB4F49024619E0911E012905
:1082200027D89A4602239E4216DA013635447B69E6
:10823000AB429CD96319665D5A78082AE2D1A91C21
:108240002144701ED7F810A031F0C0FB424902460D
:10825000504632F0CEF8E8E73AF8021F3F487B601C
:1082600030F086FF0146404631F0D6FF7B6802338E
:10827000D9E7911F012908D8A81C20441AF086FDCF
:108280000146404631F0C8FFCFE7162A33D159885E
:10829000324830F06DFF34F060F882460028C4D0D8
:1082A00001220146584632F00BFD291D7860214419
:1082B000F01E30F049FB7B6802463BB130B101460D
:1082C0003860184631F054FCD7E9002318461146AF
:1082D00031F048FDBAF80E30A3F500739BB2AAF84E
:1082E0000E30BAF80E3003F4F053002B9DD15046F7
:1082F00030F066FA99E7FF2A97D1D8789B78D7F8BB
:1083000010A043EA002030F032FA154902465046E8
:1083100032F06FF8291D2144F01ED7F810A030F07C
:1083200013FB1049024693E7D7E90301FFF7FCFC72
:1083300000287FF439AF3EE7071E0600241C060024
:108340007A19060055250600FF220600D11A0600FC
:10835000DA1A0600D7240600171E060089680600F0
:10836000531A0600421A06002DE9F04186B000AF0C
:1083700000238846391D06467B6031F071F80546BA
:10838000E0B9304632F0C8F90446786029F0C0FF01
:1083900004F58073834206D93F4901202AF01AFC74
:1083A00032463E4938E0E31D23F00703ADEB030DF1
:1083B0006D4622462946304632F01CFB7B68002B76
:1083C000EED040462FF0E2FC28B1354B3549186815
:1083D000424631F0EDFF344B1A6812F0400F1E4652
:1083E00007D1324901202AF0F5FB1837BD46BDE818
:1083F000F0812F4A12884FF6FF71914201D12D4929
:10840000F0E71A6812F0800201D02B49EAE77C6895
:10841000102C05DD2949102201202AF0DBFBE4E7BE
:10842000274B93F800C0274BA4B2BCF1000F23D117
:108430009A7C62B3B3F8760188422AD09B8A7C800A
:10844000C7F80AC0A7F80EC03B810123BB7207F131
:108450000801BB1CC7E90435FBF766FC18B97B882B
:10846000A34218BF0C2014F09DF90028BDD1336839
:1084700043F080033360B8E7B3F87601884208D050
:108480007C80C7F80A20FA81B3F84E31DCE7072078
:10849000E9E70820E7E700BFFF2206008D1C060081
:1084A0008C2E00201D1C06005CD50020271C060019
:1084B0008E2D00203B1C06004A1C0600621C060094
:1084C00088D500206CCD00202DE9F04FB04B91B045
:1084D0001B681B0700AF044607D5AE4901202AF0F0
:1084E00079FB4437BD46BDE8F08F14F0DBFF204632
:1084F0002FF034FC8046002800F05E81214607F111
:1085000014002BF049FCDFF8ACA2796981B100239B
:10851000BB61CB8903F500739BB2CB8107F11800D7
:108520001AF094FB024698B19B4901202AF052FBB5
:1085300078690028D5D0C389A3F500739BB2C381A5
:10854000C38903F4F053002BCBD130F039F9C8E7DD
:108550007D691DB1284631F0E1FC0546294607F149
:108560001C002BF019FCF969B8F1000F0FD071B1A4
:10857000CB8903F500739BB2CB8107F120001AF081
:1085800065FB024610B3854901202AF023FBF869F8
:1085900050B1C389A3F500739BB2C381C38903F4AF
:1085A000F0530BB930F00CF95DB1EB89A3F5007312
:1085B0009BB2EB81EB8903F4F05313B9284630F0FA
:1085C000FFF807F114002BF0ABFB9EE707F1280042
:1085D0003C8C97F822601BF0E1F908B1F9F752FCE6
:1085E0004FF00009002207F13001388DC7F83090B4
:1085F0001BF0D2F9052810D043F2030290420CD0B0
:10860000A8B93B8EA34214D197F83230B34210D1AF
:10861000B7F82890B9F1000F0FD1386A1AF0CCFBE7
:108620005F490446024601202AF0D4FA48E0F9F7EF
:1086300029FC3B8D01333B85D4E7FC691CB1204606
:1086400031F06CFC044600225649204631F00AFF06
:10865000002255490646204631F004FF32F089FEDB
:108660000022B8605149204631F0FCFE32F081FE14
:10867000F8602EB3002307F1240130467B6230F00E
:10868000EFFE8346002837D1304632F045F8786255
:10869000786029F03DFE7A6802F58073834221D923
:1086A000434901202AF096FAF389A3F500739BB29F
:1086B000F381F38903F4F05313B9304630F080F8B6
:1086C0005CB1E389A3F500739BB2E381E38903F412
:1086D000F05313B9204630F073F807F11C002BF06B
:1086E0001FFB40E7D31D23F00703ADEB030DEB4663
:1086F0005946304632F07EF97A6A002AD4D00021F9
:1087000079853A85494607F12802BAF80000C7F88A
:108710002CB0FDF791FE14F045F8BB6880F0010025
:108720005FFA80F813B9FB68002BBDD0BAF80020BF
:108730004FF6FF719142B7D0FB68BAF80000A7F876
:1087400030900022002BC7F83220FA867A6A7A82AB
:1087500014BF0222012287F8322007F1300107F10D
:108760001202C7E90E2BFBF7DFFA30F008029BD0AC
:1087700043F20402904297D043F20142904293D0D8
:1087800014F010F8002818BF4FF000088CE700BF65
:108790005CD50020B71E0600DF1E0600F81E06008E
:1087A000281F0600D6420600181F06001F1F0600DD
:1087B000FF2206008E2D0020002C3FF492AE2246B0
:1087C000024903202AF006FA8BE600BF4C1F060080
:1087D0002DE9F04F9BB000AF0D4604463C2200212E
:1087E00007F12C00F6F79EFE022387F82C3028466E
:1087F000062387F82F302FF0B1FA002800F08D8083
:1088000000228E49284631F02DFE38B132F0B1FDFC
:10881000002814BF0223002387F82C300022884947
:10882000284631F01FFE38B132F0A3FD002814BFF6
:108830000623052387F82F3000228249284631F08D
:1088400011FE064618B3002307F10C01FB6030F05F
:1088500007FE804600284ED1304631F05DFF81464C
:10886000F86029F055FD09F58073834237D97649C0
:1088700001202AF0AFF9F389A3F500739BB2F381CD
:10888000F38903F4F05313B930462FF099FF2846CB
:1088900000226E4931F0E6FD054690B13B6D002B9C
:1088A00036D031F073FB3B6D1880EB89A3F5007374
:1088B0009BB2EB81EB8903F4F05313B928462FF0F8
:1088C0007FFF20462FF042FA80B3E38903F500735F
:1088D0009BB2E38120466C37BD46BDE8F08F09F1BD
:1088E000070323F00703ADEB030DE8464A46414674
:1088F000304632F07FF8FA68002ABCD084B06B466C
:108900004FF6FF713B6519809A80C3F80880B2E783
:108910004F4903202AF05EF9C7E7002DD1D04D4919
:108920002A4603202AF056F90024D3E720462FF0E8
:10893000F1F906460028C8D120462FF00FFA00288A
:1089400076D0204630F01EFA0C235843073020F032
:108950000700ADEB000D214607F108002BF01CFAD3
:10896000E946DFF8E4B04D46B246B868C0B987F8CA
:108970005860C7F854901F2307F1080207F10C0153
:1089800007F12C003B81FCF775FA13F00BFF002870
:10899000CAD107F10C0138892FF0D6FF044699E7B8
:1089A00031F0BCFA07F10C010446C7F80CA030F016
:1089B00057FD804678B9204631F0AEFEF860786009
:1089C00029F0A6FC7A6802F58073834225D95946BE
:1089D00001202AF0FFF85CB1E389A3F500739BB294
:1089E000E381E38903F4F05313B920462FF0E8FE46
:1089F000B86820B1C38903F500739BB2C38132F01C
:108A000051FBFB682880AB80C5F8088007F108009F
:108A10002BF086F901360C35A7E7D31D23F00703A9
:108A2000ADEB030DE8464146204631F0E3FFD2E7C7
:108A3000002CA0D02246084973E700BF041B0600A3
:108A40000D1B0600421A0600FF220600531A0600FC
:108A50001A1B06004E1B0600841B060008B5054ABB
:108A6000136823F40073136014F0F4F9BDE80840B0
:108A700013F098BE5CD5002008B5054A136843F48E
:108A80000073136013F05EFEBDE80840FEF776BA8F
:108A90005CD5002008B518F033FD41EC100B08BD83
:108AA00008B50C4B1B884FF6FF729BB2934203D163
:108AB000094A1288934208D0084824F025F9084A48
:108AC000136843F00803136008BDBDE8084016F0C2
:108AD0004FB900BF8C2D00208E2D0020EE1B06000C
:108AE0005CD5002038B50F4C0F4900220546606860
:108AF00031F0B8FC32F0D6FAC3B27DB143F00100D8
:108B000098420ED064682FF032FE07490246204694
:108B100031F06FFCBDE83840FFF7C2BF03F0FE0044
:108B2000EEE738BD8C2E0020331D06002DE9F04104
:108B30008CB006460F462FF011F940B93EB13246CF
:108B4000524903202AF046F80CB0BDE8F08100231A
:108B5000029301934E4B039302AB05934D4B069347
:108B60004FF003080B23ADF81C300DEB0803012276
:108B70000893494B8DF803200993424601AB03A9A2
:108B80003846ADF81080ADF828800B9332F02CFFFA
:108B90000028D9D00298414D414C2FF023FA48B11A
:108BA000029A4049686831F003FC236843F00803E7
:108BB000236009E0029B002B4AD13A49686832F0F1
:108BC00043FB23685906F0D4029850B1C389A3F53A
:108BD00000739BB2C381C38903F4F0530BB92FF028
:108BE000EFFD9DF80330002B37D023682E496868CD
:108BF0009A065EBF236843F00803236032F024FB2B
:108C000032462A49686832F039FB3A462849686892
:108C100032F034FB019A1AB1236843F00803236051
:108C20002449686832F02AFB019850B1C389A3F542
:108C300000739BB2C381C38903F4F0530BB92FF0C7
:108C4000BFFD236813F0180F1BD0FFF729FF7BE748
:108C50001949404629F0BEFFB6E72368D5F80480DD
:108C60009B0648BF23684FF0000044BF43F0080351
:108C700023602FF074FD0C490246404631F0B9FBE9
:108C8000BEE7304615F062F95EE700BF4C1F0600F4
:108C9000231C0600521E0600571E06008C2E0020C4
:108CA0005CD50020611E0600901E0600991E06007D
:108CB000A31E0600AD1E06006B1E060013B5694616
:108CC000044619F0D7FF28B90749012029F082FF8F
:108CD00002B010BD054B06495868224631F068FBCA
:108CE000FFF7DEFEF4E700BFA51C06008C2E002077
:108CF000DB1C060070B50D4D2A7806460C462AB1DD
:108D000001200B4929F066FF002070BD09F010FF1B
:108D1000084B2E70186024B1E38903F500739BB2F1
:108D2000E381054B01201C60EFE700BF60D5002008
:108D30000B19060058D5002064D5002037B505462C
:108D4000002105208DF80610FFF7D4FF70B1084B05
:108D50001C6824B1E38903F500739BB2E381019998
:108D6000284613F019FB204603B030BD0446FAE74D
:108D700058D5002037B505460C4605200021FFF7E1
:108D8000B9FFD0B1214601A819F0A6FE024638B1BC
:108D90000B49012029F01EFF0024204603B030BDFE
:108DA000084B1C6824B1E38903F500739BB2E3818F
:108DB0000199284613F0F0FAEFE70446EDE700BF0B
:108DC000013D060058D5002013B5002104208DF880
:108DD0000610FFF78FFF68B1074B1C6824B1E389C9
:108DE00003F500739BB2E381019813F025FB204645
:108DF00002B010BD0446FAE758D5002013B50C4662
:108E000004200021FFF776FFC8B1214601A819F020
:108E100063FE024638B10B49012029F0DBFE002435
:108E2000204602B010BD084B1C6824B1E38903F54D
:108E300000739BB2E381019813F0FEFAF0E7044659
:108E4000EEE700BF013D060058D5002038B5124DB1
:108E50002A8801464FF6FF70904215D00320FFF795
:108E600049FF78B10D4B1C6824B1E38903F5007309
:108E70009BB2E38113212888FBF754FF13F092FC87
:108E8000204638BD0446F5E7FDF75AFEBDE83840F8
:108E9000084609F0C1BE00BF8C2D002058D5002027
:108EA0002DE9FF4100220F463849804631F0DAFAB9
:108EB00000223749064631F0D5FA6946054619F0D1
:108EC000D9FE044658B92946304630F04BFF3149A7
:108ED000032029F07FFE204604B0BDE8F0815EB19A
:108EE000F389A3F500739BB2F381F38903F4F05384
:108EF00013B930462FF064FC00222749404631F078
:108F0000B1FA32F036FA064620B1404609F084FE46
:108F10000446E0E741460220FFF7ECFE80B900245A
:108F2000002DD8D0EB89A3F500739BB2EB81EB89C0
:108F300003F4F053002BCED128462FF041FCCAE7B2
:108F4000482116482FF0F4FB04460028E7D00223FE
:108F5000014602AA3046CDE9025723F049FEE389D3
:108F6000A3F500739BB2E381E38903F4F05313B9D3
:108F700020462FF025FC0A4B1C68002CD0D0E3893A
:108F800003F500739BB2E381CAE700BF6D190600C9
:108F9000241C0600CD1906008F19060041C30200EB
:108FA00058D5002070B504460E460020184927F019
:108FB000EBF8054610B90025284670BD2246154934
:108FC00031F0F6F92846FEF70BF8EB89A3F50073AC
:108FD0009BB2EB81EB8903F4F053044613B92846A6
:108FE0002FF0EEFB002CE6D031462046FFF758FF6D
:108FF000E389A3F500739BB2E381E38903F4F053A3
:109000000546002BD8D120462FF0DAFBD4E700BF6D
:10901000071E0600241C060070B5064650B12EF04F
:109020009DFE044630B932464049032029F0D2FD66
:10903000204670BD00223E49304631F013FA044606
:109040002EF084FE98B95CB1E389A3F500739BB25E
:10905000E381E38903F4F05313B920462FF0B0FB0A
:1090600022463449032029F0B5FD0024E0E75CB135
:10907000E389A3F500739BB2E381E38903F4F05322
:1090800013B920462FF09CFB00222B49304631F0CB
:10909000E9F932F00DFF02460B4604460D4637F063
:1090A000DFFF30B9002200232046294637F0BAFFFF
:1090B00008B1224D00242B462246214823F076FD9C
:1090C000054601460120FFF715FE60B308211D4843
:1090D0002FF02EFB044670B13146FEF7BBFCE3894E
:1090E000A3F500739BB2E381E38903F4F05313B952
:1090F00020462FF065FB144B1C6824B1E38903F56F
:1091000000739BB2E381002D92D0EB89A3F500732D
:109110009BB2EB81EB8903F4F053002B88D12846F6
:109120002FF04EFB84E70446EDE700BFB11B0600BD
:10913000E61B0600441D0600B91A060000409F40C9
:1091400051BF0200ADC4020058D5002030B515460D
:1091500091B0002231F086F90446C0B16946402240
:1091600032F03CFB0C49684638F01CFA88B168467E
:109170001EF086FC2860E389A3F500739BB2E381AF
:10918000E38903F4F05313B920462FF019FB11B013
:1091900030BD0248EEE700BFC61806007F000001A0
:1091A0002DE9F04FB64B1B78B5B0022B0D460C9253
:1091B0004FF0000407D00120B24929F00BFD2046F2
:1091C00035B0BDE8F08F17A81EF094FC0028F7D04A
:1091D00011A81BF02FFA9DF845209DF84430134349
:1091E0009DF8462013439DF8472013439DF84820DF
:1091F00013439DF8492013430AD108238DF84530C5
:109200004FF4EE73ADF8463040F20233ADF848301B
:1092100028462EF0A3FD0746002855D00DF14A023E
:1092200099492846FFF792FF0DF14E0297492846CB
:10923000FFF78CFF0DF1520295492846FFF786FF94
:109240000DF1560293492846FFF780FF002292490C
:10925000284631F007F90646D8B1402224A932F059
:10926000BDFA002424AF254617F8018BB8F1000F92
:1092700014D134AB1C4404F88C5CF389A3F500735F
:109280009BB2F381F38903F4F05313B930462FF006
:1092900097FA01238DF85A30002459E040462AF00D
:1092A0003DF90F2804D800EB051523461C46DBE7E3
:1092B000B8F13A0FE1D134AA631C1444052B04F829
:1092C0008C5CDADC0025F1E71BF046FC734B744A3A
:1092D0001A600646062211A909201AF061FB042231
:1092E00010A90F2010971AF05BFB042210A901208F
:1092F0001AF056FB042210A905201AF051FB3B4638
:109300004422022130461BF0D9F8664D11A930469F
:109310001BF018FB01232B70634B1F7018F0F2FB3E
:10932000624B10F5200041F10001C3E90001604BE0
:109330001F7095F90030032BAED05B4B1B78012BCF
:109340002ED15C485C4C23F0DFFC5B4829F096FF93
:1093500011A81BF099F917A81EF0B2FB0C982EF07B
:1093600015FDC8B1002C00F0F481204630F094FBCC
:1093700024900123002024AA0C9923F039FC24987E
:1093800050B1C389A3F500739BB2C381C38903F4B1
:10939000F0530BB92FF014FAB4FA84F040090FE738
:1093A00028F092FF07460028CBD130461AF088FB00
:1093B0000246002800F02A810DF13E0300933F4948
:1093C00024AB30461AF0D6FDBDF83E303B4A432B65
:1093D00040F0B08002F11C0111AC3B4611F801CB0A
:1093E00014F8017BBC4540F00F8101339BB2062B82
:1093F000F4D1138AADF84A30538AADF84C3080B2BC
:109400002F4BF03803440D932E4B1A7807925A785D
:109410000A9293F803C09A782B4B03925A780B92D6
:109420000022DF7898781B780593CDE90822244B39
:109430000692049214460D9999420AD8049B002B77
:1094400065D0214B0B9959700599DF709870197090
:109450005DE093F800E0BEF1060F00F0AA8035D879
:10946000BEF1010F7AD0BEF1000F6FD0BEF1030F35
:1094700000F0838003F102085B78984468E000BF45
:1094800094D50020C21F0600A23D0600E01F060082
:10949000E71F0600EF1F0600F31F060010D3002091
:1094A0007856341268D5002014D3002098D50020B7
:1094B000AAD50020F71F0600B61F060018D300200B
:1094C00008D400200AD3002084D50020BEF1350F37
:1094D00040D00DD8BEF1330FCCD119799F78D87810
:1094E0000B9103F106085B790593012304932FE0A8
:1094F000BEF1360F79D0BEF1FF0FBBD1049B33B163
:10950000994B98700B9858700598DF701870099BEC
:1095100013B1964B07991970089B13B1934B0A9995
:109520005970069B13B1914B0399997012B18F4BEF
:1095300083F803C095F90030013B032B3FF6F9AEE9
:10954000DFE813F066007700A300E40003F10108F0
:10955000434670E703F103089C78F9E703F1020E34
:109560000DF14E0803F106091EF801AB08F801AB36
:10957000CE45F9D103F10608EAE793F801E003F1DB
:1095800002080DF1520903F1060A18F801BB09F8A7
:1095900001BBD045F9D14FF000090633AEF1040EFE
:1095A0001FFA89FAF24503EB090809F10109F7DB13
:1095B000CEE793F801E003F102080DF1560903F13B
:1095C000060A18F801BB09F801BBD045F9D14FF0E4
:1095D00000090633AEF1040E1FFA89FAF24503EBD7
:1095E000090809F10109F7DBB2E79A780792DA78FE
:1095F0000A921A790392012203F1060893F805C032
:109600000692CDE90822A3E7002493E7044691E7F8
:10961000022C40F09980564823F076FB4FF0FF3340
:10962000249324AA11AB534930461BF08DF82C70BB
:109630007FE6052C16D1504823F066FB1BF04EF850
:1096400011A81BF021F818F05DFA4C4B10F5200022
:1096500041F10001C3E90001494B00221A700323C4
:109660002B7066E6062C6FD1464823F04DFB18F0B0
:1096700049FA424B10F5200041F10001C3E9000115
:109680003F4B00221A700123EAE7374B1F687B1C0F
:109690003FF44FAE18F036FA7A08002382428B412D
:1096A000BFF647AE384823F02FFB384B9DF84A20D1
:1096B0001A709DF84B205A709DF84C209A709DF8B6
:1096C0004D20DA70294B1A788DF890205A788DF851
:1096D00091209A788DF892202D4ADB788DF893307E
:1096E0001368013313600DF14A0111AB24AA30460F
:1096F0001BF02AF804232B7018F004FA1F4B10F506
:10970000200041F10001C3E9000112E6052C19D146
:109710001B4A1E49002313700DF14A0211F8017B08
:1097200012F8010B874218D101339BB2042BF5D1FB
:1097300018F0E8F9114B10F5200041F10001C3E9E0
:1097400000018CE7062C92D011A930461BF09AF943
:10975000EFE502202EF08CFF0AE61AF0BFFF11A8F9
:109760001AF092FFE4E700BF84D500200AD300205E
:109770001420060006D300202B20060098D50020D8
:10978000AAD5002040200600562006003CD5002027
:1097900010D300202DE9F041364B1F78022F98B0EE
:1097A000884608D03449012029F014FA00242046C4
:1097B00018B0BDE8F0810BA81EF09CF9002857D026
:1097C00005A81AF037FF04F0AFF90A252E26044643
:1097D00004230DF11A022949CDE900561EF0B5FA0D
:1097E00004230DF11E0226492046CDE900561EF045
:1097F000ACFA04230DF1220222492046CDE900569D
:109800001EF0A3FA04230DF126021F492046CDE9DC
:1098100000561EF09AFA10233A22CDE900321B4975
:10982000062305AA20461EF090FA0BA81EF048F960
:1098300040462EF0ABFA0028B9D038462EF018FF7B
:109840003B46CDE9030403AA0020414623F0D0F9AA
:1098500003980028ABD0C389A3F500739BB2C381E2
:10986000C38903F4F053002BA1D12EF0A9FF9EE78A
:1098700004469CE794D50020C21F0600A23D0600C6
:10988000E01F0600E71F0600EF1F0600F31F06009B
:1098900010B58EB00446032101A81EF0D1F901A82D
:1098A0001EF022F901A81EF00BF9084B0849586870
:1098B000224630F07DFD074B02221A70E38903F542
:1098C00000739BB22046E3810EB010BD8C2E0020A9
:1098D0005524060094D50020024B1B68002198797E
:1098E00024F0A4B990D50020024B1B68012198797F
:1098F00024F09CB990D50020F0B50E4693B00446F4
:1099000058B123F025FA132805460DD022465749B1
:10991000012029F05FF9002403E05549012029F0D6
:1099200059F9204613B0F0BD022105A81EF088F9B0
:1099300005A88DF819508DF81A601EF0D5F84D491C
:10994000002026F021FC002104469DF81A0023F097
:109950000BFA01219DF81A0024F068F9464B474A9A
:109960001A61474A5A611A88920500D4FEE7454AAF
:109970009A61454ADA61454B01AA03F11007154681
:1099800018685968164603C60833BB423246F7D1F9
:109990001AF0A4FE9DF804305AB2102A5EDC9DF83D
:1099A00005201344DBB25AB2102A57DC9DF806207A
:1099B0001344DBB25AB2102A50DC9DF8072013443E
:1099C0005BB2102B4ADC2E46032700251B201AF021
:1099D00013F816F8013B07FA05F1AB4020EA010144
:1099E0001943C9B21B2002351AF0AAF8082DEDD18F
:1099F0009DF808305AB2102A30DC9DF80920134433
:109A0000DBB25AB2102A29DC9DF80A201344DBB2DB
:109A10005AB2102A22DC9DF80B2013445BB2102BA3
:109A20001CDC0DF10706002503271A2019F0E4FFBE
:109A300007FA05F120EA010116F8010FA8400143D9
:109A4000C9B21A2002351AF07BF8082DEDD105A80D
:109A50001EF036F80E4B02221A7062E70D4824F011
:109A600063FA05A81EF02CF855E700BFC2250600D2
:109A7000DF25060017260600B82C0020D998020022
:109A8000E9980200C19A0200C79A0200B6180600BF
:109A900094D500202026060010B5084C2368014606
:109AA000587917F091FE002805DA23684FF0FF314E
:109AB000587917F089FEC0B210BD00BF90D50020C4
:109AC000FF20FFF7E9BFFFF7E7BF1BF02BBA1BF042
:109AD0003DB9000038B5054609B11BF0C5F90022B3
:109AE0001249284630F0BEFC31F043FC10B110485A
:109AF0002FF0D2FF0446014628461BF0B5F95CB1B1
:109B0000E389A3F500739BB2E381E38903F4F05387
:109B100013B920462EF054FE01202EF020FE0549F8
:109B200002462846BDE8384030F063BC9D17060069
:109B30006CB40600C122060008B51BF095F90020A0
:109B400008BD000070B58EB0044601A80E4615464B
:109B50001EF05CF8D8B1204600220E4930F082FC9D
:109B60000446A0B132460C4930F022FC2A460B498B
:109B7000204630F01DFCE389A3F500739BB2E3811E
:109B8000E38903F4F05313B920462EF019FE0EB00A
:109B900070BD00BF971F06009B1F0600AA1F06008E
:109BA00010B58EB0044601A81EF030F830B101A8FF
:109BB00021461BF0CDFB01A81DF082FF0EB010BDA9
:109BC00038B5054630F0AAF904462EF0DFF8A0B902
:109BD0002146184829F072FB14B90024204638BDEC
:109BE000E389A3F500739BB2E381E38913F4F05595
:109BF000F3D120462EF0E4FDEFE75CB1E389A3F555
:109C000000739BB2E381E38903F4F05313B9204658
:109C10002EF0D6FD0849002026F0B6FA04460028AA
:109C2000DCD001211DF0A0FD2A460449204630F079
:109C3000BFFBD3E7C5220600EC220600F422060093
:109C400038B5054630F06AF904462EF09FF8A0B901
:109C50002146184829F032FB14B90024204638BDAB
:109C6000E389A3F500739BB2E381E38913F4F05514
:109C7000F3D120462EF0A4FDEFE75CB1E389A3F514
:109C800000739BB2E381E38903F4F05313B92046D8
:109C90002EF096FD0849002026F076FA04460028AA
:109CA000DCD000211DF060FD2A460449204630F03A
:109CB0007FFBD3E7C522060066190600F4220600E2
:109CC00030B591B0044603A80D461DF09FFF48B182
:109CD000002303A800932A4621461BF0D3F903A8CA
:109CE0001DF0EEFE002011B030BD30B58FB004463F
:109CF00001A80D461DF08AFF58B11DB12946204626
:109D0000FFF7DEFF01A821461BF022FB01A81DF092
:109D1000D7FE0FB030BD000030B58FB0054601A8AA
:109D20001DF074FF78B300211A481DF017FE044699
:109D300030B3294601A81DF0D9FD2946012220464D
:109D400033F089FB054600B30146204631F0BEF9E9
:109D5000EB89A3F500739BB2EB81EB8903F4F0531D
:109D600013B928462EF02CFDE389A3F500739BB2AE
:109D7000E381E38903F4F05313B920462EF020FD6C
:109D800001A81DF09DFE0FB030BD034829F076FA02
:109D9000EAE700BF11240600172406002DE9F0436E
:109DA00091B0814603A8884616461F461DF02EFF37
:109DB000B8B10021189830F0D9F804462EF00AF80E
:109DC00080B3304630F0E2F80646384630F0DEF830
:109DD00007461B202EF04CFC054628B903A81DF0B1
:109DE0006FFE11B0BDE8F0833B46324641462FF08E
:109DF0006CF90121189830F0B9F82646074630462C
:109E000030F0C4F880B200903B462A46494603A889
:109E10001BF038F94545E1D03A46314628462FF047
:109E200075FFDBE70CB94546E9E7E389A3F5007365
:109E30009BB2E381E38903F4F053002BF3D1204676
:109E40002EF0BEFCEFE700002DE9F04F8BB082460C
:109E500001912EF09CF820B9002630460BB0BDE8E9
:109E6000F08F03F061FE06460028F5D04FF00009A0
:109E70004FF0FF350022514605A82DF0D5FFCB4607
:109E80002C46A8462F464A464946DDE9053083421E
:109E9000C0F0D780089850B1C289A2F5007292B282
:109EA000C281C28902F4F0520AB92EF089FCB4F1E1
:109EB000FF3F08BF5C46B8F1FF3F08BFA046002F38
:109EC00009DD7A1E002150462FF042F9B8490246BA
:109ED000304630F08EFAB7482FF0DEFDB649024624
:109EE000304630F086FA791CA8EB010250462FF07C
:109EF0002FF9B2490246304630F07BFA6FF000424B
:109F0000214650462FF024F907462FF04CFA18B995
:109F1000AB4938462FF0A5F93A46AA49304630F009
:109F200068FA691C14BF2A1B6FF000422146504694
:109F30002FF00EF904462FF036FA18B9A049204642
:109F40002FF08FF92246A049304630F052FA6A1CB1
:109F500000F0B9806FF00042294650462FF0F8F823
:109F600002469A49304630F044FA09F1FF324FF682
:109F7000FE739A4240F2AB8002202EF079FB02463B
:109F80009349304630F035FA6B1C00F0A4806FF036
:109F90000042691C50462FF0DBF8019B0446002B61
:109FA00049D02DF0A1FE0546002844D102462146A5
:109FB00005A82DF039FF03F0B7FD81461B202EF0D8
:109FC00057FB07461B202EF053FB8046DDE9053288
:109FD0009342C0F08480089850B1C389A3F5007300
:109FE0009BB2C381C38903F4F0530BB92EF0E8FB95
:109FF0005CB1E389A3F500739BB2E381E38903F4C9
:10A00000F05313B920462EF0DBFB38462FF0CBF986
:10A01000002800F09780384632F09FF94146074605
:10A020002FF0C8FB3946484630F026F841463846FE
:10A030002FF098FE4C4622466649304630F0D9F95A
:10A040000BE7099888B1C05C2F2812D1B4F1FF3F0B
:10A0500008BF5C46012A01F1010106D1022904D1A1
:10A060007B1C02D13D463C465F46B8F1FF3F0DD117
:10A0700019E03A2807D17B1C02F10102F5D0631CDC
:10A08000F3D1D8460FE0B8F1FF3F16D0D84514DA27
:10A09000631C40F089802F2805D9392803D830382F
:10A0A0000A2303FB090905A8CDE902210BF1010BE5
:10A0B0002DF0B0FCDDE90221E7E63F28F3D1601C7A
:10A0C000F1D05D46EFE702202EF0D2FA48E748468D
:10A0D0002EF04DFB53E702202EF0CAFA5DE70998F7
:10A0E00000284CD0C05C262825D138462FF05BF9DB
:10A0F000C0B1384632F031F9414605462FF05AFBDF
:10A10000294648462FF0B8FF414628462FF02AFE40
:10A110001B202EF0ADFA07461B202EF0A9FA804630
:10A12000002504E040462FF03EF90028E1D105A8C3
:10A130002DF070FC4AE765B93D282AD1019DF6E76C
:10A14000824611E040462FF02EF900287FF463AFDD
:10A150006CE7252814D105A82DF05CFC099800288F
:10A16000EED0059B10F803A005A82DF053FC09992B
:10A1700009B1059BC95C504629F0E5F9C0B255B15B
:10A180008DF8130001220DF1130140462FF046F81F
:10A19000D4E72528DFD08DF8130001220DF113013B
:10A1A00038462FF03BF8BBE73F288AD07BE700BF5B
:10A1B0008E250600972506009B250600CB18060075
:10A1C00091240600A2250600A7250600B02506005A
:10A1D000B7250600BC25060070B590B004460D46B4
:10A1E0000146684616461EF005F978B13246294602
:10A1F00068461DF0F7FE68461EF0C2F8E38903F5D5
:10A2000000739BB2E381204610B070BD0446FAE7AC
:10A2100030B591B00D46014668461EF0EBF80028B7
:10A220004CD0BDF92320BDF927309A4244DC03F01D
:10A230007BFC044618B3BDF923002EF098FA2049A0
:10A240000246204630F0D5F8BDF925002EF08FFAF1
:10A250001C490246204630F0CCF8BDF927002EF00C
:10A2600086FA19490246204630F0C3F8BDF92900A4
:10A270002EF07DFA15490246204630F0BAF8C5B1F5
:10A2800000226FF07F038DF827208DF828308DF89D
:10A2900029208DF82A304FF0FF327F2368468DF851
:10A2A00023208DF824308DF825208DF826301EF0DF
:10A2B00067F8204611B030BD0024E0E70446F8E717
:10A2C000EB210600EE210600F1210600F421060034
:10A2D00070B590B004460D460146684616461EF01D
:10A2E00089F850B3BDF80530022D23F070039BB2FE
:10A2F0001DD0032D1ED0012D08BF43F03003ADF853
:10A3000005304EB1BDF80530DA064CBF83F040038E
:10A3100083F02003ADF8053068461EF031F8E3897C
:10A3200003F500739BB2E381204610B070BD43F08B
:10A330006003E4E743F05003E1E70446F4E770B557
:10A3400090B004460E460146684615461EF052F887
:10A3500070B16846ADF81660ADF818501EF010F8F0
:10A36000E38903F500739BB2E381204610B070BD12
:10A370000446FAE700B591B0014668461EF03AF887
:10A3800010B16846FCF79CFD11B05DF804FB0000BD
:10A3900000B591B0014668461EF02CF838B1BDF802
:10A3A000141011F4604305D10A482EF0E1FE11B0FB
:10A3B0005DF804FBB3F5005F03D107482FF06CFB99
:10A3C000F5E7B3F5C04F01D10448F7E708462EF092
:10A3D000CEF9ECE7C3210600CC210600D02106000F
:10A3E000F0B591B004460E460146684615461F4634
:10A3F0001EF000F800B3012E9DF81A10A8BF012628
:10A40000012DA8BF012546EAE67666F3010145EA7B
:10A41000E57565F3830187F3020767F30511684665
:10A420008DF81A101DF0ACFFE38903F500739BB2A1
:10A43000E381204611B0F0BD0446FAE72DE9F04370
:10A4400091B0044689460146684617461E46DDF827
:10A4500060801DF0CFFF002847D048462DF097FDC3
:10A4600040B92349012028F0B5FB0024204611B053
:10A47000BDE8F083FF2F01D91E49F3E730462DF0E8
:10A4800086FD28B930462DF052FE08B91A49E9E791
:10A490004A461A4920462FF08BFF3246184920467B
:10A4A0002FF086FF5FFA88F02EF061F91549024619
:10A4B00020462FF09EFF38462EF059F94FEA282506
:10A4C0000246114920462FF094FF012DB8BF012507
:10A4D00005F5C0456846ADF814501DF051FFE389FD
:10A4E00003F500739BB2E381C0E70446BEE700BFFB
:10A4F0001722060034220600512206007B220600A5
:10A5000080220600D721060085220600F0B591B012
:10A5100004460F460146684616461D461DF06AFF72
:10A5200098B1169BADF821306846ADF81B70ADF8B8
:10A530001D60ADF81F501DF023FFE38903F5007384
:10A540009BB2E381204611B0F0BD0446FAE700005B
:10A550002DE9F04F97B00E46014606A890461F46DB
:10A560001DF048FF002853D030462DF010FD002884
:10A5700051D00023092203A93046CDE903338DF8D9
:10A58000143031F02BF99DF80E109DF80D0028F0D5
:10A59000DAFF36F061FA00227F4B36F0C7FA044644
:10A5A0000D469DF80F009DF8101028F0CCFF36F0F6
:10A5B00053FA0022784B36F0B9FA002282468B46D5
:10A5C00000232046294636F023FDE0B9002200236F
:10A5D0005046594636F01CFDA8B99DF812109DF85A
:10A5E000110028F0B0FF36F037FA00226A4B36F03F
:10A5F0009DFA00220023CDE9000136F009FD10B9D3
:10A600009DF81330B3B10120644928F0E3FA00202B
:10A6100017B0BDE8F08F304631F074F9404655EC84
:10A62000104B31F06FF938465BEC10AB31F06AF942
:10A630008DED000B25F000494FF0FF32584B2046BE
:10A64000494636F00DFD002840F0A1804FF0FF3262
:10A65000534B2046494636F0F9FC002840F09780DD
:10A660002BF000494FF0FF324D4B5046494636F033
:10A67000F7FC002840F08B804FF0FF32484B5046EB
:10A68000494636F0E3FC002840F08180DDE9008394
:10A6900023F000494FF0FF32414B4046494636F027
:10A6A000DFFC002873D14FF0FF323D4B4046494656
:10A6B00036F0CCFC00286AD100223A4B20462946CD
:10A6C00036F034FA36F0E2FC0022364B04465946A6
:10A6D000504636F02BFA36F0D9FC0022314B0546B5
:10A6E000DDE9000136F022FA36F0D0FCBDF81D108D
:10A6F00011F4607184F3080385F3080280F3080005
:10A7000008D0B1F5C07F19D010D880291AD0B1F582
:10A71000807F1CD09DF8231010291FD19110DA10D2
:10A72000D20242EA411242EAE00071E7B1F5007F4D
:10A7300011D0B1F5207FEDD1114601E01946134645
:10A74000024606E01946034610460A46E2E7194665
:10A7500003460846DEE719461346F6E7202906D1E8
:10A760001B0443EA0223034343F07F4050E71829C8
:10A7700004D11B0443EA0223184349E7134403446A
:10A78000B3F5C07F4FF0FF30B8BF002040E7304640
:10A790002FF0FCFB3CE700BF0000703F8A22060060
:10A7A000FFFFEF7F000070402DE9F04F99B00D469C
:10A7B00091462DF0C7FF0446002800F0A180002D2F
:10A7C00000F09E802B68062B40F09A8029460122DB
:10A7D0000DA829F0E8FA0DA829F089F903900DA831
:10A7E00029F0B3FA0DA829F082F907460DA829F03F
:10A7F000ACFA0DA829F07BF90A900DA829F0A5FA6A
:10A800000DA829F074F90B900DA829F09EFA0DA857
:10A8100029F06DF906460DA829F097FA0DA829F040
:10A8200066F905460DA828F084FF48462DF096FAF3
:10A8300030B10022804948462FF014FE30F032FC3F
:10A84000039B8046981B0028A7EB0503B8BF404236
:10A85000002BB8BF5B429842A8BF18460523B0FB47
:10A86000F3F036F0F9F802460B460020734936F053
:10A8700087FA0022714BCDE9000136F0DDFB00289C
:10A8800042D169A3D3E90023DDE9000136F0C0FB22
:10A8900018B19FED657B8DED007BB8F1000F0ADDEF
:10A8A000404636F0D9F802460B460020634936F0A0
:10A8B00067FACDE9000103982DF059FF01462046C3
:10A8C0002FF0AAFC38462DF052FF014620462FF00B
:10A8D000A3FCDDE900AB0022584B5046594636F048
:10A8E000A1FBA0B930462DF042FF014620462FF0D3
:10A8F00093FC28462DF03BFF014620462FF08CFCB0
:10A90000204619B0BDE8F08F9FED497BC3E7524662
:10A910005B465046594636F009F95246CDE90401E6
:10A920005B460020454935F049FF02460B4680460C
:10A93000894636F0FBF84246CDE906014B464046D3
:10A94000494635F03DFF52465B4636F0EFF8CDE91B
:10A950000801039836F080F8DDE9062336F0E6F8C2
:10A9600080460A98894636F077F8DDE9082336F004
:10A97000DDF802460B464046494635F021FF804649
:10A980003046894636F068F8DDE9042336F0CEF823
:10A9900002460B464046494635F012FF0022284B3E
:10A9A00035F00EFF36F072FB2DF0E1FE0146204639
:10A9B0002FF032FC384636F04FF8DDE9062336F04A
:10A9C000B5F880460B98894636F046F8DDE908234D
:10A9D00036F0ACF802460B464046494635F0F0FEEC
:10A9E00080462846894636F037F8DDE9042336F0FC
:10A9F0009DF802460B464046494635F0E1FE0022EE
:10AA00000F4B35F0DDFE36F041FB2DF0B0FE014678
:10AA100020462FF001FC50465946DDE9002335F071
:10AA2000CFFE82468B4656E79A9999999999B93FF4
:10AA30001F85EB51B81ED53FF72106000000F03FFF
:10AA40000000E03F2DE9F04F95B0014604A81DF04D
:10AA5000D1FC28B94FF0000B584615B0BDE8F08F77
:10AA60009DF81B90B9F1010F07D0B9F1180F04D070
:10AA70004949012028F0AEF8ECE7BDF81530BDF8E3
:10AA80001960BDF81770DB0642BF33463E461F46CD
:10AA900007FB09F51F35B9F1010F4FEA65150CBF2A
:10AAA0004FF020084FF01A08AD0005FB068A50460B
:10AAB0002DF058FD83460028CCD02DF0ADF942236F
:10AAC00003704D2343700C2383733B1280F802A064
:10AAD000C3744FEA2A2A331280F80A8080F803A050
:10AAE00043750123B9F1010F83759DF81B3003767F
:10AAF00001BFFF238376C3760377731E04468774F2
:10AB0000067505FB03884FF00009B145A4D009F193
:10AB1000010300939DF81B30012B37D04FF0000A42
:10AB2000BA452ED04A46514604A81DF0FFFB9DF8B9
:10AB30001B30DB080AFB0383020AE0542344000CA9
:10AB40005A7098700AF1010AEAE700235B00039348
:10AB50004A464B1C04A801931DF0E8FB0199039B96
:10AB600000F00100514543EA0003EFD1029A02EBE5
:10AB7000EA020AF1080A02F8013CAAF10801B94206
:10AB8000E3DBA8EB0508DDF80090BEE704EB080363
:10AB90004FF0080A0293F0E76E20060038B5FFF781
:10ABA00051FF054610B90025284638BD0BF086FE3A
:10ABB000EB89A3F500739BB2EB81EB8903F4F053AF
:10ABC000044613B928462DF0FBFD002CEBD021469E
:10ABD00008482EF0CDFAE389A3F500739BB2E38118
:10ABE000E38903F4F0530546002BDDD120462DF018
:10ABF000E7FDD9E7AD20060010B5FFF7CFFF04460B
:10AC000068B123F01DFFE389A3F500739BB2E381D4
:10AC1000E38903F4F05313B920462DF0D1FD024827
:10AC2000BDE8104023F080B96BB4060030B591B098
:10AC30000C460146684615461DF0DCFB20B12A464D
:10AC4000214668461DF072FB11B030BD2DE9F04F72
:10AC500099B00546014608A81DF0CCFB28B94FF075
:10AC60000009484619B0BDE8F08F02F05DFF0446C8
:10AC70000028F4D00021284605F0C2FF0121074634
:10AC8000284605F0BDFF054638469DF82B602DF09F
:10AC90006EFD3C49024620462FF0ABFB28462DF0C6
:10ACA00066FD3949024620462FF0A3FB012E07D04E
:10ACB00030462DF05CFD3549024620462FF099FBC9
:10ACC00005FB07F0704307300021C0102EF07EFE18
:10ACD000814668B9E389A3F500739BB2E381E389F8
:10ACE00003F4F053002BBAD120462DF069FDB8E7EC
:10ACF0000146002203A82DF097F80025A846AB4690
:10AD0000AA46DDE90312914213D3069850B1C389D4
:10AD1000A3F500739BB2C381C38903F4F0530BB94D
:10AD20002DF04EFD4A461A4920462FF062FBA146FF
:10AD300097E75A46514608A81DF0F8FA0AF1010AA9
:10AD400008FA06F8574548EA000806EB050203DC56
:10AD50000BF1010B4FF0000A15460AE0083D28FAF6
:10AD600005F1C9B203A801922CF09AFE019A4FEAAC
:10AD70001828072DF2D8D5086FF0070303FB052527
:10AD8000BFE700BF9C200600A2200600A920060005
:10AD9000CF450600F0B591B004460E460146684620
:10ADA00015461F461DF026FBE8B1A7B9039B2A46AE
:10ADB000314668461DF0D5FA6846ADF81660ADF824
:10ADC00018501DF0DDFAE38903F500739BB2E381AF
:10ADD000204611B0F0BD00231A4639462046FFF741
:10ADE000B7FB0346E3E70446F2E70000000000007B
:10ADF0002DE9F04FB3B082460E46014622A80C92D0
:10AE000014933C9D1DF0F6FA28B94FF0000A504605
:10AE100033B0BDE8F08F30462CF0A0FF002800F0E2
:10AE200097800022934930462FF01CFB30F03AF90E
:10AE300000229149039030462FF014FB30F032F994
:10AE400000228E49099030462FF00CFB30F02AF991
:10AE50000128B8BF012000228949044630462FF05E
:10AE600001FB804630F01EF9002207468549304636
:10AE70002FF0F8FA814600283ED02CF04BFF50B35B
:10AE8000B9F80430022B26D100231DA948461D9392
:10AE90002EF0E6FAB9F80E30A3F500739BB2A9F8CC
:10AEA0000E30B9F80E3003F4F053834613B9484618
:10AEB0002DF086FC1D9B102B08D8734ADA40D00772
:10AEC00004D5013B0793BBF1000F17D16F49012057
:10AED00027F080FE99E7B9F80E30A3F500739BB216
:10AEE000A9F80E30B9F80E3003F4F053002BEDD171
:10AEF00048462DF065FCE9E707908346304600227E
:10AF000063492FF0AFFAB8F1000F14BF3B464FF082
:10AF1000FF3306460F93BBF1000F67D1CDF820B089
:10AF2000012C66D1269BADF86C30259BADF86E30B8
:10AF300007940DF16C0B30462CF0ECFE00285BD032
:10AF4000039B002B5EDC5349012027F043FE1CE0ED
:10AF500030462DF01CF848B130462CF0DBFE60B9CD
:10AF6000F38903F500739BB2F3810AE030462CF0BD
:10AF7000D1FE0028F0D14849A9E730462DF0D8FF8E
:10AF8000064630462DF003F880B9002E3FF43DAF61
:10AF9000F389A3F500739BB2F381F38913F4F05A9C
:10AFA0007FF433AF30462DF00BFC30E70021304604
:10AFB0002EF06AF80121074630462EF065F802218E
:10AFC000834630462EF060F8010640F1488200F0DA
:10AFD0007F04032130462EF057F804230F90089386
:10AFE00000230397CDF824B0079399E70023089333
:10AFF000A1E74FF0000B9EE730462CF0C8FF002879
:10B000009ED1A0E7099B002B9DDD202C9BDC01231A
:10B01000A340013B072C1693D6BF08230023B3FBA4
:10B02000F4F33046D8BF03F1FF3315932DF080FFC2
:10B0300006905EB1F389A3F500739BB2F381F389A7
:10B0400003F4F05313B930462DF0BAFB0DF1740937
:10B05000089A069948462CF0E7FE002D6ED1149F01
:10B06000099B3B4400932E46DDF83080039B43440C
:10B0700004931DE09C200600A2200600A9200600E3
:10B08000C6200600D220060014000100DA200600C7
:10B09000CF45060058210600232106002B02219DE2
:10B0A0000DB11D9AAD5C48461D432CF0B3FC08362B
:10B0B000A642F3DB169A361B25FA06F313400F9AC5
:10B0C00093420BD0BBF1000F03D0079A13403BF81B
:10B0D00013303A46414622A81DF043F9049B08F17B
:10B0E00001084345E4D1009B0137BB42BCD1209805
:10B0F00050B1C389A3F500739BB2C381C38903F424
:10B10000F0530BB92DF05CFB069B63B1DB89069A0B
:10B11000A3F500739BB2D381D38903F4F05313B921
:10B1200010462DF04DFB22A81DF02AF9BAF80E307A
:10B1300003F500739BB2AAF80E3068E628462CF09F
:10B140000DFE0028D3D0039BAB4963430733DB10CC
:10B150000022284617932FF085F930F0A9FECDE99B
:10B160000001DDE9006323F000474FF0FF32A34BFD
:10B170003046394635F074FF70B94FF0FF329F4BBF
:10B180003046394635F062FF30B900220023DDE950
:10B19000000135F047FF18B19FED957B8DED007BE9
:10B1A0000022974928462FF05DF930F081FE21F00A
:10B1B00000430593049006460F464FF0FF328F4B35
:10B1C000DDE9040135F04CFF38B94FF0FF328B4B0D
:10B1D000DDE9040135F03AFF08B100260027039BA2
:10B1E000DD01099B47EC106BDB01189333F014FB76
:10B1F00059EC108B47EC106B33F0FEFBDDE90023BC
:10B200004046494657EC106B35F0BAFD00227D4BA5
:10B2100035F08CFC00227C4B35F0D2FA35F036FF4D
:10B22000DDE900230D903946304635F0A9FD0022B6
:10B23000744B35F07BFC0022734B35F0C1FA35F0CE
:10B2400025FF0E90039835F007FC29F00043CDE967
:10B2500010010998CDF828800B9335F0FDFBDDE94E
:10B260000A23CDE91201DDE9100135F05FFCB0469B
:10B2700027F0004906460F4642464B46DDE91201DB
:10B2800035F054FC02460B463046394635F098FA04
:10B29000DDE9002335F04AFC00225B4B35F090FAE3
:10B2A00035F0F4FE42464B460746DDE9100135F025
:10B2B0003DFCDDE9122380468946DDE90A0135F0CF
:10B2C00035FC02460B464046494635F079FADDE941
:10B2D000002335F02BFC00224B4B35F071FA35F092
:10B2E000D5FE4FF0FF320646444BDDE9040135F050
:10B2F000B7FE98B94FF0FF32404BDDE9040135F05D
:10B30000A5FE58B90C9A07EBD773A2EB6303149A06
:10B310000C9306EBD673A2EB630314930D9B0E9A6A
:10B320007B43013306FB023303EBD373A5EB6303CB
:10B330007F3304930D9B7343013307FB1233189A39
:10B3400003EBD373A2EB63037F3300934FF000084A
:10B35000B045BFF6CCAE009B0A93049B1093149BA0
:10B3600043444FF00009129334E0109B1A1227D483
:10B370000A9B1D1224D4039B934221DD099BAB42FF
:10B380001EDD082C42D1089B06991A44179B1DA864
:10B3900005FB03222CF066F9219B0BB11D9A9B5CE7
:10B3A0000F9A93420CD0BBF1000F03D0079A1340C1
:10B3B0003BF813300C99129A494422A81CF0D1FF93
:10B3C000109B0D9A134410930E9A0A9B9B1A09F135
:10B3D00001090A93B945C8DB049B0E9A13440493F0
:10B3E0000D9A009B134408F101080093B0E700BFD9
:10B3F000000000000000F03F82210600FFFFEF7F09
:10B4000088210600000070400000E03F039B069981
:10B4100005FB0325089B654303EBE5021DA82CF003
:10B4200021F9219B0BB11D9A9B5C0821A14207DBEE
:10B43000159A22EA05056543169AEB401340AFE7DB
:10B440001DA8CDE918312CF0E5FA189B219A19991D
:10B450001B020AB11D98125C13430831E6E703236F
:10B4600008934FF0FF3304460F93B9E5F0B5DDB014
:10B4700004460D4601460CA81CF0BCFF18B9002478
:10B4800020465DB0F0BD28462CF0ACFD0028F6D07B
:10B490002946012201A828F086FC1CAE002537466B
:10B4A00001A828F0A0F908B1802D16D101A828F034
:10B4B00040F9802D03D140210D4827F0DFFE3A46A8
:10B4C00069100CA81CF0E5FD0CA81CF059FFE389DD
:10B4D00003F500739BB2E381D2E701A828F007FBD4
:10B4E00026F8020B01A8013528F02FFCD8E700BF91
:10B4F0008F2106002DE9F0479EB004460D46014617
:10B500000EA892461CF076FF20B9002420461EB0FB
:10B51000BDE8F08728462CF065FD0028F5D0012213
:10B52000294603A828F03FFC002703A828F05BF970
:10B53000C0B903A828F0FDF8BAF1000F09D0CDF882
:10B5400000904346BDF95020BDF94E100EA81CF0E6
:10B5500078FE0EA81CF014FFE38903F500739BB27C
:10B56000E381D3E703A828F0C2FAFB0705460FD50D
:10B57000012F13D000903346BDF95020BDF94E1075
:10B580000EA81CF05EFEADF85050ADF84E6035468A
:10B5900003A8013728F0D9FB2E46C6E78146B046FE
:10B5A000F1E770B592B004460E46014602A8154672
:10B5B0001CF020FFB8B13346BDF92020BDF91E10A4
:10B5C000009502A81CF03DFE02A8ADF81E60ADF883
:10B5D00020501CF0D5FEE38903F500739BB2E38194
:10B5E000204612B070BD0446FAE7F0B593B00446A9
:10B5F0000D46014602A816461F461CF0FBFE90B100
:10B60000189B009332463B46294602A81CF019FEBF
:10B6100002A81CF0B5FEE38903F500739BB2E38139
:10B62000204613B0F0BD0446FAE700002DE9F04FC4
:10B6300099B007468846014608A81CF0DBFE0028A2
:10B640003FD0BDF8345005F46044B4F5C04FC5F3A5
:10B650000C0539D100223A4938462EF003FF00226A
:10B660003849064638462EF0FDFE2FF01BFD0746F2
:10B6700040462FF0D9FE00220146814603A82CF057
:10B68000D3FB4FF00008AB000093C2464FF0C00B55
:10B69000DDE903218A421AD3069850B1C289A2F586
:10B6A000007292B2C281C28902F4F0520AB92DF03E
:10B6B00087F8484631462EF055FBC2455046B8BF84
:10B6C000404619B0BDE8F08F00273E46D0E7079905
:10B6D00039B1895C0A2907D1D045B8BFD0464FF0AF
:10B6E000000A8CB922460AE074B92039CAB25E2A2F
:10B6F000F8D8154B13F811206A43B2FBFBF29244C1
:10B7000003A82CF087F9C3E7B4F5005F02D1009BD2
:10B710009A44F5E7B4F5C04FF2D1304601912CF0D0
:10B7200036FC48B10199B942EADBC91B30462DF01D
:10B73000ABFC00FB05AAE3E730462EF027FCF8E758
:10B740008022060085220600CC3A06002DE9F04F43
:10B75000B3B002AF0D4638651C46014697F8E83095
:10B76000BB6107F1800093461CF044FE002800F006
:10B770004A8207F18000FBF7A3FBB7F894303863E7
:10B7800003F46042B2F5C04FC3F30C033A647B6527
:10B790007FD10022AC49386D2EF064FE0022F862A1
:10B7A000AA49386D2EF05EFE0022B864A849386DB3
:10B7B0002EF058FE2FF076FCF86497F89A20B7F830
:10B7C0008530BB8202F0300110299BB266D183F034
:10B7D0003003B7F88710A7F885300BF10103A346B3
:10B7E000CC1A02F00302012A0DD82946386DFFF762
:10B7F0001DFF97F89A3003F0030303FB000000EBF2
:10B80000D070ABEB600B97F89A30C3F38103012B38
:10B810009FBF3A6B03FB022303EBD373A4EB6304D8
:10B82000B7F89B30BB63B7F89D30FB63B7F89F3028
:10B830007B63B7F8A1307B64B7F88530DB0607D5AA
:10B84000D7E90E32C7E90E237B6C7A6B7A647B638F
:10B8500028462FF0E9FD00223862014607F1580022
:10B860002CF0E2FA7B6D9B003B61DA46D7E91623A8
:10B870009A4280F0A180BB6E73B313F80290B9F1C5
:10B880000A0F2AD13B6B07F158001C442CF0C2F878
:10B89000EBE70023C7E91233FB628EE720290ED1C4
:10B8A00083F06003B7F88710A7F885300BF1010328
:10B8B000A1EB030BB7F8893001341C1B91E7302949
:10B8C0008FD183F05003B7F88910A7F88530631C37
:10B8D0005C46A1EB030B84E799463B6C002B40F0E0
:10B8E0009280A9F120095FFA89F35E2B98BF594A2B
:10B8F000B7F8948097BF12F819603E6C08FB06F603
:10B90000C02298BFB6FBF2F6BA6B921B52454DDAD5
:10B910007A6B92454ADAFA6BA2EB0802A24245DA48
:10B920007A6C944242DA5E2B40D800231D4699453A
:10B930005EDC484B484AC7F824D003EB490988B07D
:10B9400099F80130BB62002002AB15448146BA6A07
:10B95000914529DA2A7895F801C002F07F0208FBA8
:10B9600002F24FF0600E3032B2FBFEF2524423F886
:10B9700010200CF07F0203EB400108FB02F2303292
:10B980001CF0800FB2FBFEF222444A8000F102005C
:10B9900035D01A46411007F18000FB611CF079FB9D
:10B9A00026F092FCFB6950B3D7F824D0B24426F0BD
:10B9B0008BFC002800F01481786E002840F015817F
:10B9C000BA6CF96A386A2EF0A1F9BB8AA7F88530FB
:10B9D00007F180001CF0D4FC3B6D3A6DDB8903F568
:10B9E00000739BB2D381386DC437BD46BDE8F08F7C
:10B9F000184A02EB430201335278154497E709F1E4
:10BA000002090235A3E73B6CB3F5005F26D1BB6B9F
:10BA1000033B534514DC7B6B9A4511DAFB6B053B0A
:10BA2000A3420DDC7B6C9C420ADABB6901937B6DFF
:10BA3000009322464B46514607F180001CF0E8FD7A
:10BA40003B699A44B3E700BF7B22060080220600D0
:10BA500085220600CC3A0600B02606003B6CB3F502
:10BA6000C04FA4D1B86C2CF092FA002865D0FB6CC2
:10BA70004B4500F3B38007F16C050022B96C2846F2
:10BA80002CF0D2F9FB6C0026A9EB0309F86E3B6F92
:10BA9000F96F984203D27A6F02444A4544DB002989
:10BAA00049D00D5CB86F50B1C389A3F500739BB248
:10BAB000C381C38903F4F0530BB92CF081FEBB6B37
:10BAC0005B1B534544DA7B6B9A4541DAFB6B3A6B5F
:10BAD0009B1AA3423CDA7B6C9C4239DA134607F18D
:10BAE0006C087A6D93FBF2F35E43F208F96AFB612E
:10BAF00040462CF099F97B6DC7F804800AEB0309E6
:10BB0000002306F00706BB62BB6A9D4256DD7B6DD3
:10BB1000A9EB0303BB6009F1FF33FB607B6D04EB12
:10BB2000030800237B623FE001B1095C28460E4414
:10BB30002BF070FFAAE70D46B4E7B86C2EF026FA9A
:10BB4000FB6CA9EB03064B45054600FB06F6B6DD8C
:10BB50007B6D05FB03AA2AE7FB6F0BB1FA6E9B5CBA
:10BB6000BA69B34003F0800302B98BB1D7E923105F
:10BB700008F1FF32002B08BF0146CDE900217A6DA4
:10BB8000FB68B968A8EB020207F180001CF0B6FB65
:10BB90000136082E03D178682BF03CFF00267B6A23
:10BBA00001337B627B6D98447B6AFA699342D3DBF5
:10BBB000BB6A0133BB627B6D9944A5E7B86F00286F
:10BBC000C6D0C389A3F500739BB2C381C38903F4B4
:10BBD000F053002BBCD12CF0F3FDB9E70025B7E7FB
:10BBE00007F158002BF016FF40E6C389A3F5007358
:10BBF0009BB2C381C38903F4F053002B7FF4E0AE02
:10BC00002CF0DEFDDCE63865EDE600BFF0B593B064
:10BC10000446014602A81CF0EDFB18B90025284691
:10BC200013B0F0BD2CF08EFD05460028F6D0274855
:10BC3000274F2DF031FF014628462EF0EDFA25481A
:10BC40002DF02AFF014628462EF0E6FA204624F081
:10BC50001FFA0146064601A828F09EF8019C7CB90F
:10BC6000002EDCD0F389A3F500739BB2F381F38936
:10BC700003F4F053002BD2D130462CF0A1FDCEE7D7
:10BC8000E38903F500739BB2E38101223946204624
:10BC90002DF026F948B107216FF0004220462DF023
:10BCA00057FA014628462EF0B7FAE389A3F5007348
:10BCB0009BB2E381E38903F4F05313B920462CF0DF
:10BCC0007FFD01A828F02CF8C8E700BFCC210600B2
:10BCD000E3210600DC2106002DE9F0439DB000AF12
:10BCE00000230E4607F108018046BB602DF0B8FB2B
:10BCF0000546F8B940462EF00FFD0446B86026F020
:10BD000007FB04F58073834209D95949012026F0C5
:10BD100061FFA84640467437BD46BDE8F083E31D89
:10BD200023F00703ADEB030D6D462246294640463E
:10BD30002EF060FE012E01D1142000E0F0104FF033
:10BD40000009391DC7F80490F5F732F97C68804680
:10BD500024B9484827F0B2FAA046DBE7012E78D193
:10BD60005C22494607F11400BE68F3F7DBFB424B47
:10BD7000FB6103F188333B6203F12943A3F596137A
:10BD8000A3F68B637B62A3F18833BB623B4BFB6200
:10BD90002EB13246294607F1140016F047FE7A69A3
:10BDA000B969530F43EAC1031BBAFB60D30002F029
:10BDB0003F02372A1BBA94BFC2F13802C2F178029F
:10BDC0002F493B6107F1140016F030FE082207F1FD
:10BDD0000C0107F1140016F029FEFB7F2370FB8B8A
:10BDE0006370FB691B0AA370FB69E37097F823304B
:10BDF00023717B8C63713B6A1B0AA3713B6AE371FD
:10BE000097F827302372FB8C63727B6A1B0AA3723C
:10BE10007B6AE37297F82B3023737B8D6373BB6A65
:10BE20001B0AA373BB6AE37397F82F302374FB8D4F
:10BE30006374FB6A1B0AA374FB6AE37400231A464B
:10BE400007F11401194401335D2B3FF463AF0A700D
:10BE5000F6E7E02E06D101232246B968284616F0FF
:10BE60001BFD57E7B6F5807F7FF454AF4B46F3E7F1
:10BE7000FF220600721F060001234567F0E1D2C3CE
:10BE800070260600024B0349586800222EF0EABAD9
:10BE90008C2E00200119060010B51D4C237883421A
:10BEA00006D002461B490420BDE8104026F092BE91
:10BEB00000232370184C206890B129B3114604F078
:10BEC000D5FB206850B1C389A3F500739BB2C38131
:10BED000C38903F4F0530BB92CF072FC00232360E8
:10BEE0000E4C206850B1C389A3F500739BB2C38187
:10BEF000C38903F4F0530BB92CF062FC00232360D8
:10BF0000074B01221A7010BD114604F00FFCD8E750
:10BF100060D50020D018060058D5002064D5002038
:10BF200069D5002010B50A460C460021FFF7B4FF82
:10BF30006CB1E389A3F500739BB2E381E38903F459
:10BF4000F05323B92046BDE810402CF039BC10BD99
:10BF500010B5094B1C78012C0CD100210846FBF7C9
:10BF600079FD06482DF098FD01462046BDE81040B9
:10BF7000FFF7D8BF10BD00BF60D50020CD1B060065
:10BF80000A460021FFF788BF73B5002241490546E4
:10BF90002EF068FA2FF086F83F4B40490646032200
:10BFA00058682EF05FFA044678B12A46B1B22EF0F6
:10BFB0008BF9E389A3F500739BB2E381E38903F472
:10BFC000F05313B920462CF0FBFB002234492846DD
:10BFD0002EF048FA2FF066F880B2002846D12946A4
:10BFE0000820FCF787FE18B90024204602B070BD77
:10BFF0002C4B1C6824B1E38903F500739BB2E381E9
:10C00000294E33884FF6FF729A4207D127482DF008
:10C0100043FD01460820FFF785FFE6E700221D49A2
:10C0200028462EF01FFA2FF03DF8013080B2ADF80F
:10C030000400ADF8060001A9308815F00DFA15F0DE
:10C040009DF905460028D0D001460820FFF798FF4B
:10C05000EB89A3F500739BB2EB81EB8903F4F053FA
:10C06000002BC2D128462CF0ABFBBEE700210920F3
:10C07000FCF740FE0028B7D00A4B1C6824B1E389C6
:10C0800003F500739BB2E3810121284610F002F909
:10C09000ABE700BF991906008C2E0020A6190600F8
:10C0A0007F19060058D500208C2D00208B19060022
:10C0B00070B5014606460720FCF71CFE00283AD062
:10C0C0001E4B1C6824B1E38903F500739BB2E38126
:10C0D0001B4D2B884FF6FF729A4208D119482DF05C
:10C0E000DBFC01460720FFF71DFF204670BD002244
:10C0F000154930462EF0B6F92EF0D4FF2B8881B2C8
:10C100000022184615F0A6F915F038F90546002862
:10C11000EBD001460720FFF733FFEB89A3F500734F
:10C120009BB2EB81EB8903F4F053002BDDD1284661
:10C130002CF046FBD9E70446D7E700BF58D50020CE
:10C140008C2D00208B190600991906002DE9F04F5F
:10C1500085B0884600AF00230646394640463B601E
:10C160002DF07EF90546F8B940462EF0D5FA044682
:10C17000386026F0CDF804F58073834209D942492E
:10C18000012026F027FD2C4620461437BD46BDE889
:10C19000F08FE31D23F00703ADEB030D6D46224640
:10C1A000294640462EF026FC00210620FCF7A2FD81
:10C1B00008B90446E8E7354B1C6824B1E38903F568
:10C1C00000739BB2E381324B1A884FF6FF719142A4
:10C1D000984607D12F482DF05FFC01460620FFF757
:10C1E000A1FED1E700222C49D7F8009030462EF06E
:10C1F00039F92EF057FF00221FFA80FA27493046FE
:10C200002EF030F9064600283CD0002224492EF0BA
:10C2100029F92FF0AEF8F389A3F500739BB2F381EF
:10C22000F38903F4F053834613B930462CF0C8FA6F
:10C2300000239B453B8114BF022301233B71391D21
:10C240000123B8F800007B71FD60A7F806A0A7F8ED
:10C250000A9015F0FDF815F091F80546002893D0E6
:10C2600001460620FFF78CFEEB89A3F500739BB215
:10C27000EB81EB8903F4F053002B85D128462CF099
:10C280009FFA81E78346D3E7FF22060058D50020B6
:10C290008C2D00208B19060099190600AD19060097
:10C2A000B819060038B50D4601460A20FCF722FDF4
:10C2B000002839D01D4B1C6824B1E38903F50073B5
:10C2C0009BB2E3811A4B1A884FF6FF71914208D155
:10C2D00018482DF0E1FB01460A20FFF723FE204617
:10C2E00038BD1888144B1B7880B2DBB100232A4676
:10C2F0001946F8F7DFFA15F041F805460028EED0A8
:10C3000001460A20FFF73CFEEB89A3F500739BB2C0
:10C31000EB81EB8903F4F053002BE0D128462CF09D
:10C320004FFADCE70820E6E70446D8E758D50020B6
:10C330008C2D00208B190600ECCE002000000000A0
:10C34000F0B58BB06D460C46294616F093FC0028DC
:10C3500000F08D800022012395E80300ADF818203D
:10C360008DF81830A023ADF81A30454BADF80C10FD
:10C37000CDE90732434B0290090C58688DF80E1036
:10C38000414909922EF06EF82EF08CFEC3074CBF87
:10C390003E4B3F4B089320464FF0C87309932BF058
:10C3A000DDFC002841D000223A4920462EF05AF800
:10C3B0002FF07EFD02460B4606460F4634F050FE37
:10C3C00090B90022344B3046394634F0AFFB2AA3F3
:10C3D000D3E9002334F0D4FC0022304B34F0F0F9E0
:10C3E00034F07CFEADF8200000222D4920462EF0CE
:10C3F00039F82FF05DFD02460B4604460D4634F039
:10C400002FFE90B90022244B2046294634F08EFBA3
:10C4100019A3D3E9002334F0B3FC00221F4B34F0FE
:10C42000CFF934F05BFEADF8220002AB93E80300D5
:10C43000ADF81410090C04908DF8161008AA06A97E
:10C4400004A815F00FF814F099FF044678B10146DE
:10C450000220FFF795FDE389A3F500739BB2E3810A
:10C46000E38903F4F05313B920462CF0A9F90BB07B
:10C47000F0BD00BFAFF300800000000000889340D3
:10C48000900004008C2E0020331D06009001200334
:10C490001000A0001B1D060000408F400000E03F80
:10C4A000271D06000A460121FFF7F6BC38B5124BDE
:10C4B0001C78012C05461DD100210846FBF7CAFA5D
:10C4C00021460E482DF0EDFE044609F08DFE5CB1CC
:10C4D000E389A3F500739BB2E381E38903F4F0538E
:10C4E00013B920462CF06CF929460120BDE83840EC
:10C4F000FFF7D8BF38BD00BF60D5002064D500204D
:10C500007CDF70472DE9F04FAC4D85B02B6800AF54
:10C51000044603F0040308460E463B602BF01EFC65
:10C52000002800F0BC800022A54930462DF09AFF7B
:10C53000B0B12EF0B7FD4FF47A73584340F2712337
:10C5400090FBF3F080B2B0F5804F9E4B28BF4FF4C4
:10C55000804020281A8838BF2020824218BF1880C7
:10C560000022994930462DF07DFF38B12EF001FFB1
:10C570002B68002875D023F400632B6000229349B8
:10C5800030462DF06FFF38B12EF0F3FE2B680028F7
:10C590006AD023F480532B6000228D4930462DF061
:10C5A00061FF8146002800F08480002307F10C0120
:10C5B000FB602CF055FF8046002864D148462EF0E1
:10C5C000ABF88246F86025F0A3FE0AF5807383423B
:10C5D0004DD98049012026F0FDFAB9F80E30A3F5B7
:10C5E00000739BB2A9F80E30B9F80E3003F4F05383
:10C5F00013B948462CF0E4F820462BF0AFFB8246F6
:10C6000008B9002C58D131462046FCF7E1F8002C3F
:10C6100040F0D2800024704D7049686822462EF0A8
:10C620002DFE32466E4968682EF028FE5CB1E38923
:10C63000A3F500739BB2E381E38903F4F05313B9CC
:10C6400020462CF0BDF83B680BB110F07BF840465B
:10C6500010F0A8F83B6843B310F0FCFB10F0A2F810
:10C6600023E043F4006388E743F4805393E70AF13F
:10C67000070323F00703ADEB030DE846524641469E
:10C6800048462EF0B7F911234146BA893B7207F1AB
:10C690000800FFF735FF804610F084F89DE746B1AB
:10C6A00032465049032026F095FA1437BD46BDE8BE
:10C6B000F08F4FF000089FE720462BF047FB786093
:10C6C000002868D0E38903F500739BB2E3812B68EF
:10C6D00023F47F0323F40043214607F10C002B6071
:10C6E00027F05AFBD346F86850B9BAF1000F92D040
:10C6F000BBF1010F8FDD2B6843F400432B608AE709
:10C700002DF00CFC81462BF029FB10B9B9F1000F7C
:10C710001ED131464846FCF75BF88246F86810B1F6
:10C7200051462DF025FABAF1000F0ED0BAF80E30AE
:10C73000A3F500739BB2AAF80E30BAF80E3003F4DA
:10C74000F05313B950462CF03BF8D7F804A009E099
:10C7500048462BF0FBFA0028F7D148462BF0DAFACE
:10C760000028F2D10BF1010BB9F1000F0ED0B9F88E
:10C770000E30A3F500739BB2A9F80E30B9F80E3055
:10C7800003F4F05313B948462CF01AF807F10C00E3
:10C7900027F0C6FAA7E720462BF0BCFA00283FF4A2
:10C7A00039AFE38903F500739BB2E3812B6823F46F
:10C7B0007F0323F40043A1E704462CE75CD5002067
:10C7C000E31C0600502D0020EC1C0600F81C06009F
:10C7D000D7240600FF2206008C2E0020021D060032
:10C7E0000C1D06004E1B060072DF7047F0B5264B8D
:10C7F000264983B0044600AF024658682EF03EFD3D
:10C8000020462BF0A3FAE8B10023391D20467B60B7
:10C810002CF026FE054668BB20462DF07DFF06461F
:10C82000786025F075FD06F58073834217D91849A5
:10C83000012026F0CFF91749032026F0CBF90C3759
:10C84000BD46F0BD20462BF065FA0028DCD1002C57
:10C85000F5D022461049032026F0BCF9EFE7F31D7E
:10C8600023F00703ADEB030D6D4632462946204603
:10C870002EF0C0F800213B792A460846FFF7B4FFA6
:10C880000FF090FFDBE700BF8C2E0020A11D0600FB
:10C89000FF220600AA1D0600D61D060070B5394C01
:10C8A0003949206800222DF0DDFD054678B10021D0
:10C8B00001200FF01DFFEB89A3F500739BB2EB8104
:10C8C000EB8903F4F05313B928462BF079FF0022CB
:10C8D0002E4920682DF0C6FD054670B101200FF0ED
:10C8E000DDFEEB89A3F500739BB2EB81EB8903F4CA
:10C8F000F05313B928462BF063FF002224496068E7
:10C900002DF0B0FD00220546224960682DF0AAFDF9
:10C91000064605B918B131462846FFF7F3FD28460B
:10C9200031462DF01FFA00221B4960682DF09AFD58
:10C93000054668B111F00AFBEB89A3F500739BB2C1
:10C94000EB81EB8903F4F05313B928462BF038FF41
:10C950006068124900222DF085FD044668B1FFF79A
:10C9600045FFE389A3F500739BB2E381E38903F4F8
:10C97000F05313B920462BF023FFBDE8704010F0B0
:10C980007BBC00BF8C2E0020961D0600741906008B
:10C99000021D06000C1D0600991E0600A11D0600C2
:10C9A0002DE9F043C38903F5007391B09BB20446AF
:10C9B000C38103A8884615461BF028F990B30121CE
:10C9C0002E481AF0CBFF064648B31FFA88F02BF02A
:10C9D000CEFE2B49024620462DF00BFD00222949B0
:10C9E00020462DF03FFDDDF82690009007461FFA07
:10C9F00088F30022294603A8C847002816DA2249EE
:10CA0000042026F0E7F801202BF0A9FE1F4902467A
:10CA100020462DF0EEFC314638462DF0A3F903A850
:10CA20001BF04EF8204611B0BDE8F08301302BF02A
:10CA30009EFE1749024620462DF0DBFC022D17D141
:10CA4000012114481AF08AFF05460028E3D0214648
:10CA50002DF0C0FBEB89A3F500739BB2EB81EB8952
:10CA600003F4F053002BD6D128462BF0A9FED2E7D1
:10CA7000214630462DF0AEFBCDE700BF1124060065
:10CA8000B7250600971F0600292406004224060049
:10CA9000492406004E24060013B5C389019003F50E
:10CAA00000739BB20C46C3810E492DF081FC02221B
:10CAB00021460198FFF774FF50B1C389A3F50073B5
:10CAC0009BB2C381C38903F4F0530BB92BF078FEFA
:10CAD00001980449012301AA20F0D8F8019802B076
:10CAE00010BD00BF8F1F06002DE9F0478EB0054630
:10CAF0008A4617462BF04BFA814620B12846002182
:10CB0000FDF7A2F9054628462BF028F9044638B966
:10CB10005748294626F0D2FB20460EB0BDE8F087E4
:10CB2000BAF1000F07D050462BF030F9044610B987
:10CB300051465048EEE7022F16D101A81AF0DAFF4D
:10CB400090B100224C4928462DF08CFC2EF0AAFA18
:10CB5000DDF80D30834204DACDF80D0001A81AF09B
:10CB6000C3FF01A81AF0ACFF012144481AF0F6FEF9
:10CB7000064600287AD0012F6DD14149002023F0CC
:10CB800003FB044690B9F389A3F500739BB2F381CC
:10CB9000F38903F4F05313B930462BF011FEB9F1C9
:10CBA000000FB9D0002D39D12C46B5E7354900200A
:10CBB00023F0EAFAA046044644B3394620461AF068
:10CBC000D3FDBAF1000F10D02F4A514620462DF068
:10CBD0002EFF50B1C389A3F500739BB2C381C389F3
:10CBE00003F4F0530BB92BF0EBFD214630462DF04A
:10CBF000F1FAB8F1000F04D04246244920462DF046
:10CC0000D7FB2A46224920462DF0D2FB314640462A
:10CC10002DF0A8F8B9F1000F0CD05DB1EB89A3F5A8
:10CC200000739BB2EB81EB8903F4F05313B92846F0
:10CC30002BF0C6FD002F7FF46FAF01A81AF0E6FFBE
:10CC400000283FF469AF01A8214618F08DF901A82A
:10CC50001AF036FF60E7022F0CBF0E490E49002084
:10CC600023F092FA4FF000080446A5E70446D1E706
:10CC7000AF230600C5220600DF230600EE230600D0
:10CC8000F5230600FD230600F4220600604006009E
:10CC9000971F0600052406000A24060070B58EB012
:10CCA000044601A80E461AF0B1FF18B90024204628
:10CCB0000EB070BD20462BF051F858B11F482CF033
:10CCC000EBFE1F4A0146054620462DF0A3FE2946ED
:10CCD0002DF048F830462DF021F90546F8B12BF03B
:10CCE00055F880B92946174826F0E8FAEB89A3F5EC
:10CCF00000739BB2EB81EC8914F4F054D6D1284632
:10CD00002BF05EFDD3E7EB89A3F500739BB2EB81BB
:10CD1000EB8903F4F05313B928462BF051FD20465C
:10CD200001223146FFF7E0FE044618B1014601A892
:10CD300018F00EFB01A81AF0C3FEB8E7972506000D
:10CD40009B250600C522060010B504461BF018FB03
:10CD5000094B01221A70206860B1C389A3F50073E2
:10CD60009BB2C381C38903F4F0531BB9BDE81040E3
:10CD70002BF026BD10BD00BFAFD5002038B505464D
:10CD800000F02AFC044610B90025284638BD0146AB
:10CD900028461BF02FFB05460028F6D1E389A3F5B2
:10CDA00000739BB2E381E38903F4F053002BEBD1D2
:10CDB00020462BF005FDE8E700B50A4A137891B04C
:10CDC000013B68461370FFF7D9FF40B168466FF02A
:10CDD000050200211BF006F96846FFF7B5FF11B008
:10CDE0005DF804FBCC2D0020034B00221A705A7012
:10CDF0009A70DA70704700BFABD50020F7B50546D2
:10CE000018460E4617462CF047FE002304460093B2
:10CE100001463B4632462868FEF798FC214603B09F
:10CE2000BDE8F0402CF09EBF70B590B004460D46B2
:10CE30000146684616461BF0DDFA88B33EB140F263
:10CE4000FF339D42A8BF1D46012DB8BF0125BDF887
:10CE5000143003F46043B3F5C04F14D105F46043BC
:10CE6000B3F5C04F0FD00F4920462EF0EDF90E4913
:10CE700020462EF0E9F90D4920462EF0E5F90C493F
:10CE800020462EF0E1F96846ADF814501BF078FA10
:10CE9000E38903F500739BB2E381204610B070BDB7
:10CEA0000446FAE77B22060080220600D72106000E
:10CEB000852206002DE9F84F074608460E4615461E
:10CEC0002BF065F8002862D00122324930462CF060
:10CED00007F88046E8B16FF00042062130462CF09A
:10CEE00037F92EF0DFF8002D02DC84B2012505E0D1
:10CEF000ACB241F6FF708542A8BF054676B905F58C
:10CF00000054A4B2424621463846BDE8F84FFFF728
:10CF10008BBF002D4FF6FF74EBDCE7E71E49304670
:10CF20002BF0E6FF83460028E9D14FF6FF739C42C1
:10CF3000E8D1314619482CF01BF95A460146814682
:10CF4000384625F0B1FF824698B15B465A463946CD
:10CF500021F0CEFE50B1C389A3F500739BB2C3810B
:10CF6000C38903F4F0530BB92BF02AFC05F5C04438
:10CF7000A4B2494650462CF0F5FE4FF6FF739C4292
:10CF8000C0D132460649012025F024FEBAE7BDE8AB
:10CF9000F88F00BFDC210600CC210600FD21060031
:10CFA0000722060001381F289DBF034B23FA00F01B
:10CFB00000F00100002070478B80808030B551EC7C
:10CFC000100B85B053EC112B8DED000B55EC124B73
:10CFD0008DED021B34F01CF89DED000B28B19DED8A
:10CFE000021BB0EE410AF0EE610A53EC102B204612
:10CFF00029468DED000B34F00BF89DED000B08B1C8
:10D0000045EC104B05B030BD38B555EC104B002247
:10D01000002310EE100A294633F0FAFF10B105F193
:10D0200000431D4645EC104B38BD10B413460A466C
:10D0300053F8044B0021A4465DF8044B60472DE9EA
:10D04000F04F9BB00AAD80460F4601462846164673
:10D050001C461BF0CFF90290002800F09C80249B16
:10D06000099307AA06A92846CDE9067608941AF07E
:10D070009BFF09AA08A928461AF096FF0698089B64
:10D080000799099CC21802EBD27252101B1A009227
:10D0900003EBD3730A19641A5B1004EBD4746410A5
:10D0A00005935B43039302EBD27204FB04F352102B
:10D0B00004930192DDE903326600013E03FB16266C
:10D0C0000027009B03EB070B019B03EB040A52466E
:10D0D0000D9B594628461AF0C2FE009BA3EB070998
:10D0E00052460D9B494628461AF0B9FE019BA3EB18
:10D0F000040A52460D9B594628461AF0B0FE2846AF
:10D100000D9B524649461AF0AAFE049A7B0003FB87
:10D11000022271009142BFBF049A0298033302FBBE
:10D1200003664FEA440C039BCCF1010203FB02F2BD
:10D13000B4BF01370020914208DD039AACF103032C
:10D14000013C02FB1366002CBBDA01E00028FAD197
:10D15000059BBB4207F101040DDC28461BF010F9CA
:10D16000B8F80E3003F500739BB2A8F80E304046B5
:10D170001BB0BDE8F08FDDE900120D9B214428466D
:10D180001AF06DFEDDE900120D9B091B28461AF00E
:10D1900066FE2746DCE7DDF80880E8E737B5054698
:10D1A0001C4613440093121B0B19091BFFF747FF82
:10D1B000EB8903F500739BB22846EB8103B030BDC9
:10D1C0002DE9F04F9DB00CAD80460F460146284634
:10D1D00016461C461BF00EF90590002800F08C80C6
:10D1E000269B0B9309AA08A92846CDE908760A943C
:10D1F0001AF0DAFE0BAA0AA928461AF0D5FE0898FA
:10D200000A9B09990B9CC21802EBD272521003922E
:10D210000A19641A1B1A04EBD474641003EBD37359
:10D220005B1002EBD27266005210079304FB04F904
:10D230005B43013E0492069303FB16960027039B73
:10D2400003EB070A049B1A19039BA3EB070B0F9B25
:10D250005146CDE9002328465B461AF0A1FD049B08
:10D260001A1B0F9B2846CDE9002351465B461AF056
:10D2700097FD7B0003FB099271009142BCBF033311
:10D2800009FB03664FEA440C069BB8BF0598CCF136
:10D29000010203FB02F2B4BF01370020914208DD16
:10D2A000069AACF10303013C02FB1366002CC6DABC
:10D2B00001E00028FAD1079BBB4207F101040DDC15
:10D2C00028461BF05DF8B8F80E3003F500739BB2EA
:10D2D000A8F80E3040461DB0BDE8F08F0F9B0193BB
:10D2E000DDE90312049B0093039B21441B1B28468A
:10D2F0001AF056FD2746DEE7DDF81480EAE737B579
:10D3000005461C4613440093121B0B19091BFFF71B
:10D3100057FFEB8903F500739BB22846EB8103B0FE
:10D3200030BDF0B597B004460F46014606A8164634
:10D330001D461BF05FF800283FD01C9B059303AAF5
:10D3400002A906A8CDE9027604951AF02DFE05AAD9
:10D3500004A906A81AF028FE039A099B0299CDE9B0
:10D36000002306A8049B1AF01BFD099B0193059B53
:10D370000093DDE9032306A819461AF011FD059A6A
:10D38000099B0299CDE9002306A8049B1AF008FD29
:10D39000099B0193039B0093029B059A194606A8DB
:10D3A0001AF0FEFC06A81AF0EBFFE38903F5007300
:10D3B0009BB2E381204617B0F0BD0446FAE7F0B512
:10D3C00093B004460D46014602A816461F461BF0C0
:10D3D00011F8A0B1069B0193189B009332463B467F
:10D3E000294602A81AF08AFF02A81AF0C9FFE389A9
:10D3F00003F500739BB2E381204613B0F0BD0446F1
:10D40000FAE7F0B593B004460D46014602A8164669
:10D410001F461AF0EFFFA0B1059B0193189B0093E4
:10D4200032463B46294602A81AF068FF02A81AF0C5
:10D43000A7FFE38903F500739BB2E381204613B095
:10D44000F0BD0446FAE710B590B0044601466846C0
:10D450001AF0D0FF60B3002242F201012046FFF72C
:10D46000E3FCBDF80730013BADF81F30BDF80930D3
:10D47000013B0022ADF821304FF0FF33CDE90332FC
:10D4800042F201030593069BADF81C2003F4400310
:10D4900043F47023684606938DF81E201AF070FF3F
:10D4A000E38903F500739BB2E381204610B010BD01
:10D4B0000446FAE710B5044690B069B1FFF7C3FF20
:10D4C00050B1C389A3F500739BB2C381C38903F430
:10D4D000F0530BB92BF074F9214668461AF08AFF15
:10D4E00068B168461AF0AAFC68461AF049FFE38959
:10D4F00003F500739BB2E381204610B010BD0446D3
:10D50000FAE70000024621B3012924D0022924D0E1
:10D51000032924D0042924D0052924D0062924D085
:10D52000072924D0082924D0092924D00A2924D065
:10D530000B2924D00C2924D00D2924D00E2924D045
:10D54000134B14480F2908BF03461349012025F047
:10D5500041BB124BF9E7124BF7E7124BF5E7124BC1
:10D56000F3E7124BF1E7124BEFE7124BEDE7124BEB
:10D57000EBE7124BE9E7124BE7E7124BE5E7124BFB
:10D58000E3E7124BE1E7124BDFE7124BDDE700BFA9
:10D590005D3C0600F43C0600FC3C0600653C0600D1
:10D5A000683C0600713C0600793C0600833C06009E
:10D5B0008B3C0600933C0600A03C0600A73C0600FE
:10D5C000AD3C0600BC3C0600CC3C0600DA3C060044
:10D5D000E63C0600503C0600024B03495868002216
:10D5E0002CF040BF8C2E0020177E060070B5002264
:10D5F00086B00E461D492CF035FF04462AF0C7FCC4
:10D600000546B0B10022214601A82AF00DFC0025F4
:10D61000DDE9013293421CD3049850B1C389A3F5CC
:10D6200000739BB2C381C38903F4F0530BB92BF091
:10D63000C7F85CB1E389A3F500739BB2E381E3898A
:10D6400003F4F05313B920462BF0BAF8284606B07D
:10D6500070BD059800B1C05C864214BF284645F0F5
:10D660000100C5B201A82AF0D5F9D1E7AD40060006
:10D670002DE9F04390461D46421E47F6FE739A423E
:10D6800091B006460F4602D84A1E9A4208D931493F
:10D69000012025F09FFA0024204611B0BDE8F08358
:10D6A0004046FFF77FFC044620B92B49012025F0B6
:10D6B00091FAF1E728462AF051FBD8B10022274918
:10D6C00028462CF0CFFE00220446254928462CF09F
:10D6D000C9FE2546814628462AF058FB044680B9F3
:10D6E0002A462049012025F075FA494628462CF0A3
:10D6F00039FBD1E7EB8903F500739BB2EB818146DF
:10D70000E9E7B9F1000F06D048462AF03FFB04468E
:10D7100008B94A46E5E71449002022F035FD0446E1
:10D720000028B9D043463A46314668461AF02EFFE3
:10D7300001232A460D498DF80430204600942CF030
:10D7400037FE4A460A4900982CF032FE68461AF025
:10D7500017FECAE7F53E0600023F06000E3F060030
:10D76000173F0600203F060093200600543F0600A6
:10D770005E3F060070B506460D462AF008FC0446DA
:10D7800030B932461349032025F024FA204670BDF3
:10D790001149002022F0F8FC3246104904462CF0D2
:10D7A00007FE45B128462AF0F2FB68B9324609491E
:10D7B000032025F00FFA00202AF0D9FF084902467D
:10D7C00020462CF016FEE1E72A46064920462CF0BA
:10D7D000EFFDF0E771400600961706009C4006003A
:10D7E000A3400600AD40060038B5002208490546B2
:10D7F0002CF038FE044640B9064922F0C5FC044925
:10D800000446024628462CF0D3FD204638BD00BF12
:10D810004BB00600644006002DE9F04190461D46DD
:10D82000421E47F6FE739A4290B006460F4602D853
:10D830004A1E9A4205D96349012025F0CBF90024FC
:10D8400008E04046FFF7AEFB044638B95E490120C8
:10D8500025F0C0F9204610B0BDE8F0815B490020FA
:10D8600022F092FC04460028F4D031466846434634
:10D870003A461AF08BFE002628468DF804608DF893
:10D8800005608DF8066000942AF068FA002865D0DB
:10D8900032464F4928462CF0E5FD2DF06AFD28B1AF
:10D8A000BDF8053043F00103ADF8053000224949C9
:10D8B00028462CF0D7FD2DF05CFD28B1BDF80530D1
:10D8C00043F00403ADF805300022434928462CF00C
:10D8D000C9FD2DF04EFD28B1BDF8053043F0080319
:10D8E000ADF8053000223D4928462CF0BBFD2DF057
:10D8F00040FD88B19DF80B0001280BD1BDF8053023
:10D9000043F00203ADF80530BDF809305B0703D0E2
:10D91000334992E733498FE72846002232492CF0F9
:10D92000A1FD0546D0B131492BF0E2FA50B930499A
:10D9300028462BF0DDFAC0B9BDF8053043F080036E
:10D94000ADF80530EB89A3F500739BB2EB81EB8951
:10D9500003F4F05313B928462AF032FF68461AF050
:10D9600005FA68461AF00CFD74E7224928462BF0A8
:10D97000BFFA20B9BDF8053043F48073E0E71E49D3
:10D9800028462BF0B5FA20B9BDF8053043F4C07332
:10D99000D6E71A4928462BF0ABFA20B9BDF8053076
:10D9A00043F40073CCE7164928462BF0A1FA20B9BE
:10D9B000BDF8053043F42073C2E7124825F05EFC41
:10D9C000C0E700BFF53E0600023F060093200600B8
:10D9D000223E0600293E06002D3E0600393E060086
:10D9E000773E0600473E0600B03E0600BC3E0600FD
:10D9F000C03E0600C43E0600C83E0600CC3E0600FF
:10DA0000D03E0600D43E060008B500222DED028B64
:10DA1000B0EE408AF0EE608A002351EC100B33F038
:10DA20000BFB98B1B0EE480AF0EE680A31F0CCF882
:10DA30000B4B51EC100B002233F078F8BDEC028B4D
:10DA400041EC100BBDE8084031F03AB8BDEC028B58
:10DA50009FED010B08BD00BF000000000000F87F33
:10DA60000000E03F00000000F8B555EC104B25F039
:10DA700000474FF0FF32284B2046394633F0F0FA8A
:10DA800060B94FF0FF32244B2046394633F0DEFABE
:10DA900020B9B5F1004F08BF002C05D145EC104B63
:10DAA000BDE8F8402AF051BE002200232046294656
:10DAB00033F0AEFAC8B912A1D1E900012B462246D3
:10DAC00032F07EFE06460F4633F090FB04460D46CC
:10DAD00054EA05030DD1002200233046394633F0C5
:10DAE00097FA30B19FED080BDAE709A1D1E90001FF
:10DAF000E4E720462946BDE8F8402AF04CBE00BFC6
:10DB00002083E4FFFFFFDF3F0000000000000080F3
:10DB10002083E4FFFFFFDFBFFFFFEF7F30F0CCBFCC
:10DB200030F04EBC30F068BF05202AF0A1BD0000E7
:10DB30002DE9F0478AB080462AF029FA044638B920
:10DB40006149032025F046F820460AB0BDE8F08779
:10DB50000022414668462AF067F900273C463E46C7
:10DB6000B9463D46DDE90032934212D3039850B1E5
:10DB7000C389A3F500739BB2C381C38903F4F05337
:10DB80000BB92AF01DFEFFF7CFFF0546D8B90024D8
:10DB9000DAE7049A6AB1D35C0A2B0AD155EA090381
:10DBA00008BF012709F101090025684629F032FF65
:10DBB000D8E7A14505F10105A8BF09F10104AE426E
:10DBC000B8BF2E46F1E730462AF0D1FD3F49024664
:10DBD00028462CF00EFC20462AF0C9FD3C4902469E
:10DBE00028462CF006FC04FB06F007300021C0108C
:10DBF0002BF0ECFE044668B9EB89A3F500739BB2E9
:10DC0000EB81EB8903F4F053002BC0D128462AF0B6
:10DC1000D7FD99E73A46414668462AF005F94FF0A4
:10DC2000000847464FF08009DDE90032934213D3E4
:10DC3000039850B1C389A3F500739BB2C381C38914
:10DC400003F4F0530BB92AF0BBFD224621492846C4
:10DC50002CF0CFFB2C4677E7049A5AB1D35C0A2B01
:10DC600006D108F101080027684629F0D3FEDBE75A
:10DC7000202B26D020462AF08AF910B306FB087A1A
:10DC800021464FEADA0205A82AF0CEF8099909B12F
:10DC9000059BC95C0AF0070A49FA0AFA41EA0A0137
:10DCA00005A8C9B229F0CAFD089850B1C389A3F5E7
:10DCB00000739BB2C381C38903F4F0530BB92AF0FC
:10DCC0007FFD0137D0E700BF683F06009C200600BB
:10DCD000A2200600CF450600FFF726BFFFF724BFAE
:10DCE00008B50B464022014618462DF077FD402826
:10DCF00005D10120034924F06DFF002008BD01205B
:10DD0000FCE700BFF53B0600F8B50F4606460022CB
:10DD1000114938462CF0A6FB0546D8B12AF073F815
:10DD2000044648B128462AF077F83760706090F8CA
:10DD30002642631E5C425C41EB89A3F500739BB2F3
:10DD4000EB81EB8903F4F05313B928462AF038FD30
:10DD50002046F8BD0446FBE7F03B060070B590B0E6
:10DD600006462AF03FF9054638B9324629490320CC
:10DD700024F030FF284610B070BD0122314605A8BE
:10DD800026F011F800231A4605A923481AF0F1FDE0
:10DD9000044605A825F0CDFC204600212BF016FEF8
:10DDA000044620B91D4825F089FA2546E2E70122FC
:10DDB000314605A825F0F7FF0022214668462AF0E3
:10DDC00033F86B46164A144805A91AF0D2FD039899
:10DDD00050B1C389A3F500739BB2C381C38903F417
:10DDE000F0530BB92AF0ECFC05A825F0A2FC0021A9
:10DDF00020462BF07BFBE389A3F500739BB2E38104
:10DE0000E38903F4F0530546002BB3D120462AF0F2
:10DE1000D7FCAFE77B3F06008D670400721F06004A
:10DE2000AF67040070B590B006462AF0DBF80546EF
:10DE300038B932462949032024F0CCFE284610B0D8
:10DE400070BD0122314605A825F0ADFF00231A461A
:10DE500005A923481AF081FE044605A825F069FCAF
:10DE6000204600212BF0B2FD044620B91D4825F0C4
:10DE700025FA2546E2E70122314605A825F093FF61
:10DE800000222146684629F0CFFF6B46164A144807
:10DE900005A91AF062FE039850B1C389A3F5007377
:10DEA0009BB2C381C38903F4F0530BB92AF088FCF9
:10DEB00005A825F03EFC002120462BF017FBE38946
:10DEC000A3F500739BB2E381E38903F4F0530546A5
:10DED000002BB3D120462AF073FCAFE77B3F06004E
:10DEE0008D670400721F0600AF670400F8B5051EB9
:10DEF0000C4606DC2949012024F06CFE0024204653
:10DF0000F8BD084629F02AFF0646A8B10022244998
:10DF100020462CF0A7FA2DF02CFA002221490646C3
:10DF200020462CF09FFA2DF0BDF830F0080309D000
:10DF3000102809D01C49DEE724B122461B490120E4
:10DF400024F048FE012400E00224294620462AF05D
:10DF50001CFD07469EB1294620462AF016FD0546BF
:10DF60001349002022F010F9044610B10FB146B158
:10DF70003DB92A46394620462BF0C8FEBEE7354655
:10DF8000EEE73A460B4920462CF033FA002DB6D086
:10DF90002A46094920462CF02CFAB0E7DC4206005C
:10DFA000FB4206001A430600084306001F43060012
:10DFB00056430600CF4506005F43060070B50D1EB0
:10DFC000064606DA0B49012024F004FE0024204610
:10DFD00070BD1B202AF04CFB044615F1FF35F6D32B
:10DFE00024F072F90028F2D1314620462BF0ABF82C
:10DFF000F3E700BFC842060038B5044629F0AEFE7C
:10E00000D8B100220E4920462CF02CFA054629F002
:10E01000BEFF10B128462BF0C6F904465DB1EB896E
:10E02000A3F500739BB2EB81EB8903F4F05313B9B2
:10E0300028462AF0C5FB204638BD0446FBE700BF52
:10E0400087420600F8B506460F46144629F09FFFA2
:10E050000546E8B1204629F0BDFED8B120462BF098
:10E0600095FF054638462DF0DFF904462BF09BF965
:10E070002D1A13D500255CB1E389A3F500739BB27B
:10E08000E381E38903F4F05313B920462AF098FBA7
:10E090002846F8BD30462BF086F9E2E720462BF003
:10E0A00082F92F1830462BF07EF98742E2D82A46B3
:10E0B000012321463046F2F75FFCB0FA80F56D0986
:10E0C000D9E7F8B507460D46164629F060FF044625
:10E0D00098B128462DF0A8F9002E05460FDA002445
:10E0E0005DB1EB89A3F500739BB2EB81EB8903F47F
:10E0F000F05313B928462AF063FB2046F8BD2BF0F5
:10E1000052F9841938462BF04EF98442E7D801239E
:10E11000324629463846F2F72FFCB0FA80F46409FB
:10E12000DEE7F0B587B02DF07FF90546002842D034
:10E130000146002201A829F077FE4FF0FF340027A6
:10E14000DDE901639E4225D3049850B1C389A3F54C
:10E1500000739BB2C381C38903F4F0530BB92AF057
:10E160002FFBA742DABFE21B0132002239462846C4
:10E170002AF0EEFFEB89A3F500739BB2EB81EB89EC
:10E1800003F4F053044613B928462AF019FB20463D
:10E1900007B0F0BD059800B1805D25F0F1F930B908
:10E1A000039B1E4437EA240728BF3746344601A89C
:10E1B00029F030FCC4E70446E9E7F8B506460D4609
:10E1C0000AB310462BF0E2FE002D044603DA304677
:10E1D0002BF0E9F80544002C03DA30462BF0E3F885
:10E1E00004441B202AF044FA25EAE57524EAE47485
:10E1F000074630B1A54204DA631B2A4631462AF0AD
:10E2000064FF3846F8BD00296FF00044E9DADEE724
:10E21000F8B505460C46C2B110462BF0B7FE20EA11
:10E22000E076002C05DA28462BF0BDF8044424EAF9
:10E23000E4741B202AF01CFA074620B1334622461C
:10E2400029462AF042FF3846F8BD6FF00046E8E75D
:10E25000F8B507460C46CAB110462BF097FE20EAE7
:10E26000E07524EAE474A542B8BF23464FF01B00D2
:10E27000BCBF2C461D462AF0FBF9064620B12B1BDD
:10E28000224639462AF021FF3046F8BD6FF00040A3
:10E29000E5E708B508B1036823B91B20BDE80840CD
:10E2A0002AF0E6B900212BF061FEBDE808402DF010
:10E2B000E9B908B52AF0E8FE08BD70B5054686B094
:10E2C0001B200E462AF0D4F9044630B3284629F024
:10E2D0005EFE10B3002E20DB3246294601A829F04D
:10E2E000A3FDDDE901239A420AD2059B03B19B5CA1
:10E2F0008DF8033001220DF1030120462AF08EFF34
:10E30000049850B1C389A3F500739BB2C381C3893C
:10E3100003F4F0530BB92AF053FA204606B070BD4F
:10E3200037B505461B202AF0A3F9044628B1294633
:10E3300001A825F031FD019810B9204603B030BD89
:10E340002BF0ECFD2CF0AEFE01228DF803000DF158
:10E35000030120462AF062FF01A825F0E1FCEAE76C
:10E36000F8B507460E4629F0F9FC00283CD00022FB
:10E370001E4938462CF076F8044629F008FE70B3A2
:10E3800020462BF010F8002E01DD864206D31749F7
:10E3900038462CF059FF25462846F8BD3246002164
:10E3A00020462AF0D5FE6FF0004231460546204651
:10E3B0002AF0CEFE0D49024638462CF01AF8002C01
:10E3C000EAD0E389A3F500739BB2E381E38903F408
:10E3D000F053002BE0D120462AF0F2F9DCE71B20B5
:10E3E0002AF046F90546EAE70546D5E787420600E2
:10E3F0002DE9F041CB1D23F0070300AFADEB030D7A
:10E40000134614466E460D4653F8048B0A463146B1
:10E41000C047A3692B44A36163692B4463613544FE
:10E420001C34AE4202D1BD46BDE8F081204616F84C
:10E43000011B25F0FAF9204625F0A9F9F1E70000C3
:10E440002DE9F04F93B000AF0E46154681461EF001
:10E450007FFC4FF0010A044607F11701304687F8A8
:10E4600017A0F3F763FB002D804606DC4FF0000891
:10E4700040464C37BD46BDE8F08F23F049FF05F517
:10E480008073834204D95F49504624F0A3FBEDE733
:10E49000EB1D23F00703ADEB030D142C6E463BD1AF
:10E4A000594B1B78CBB1002307F120024FF04021DC
:10E4B0005648C7F82230C7F826307B8587F820A059
:10E4C00087F8218087F822507E62F7F7B3F802467A
:10E4D00018B14F49042024F07DFB294601202AF081
:10E4E00054FA80460028C1D00146002207F12000DE
:10E4F00025F0B9FB354416F8011B07F1200025F083
:10E5000094F907F1200025F042F9B542F3D107F163
:10E51000200025F0FEF8ABE7002CA7D13D492246AC
:10E5200048462BF09FFF8246014607F118001DF078
:10E530000DFA002859D02246374948462BF092FF61
:10E540002CF017FF3B7FB877FF2B4ED07A7FFF2A46
:10E550004BD0F97D87F8212087F82030BA6987F8F9
:10E5600022002E4B93FBF2F307F12000012BD8BFC2
:10E570002346F9607B621DF0AFF94FEA480101F4D0
:10E58000FF7141F0010107F120001DF05DF905F177
:10E59000FF38A8EB04035942594108224FF0000B01
:10E5A00007F12000C7E901121DF0F6F8BA68796892
:10E5B0004FEA4B0B013A40EA0B0BF1D107F1200077
:10E5C0001DF018F9012197F8210013F081FA06F8DF
:10E5D00004B00134A542DCD1FB681BB107F1200077
:10E5E0001DF046F997F82230BB77B87F2AF0B7F8CC
:10E5F0000949024648462BF0DBFE51462BF0B2FBA0
:10E600006BE700BFA03F060000D30020B8CB00207E
:10E61000D53F0600E83F0600F13F060090D003001A
:10E620002DE9F04F89B000AF0D46924680461EF0AE
:10E630008FFB4FF0010BF91D0446284687F807B001
:10E64000F3F774FA0023064607F108015046BB6051
:10E650002AF006FF0546F0B950462CF05DF88146D9
:10E66000B86023F055FE09F58073834207D9454908
:10E67000584624F0AFFA2437BD46BDE8F08F09F1C3
:10E68000070323F00703ADEB030D6D464A46294609
:10E6900050462CF0AFF9BB68002BECD0142C1DD1E8
:10E6A000394A1278002AE6D0F9793848BD6100224B
:10E6B00091427A61FA61BB754FF0402114BF134655
:10E6C000202307F114027E75F6F7B4FF02460028F6
:10E6D000D1D02F49042024F07DFACCE7002CCAD1F8
:10E6E0002C49224640462BF0BDFE8146014607F1EB
:10E6F0000C001DF02BF990B32246274940462BF021
:10E70000B1FE2CF036FE3B7CB874FF2B27D07A7C10
:10E71000FF2A24D07A753B75B875FA681F4B93FBB6
:10E72000F2F307F11400012BD8BF2346D7F808B045
:10E7300097F807A0BB611DF0CFF8710001F4FF71DD
:10E7400007F114001DF080F8A34514DCBAF1000FA6
:10E7500003D007F114001DF08BF8BB7DBB74B87CAF
:10E7600029F0FDFF0C49024640462BF021FE4946A8
:10E770002BF0F8FA7FE7295D07F114001DF064F82B
:10E780000134E1E7FF22060000D30020B8CB0020CF
:10E7900045400600E83F0600F13F060090D0030028
:10E7A0002DE9F04F89B0894600901EF0D1FA494614
:10E7B000044602A81DF0CAF840B3142C40F00281B0
:10E7C0009DF80C4020461EF011FC9DF80D5018B12C
:10E7D00028461EF00BFCE0B9224629468A4824F060
:10E7E0006DFDB9F1000F00F00A81884A0098494692
:10E7F0002CF010F950B1C389A3F500739BB2C3810B
:10E80000C38903F4F0530BB929F0DAFF09B0BDE86E
:10E81000F08F7F49029E7F4B04EB440405EB4505D6
:10E820000C440D449E4294F801806F7858DD7A4B79
:10E830009E42D4BF4FF080664FF0CD66774A784C49
:10E8400013785BB323681BB1764B1021C3F880109B
:10E850004FF040234FF0FF31C3F80813D3F80012F4
:10E860000021C3F80012C3F80015012184F822101A
:10E8700094F8271079B9D3F808154FF0A04001F5A6
:10E88000E07140F2023540F82150D3F80C3503F521
:10E89000E07340F82350002384F8223094F82230AB
:10E8A00001251570FBB108225F49042024F092F97C
:10E8B0009DF80C4020461EF099FB20B14FF42071CA
:10E8C000204613F08BFA9DF80D4020461EF08EFB7B
:10E8D000002886D04FF49451204613F07FFA80E749
:10E8E0004FF0CC76AAE79DF81E2084F827209DF8EB
:10E8F0001D20A360C4E9003384F8253084F8243057
:10E9000072B34FEA8800B90000F1A04001F1A041C4
:10E9100040F20C624FF0A04BC0F8002705FA08FA4D
:10E92000C1F80027BD4040F20D620193CBF808A565
:10E93000CBF80855C0F80027C1F800270420F4F7E9
:10E94000B5F9019BDBF810150D422BD043B14FF008
:10E95000A04A0420CAF80C55F4F7A8F9CAF80855DB
:10E960004FF0A04308F5E07140F20C6243F821201B
:10E9700007F5E07143F821204FF040231D46C3F80E
:10E980000885C3F80C75C3F8246522681AB10621FE
:10E990000420F7F709F80523C5F80035022384F8A9
:10E9A000223085E701930420CBF80CA5F4F77EF91B
:10E9B000CBF808A50420F4F779F9019B0133092B62
:10E9C000C0D1C4E7002C7FF40CAF9DF80C00FF28E9
:10E9D00007D0012113F07CF803219DF80C0013F0FF
:10E9E00043FB9DF80D00FF283FF4FBAE012113F01F
:10E9F0006FF803219DF80D0013F036FBF1E6034993
:10EA000000982CF021FC01E7F93F0600E83F0600E2
:10EA1000D017060097AB020087F5040000D3002052
:10EA2000B8CB002000E100E028400600F0B58DB032
:10EA30000D4616461C461EF08BF913289DF84870AB
:10EA400005D02F49012024F0C5F80DB0F0BD16B94E
:10EA50000CB90F2403262B4B1B78F6B2E4B25BB93A
:10EA60002949ADF810306FF0FF02CDE9011201A87D
:10EA7000264A039213F0D0F9FF2F03D00021384625
:10EA80001FF0D4F8284629F0A5F980B128462BF0CC
:10EA90007DFA22463146C0B2F2F752FDF2F730FC61
:10EAA000FF2FD2D0012138461FF0C0F8CDE728460D
:10EAB00029F098FAE8B1802383F3118801222946CE
:10EAC00001A825F070F901A824F08DFE054601A8E3
:10EAD00025B924F02EFE85F31188DFE725F007F82D
:10EAE00022463146C0B2F2F72BFD01A825F02DF9E0
:10EAF000E9E72A460649012024F06CF8CEE700BF7A
:10EB0000C0410600F2D20020A086010000010800EA
:10EB1000E8410600F0B58DB00D4616461C461EF0C5
:10EB200017F913289DF8487005D03049012024F0CA
:10EB300051F80DB0F0BD16B90CB9032401262C4BC9
:10EB40001B7806F00F0604F00F045BB92949ADF8F5
:10EB500010306FF0FF02CDE9011201A8264A03929E
:10EB600013F05AF9FF2F03D0002138461FF05EF84A
:10EB7000284629F02FF980B128462BF007FA2246C3
:10EB80003146C0B2F2F79CFCF2F7BAFBFF2FD0D0AF
:10EB9000012138461FF04AF8CBE7284629F022FA2F
:10EBA000E8B1802383F311880122294601A825F0CA
:10EBB000FAF801A824F017FE054601A825B924F0AB
:10EBC000B8FD85F31188DFE724F091FF2246314636
:10EBD000C0B2F2F775FC01A825F0B7F8E9E72A46BC
:10EBE0000649012023F0F6FFCEE700BF984106005A
:10EBF000F2D20020A086010000010800E8410600D2
:10EC0000F0B58BB004460E461EF0A2F801AD0746E3
:10EC10002A46694620461BF051F8B8B1009B05937F
:10EC200095E80F0006AC07C423808EB9FF2505AA1E
:10EC3000224930462BF042FC132F01D1F2F760FB42
:10EC4000FF2D03D0012128461EF0F0FF0BB0F0BDD0
:10EC500031680029EADD013930462BF087F9044696
:10EC600029F084FA30B320461EF045F905463046B7
:10EC70002CF098FA50B1C389A3F500739BB2C381FD
:10EC8000C38903F4F0530BB929F09AFD5CB1E38911
:10EC9000A3F500739BB2E381E38903F4F05313B946
:10ECA000204629F08DFDFF2DC1D0002128461EF001
:10ECB000BDFFBCE7002CB9D0FF25E8E72BD0020050
:10ECC0002DE9F041B8B00D46164607A908AA1AF07A
:10ECD000F5FF002800F08480FF2E03D0002130468D
:10ECE0001EF0A4FF284629F075F880462846B8F1A2
:10ECF000000F18D02BF04AF918A98DF8600008AB66
:10ED000008460122079CA0479DF8600029F02FFDCE
:10ED10000446FF2E03D0012130461EF087FF204617
:10ED200038B0BDE8F08129F032F9074600283DD01F
:10ED30001B2029F09DFC42460446294602A829F0E2
:10ED400073F8DDE902239A420FD305980028E0D03A
:10ED5000C389A3F500739BB2C381C38903F4F05345
:10ED6000002BD6D129F02CFDD3E723F0ADFA0028F3
:10ED7000EBD101AA694602A828F004FE019D002DEE
:10ED8000DFD0802D28BF802508AB2A4618A900981F
:10ED9000079FB8472A4618A920462AF03FFA019B48
:10EDA0005B1B0193009B1D440095E7E728462BF071
:10EDB000B3FC0146012029F0E8FD04460028A8D054
:10EDC0003A4601460EA8CDE90C7724F04CFF07AA7D
:10EDD000044928462BF072FB0EA824F09AFC98E711
:10EDE00004469CE7F1E302007FB50C4605461DF0A2
:10EDF000AFFF2146064668461AF0BCFEB0B1132E9E
:10EE000016D1684613F008F854B3184A214628462C
:10EE10002BF000FE50B1C389A3F500739BB2C381F0
:10EE2000C38903F4F0530BB929F0CAFC04B070BDD8
:10EE3000002EFBD19DF80500FF2802D0012113F020
:10EE400013F99DF80600FF2802D0042113F00CF9F5
:10EE50009DF80700FF28D7D0012113F005F9D3E76B
:10EE6000024928462CF0F0F9E0E700BFE83F060031
:10EE70002DE9F04300228DB0244906462BF0F2FA2A
:10EE800005AD014628462DF085FD1B22541E295D47
:10EE900009B1144602E02246002CF7D10CAB4FF02A
:10EEA00001081C440DF1240904F81C8C99E80700A2
:10EEB0008DE8070095E80F002DF04AFC08F10108E5
:10EEC00007460028F0D1012029F051FC10490246E4
:10EED00030462BF08EFA384629F049FC0D4902469F
:10EEE00030462BF086FA384629F041FC0A490246A2
:10EEF00030462BF07EFA384629F039FC07490246A5
:10EF000030460DB0BDE8F0432BF073BAD7240600AD
:10EF1000364206003C420600434206003D4D0600D4
:10EF20002DE9F04F00229BB00C46894906462BF094
:10EF300099FA2CF0B7F8C0B2772808D0612806D02B
:10EF40008449012023F046FE1BB0BDE8F08F204627
:10EF50002CF06AFA04460028F6D02AF024FA8146FA
:10EF60000028F1D000227C4930462BF07BFA2CF0AF
:10EF700099F800227949834630462BF073FA2CF039
:10EF800091F800227649804630462BF06BFA0BADA3
:10EF9000014628462DF0FEFC1B235F1EEA5D0AB1E8
:10EFA0001F4602E03B46002FF7D11AAB1F44002258
:10EFB0006C4907F83C8C30462BF054FA2CF072F870
:10EFC000CBF57E6A68BB4FF47E63CDE90503402331
:10EFD000CDE903430FAF97E807008DE8070095E8F8
:10EFE0000F002DF0B3FA00284ED012AB039397E830
:10EFF00007008DE8070095E80F002DF060FA054640
:10F00000484629F0B4FB5449024630462BF0F1F94A
:10F01000284629F0ACFB5349024630462BF0E9F96B
:10F0200032E0D1450BEB00030ADA2046194607F01F
:10F03000F1FE0BEB090029F09AFB47490246ECE789
:10F0400000215246204609932AF082F8099B834604
:10F05000194607F0DFFEBBF1000F0ED0BBF80E30F3
:10F06000A3F500739BB2ABF80E30BBF80E3003F47F
:10F07000F05313B9584629F0A3FBB8F1FF0F12D192
:10F080003949012023F0A6FDE389A3F500739BB263
:10F09000E381E38903F4F053002B7FF455AF20465E
:10F0A00029F08EFB50E708F1010007F83C0C29F02D
:10F0B0005EFB2A49024630462BF09BF96FF0004276
:10F0C000514620462AF044F800234FF47E62CDE9F1
:10F0D00005324023CDE903030DF13C08074698E8CB
:10F0E00007008DE8070095E80F002DF02FFA0028A3
:10F0F000CAD012AB039398E807008DE8070095E8A3
:10F100000F002DF0DCF90546484629F030FB124986
:10F11000024630462BF06DF9284629F028FB1149AC
:10F12000024630462BF065F938462AF03CF9054690
:10F130005FB1FB89A3F500739BB2FB81FB8903F4EC
:10F14000F05313B9384629F03BFB284673E700BF5C
:10F150003D4D0600604206003C4206003642060075
:10F16000D7240600434206007942060010B58CB051
:10F1700005AC014620462DF0F3FB0CAB13E907006C
:10F180008DE8070094E80F002DF0E2FA0CB010BDF6
:10F190002DE9F0474149A4B000222BF063F905ACFA
:10F1A0000546014620462DF0DBFB5DB1EB89A3F55A
:10F1B00000739BB2EB81EB8903F4F05313B928463B
:10F1C00029F0FEFA1B235E1EA25D0AB11E4602E074
:10F1D0003346002EF7D124AB1E444FF001080CAF8C
:10F1E00006F87C8C0DF12409039799E807008DE857
:10F1F000070094E80F002DF062F90546002847D07B
:10F200000C9B23F07F4303444FF0000A13F8013CAA
:10F21000FF2B02D0B8F1FF0F1ED10024C4F57E668B
:10F22000002E14DD402EA8BF40263246611914A8D6
:10F2300032F090F914AA002312F8011BFF2925D0FF
:10F2400001339E42F8D100221C44002AE6D004EB90
:10F250000A0024B0BDE8F08708F1010806F87C8CAC
:10F26000039799E807008DE807000C9B23F07F4384
:10F270009A4494E80F002DF022F9054658B10C9BF2
:10F2800023F07F43034413F8013CC1E70122DBE78D
:10F2900082460446DBE70446D9E700BFD7240600D0
:10F2A0002DE9F04F0022A1B00D46664906462BF02D
:10F2B000D9F82BF0F7FEC0B2722808D062490120BD
:10F2C00023F088FC0027384621B0BDE8F08F0022EB
:10F2D0005E4930462BF0C6F82BF0E4FE804600284D
:10F2E00000F0AD8000225A4930462BF0BBF82BF0DD
:10F2F000D9FE00225749814630462BF0B3F82BF057
:10F30000D1FE00225449824630462BF0ABF80DF175
:10F31000240B014658462DF03DFB1B22531E1BF8C3
:10F32000031009B1134602E01A46002BF6D120AAB9
:10F33000D318069303F85CACEB0F059318BF202598
:10F3400000273DBB72E04FF000083BE012F8011BC4
:10F35000FF291CD005980133002862D00A2960D10A
:10F3600000221C46059237B91B20079329F080F92B
:10F37000079B074630B1224610A93846079329F06B
:10F380004DFF079B059AA1441AB91D1BD9E71C46DE
:10F390004AE02025C9F57E64002C33DCBAF1FF0F6A
:10F3A000D1D0069B0AF1010A03F85CAC18AB0393B9
:10F3B0000DAB93E807008DE807009BE80F002DF0E8
:10F3C0007EF88046404629F0D2F920490246304670
:10F3D0002BF00FF8002029F0CAF91D4902463046EB
:10F3E0002BF007F8504629F0C2F91A490246304678
:10F3F0002AF0FFFFB8F1000F3FF465AF4FF47E64D1
:10F400004FF00009202D2B46A8BF20239C42A8BF07
:10F410001C46224609EB080110A832F09BF810AAFE
:10F420000023A34292DB2B46002C9CD1484629F0B6
:10F430009EF90749024630462AF0DBFF43E70746BC
:10F4400041E700BF3D4D060048420600434206002A
:10F450003C42060036420600D72406004FF0FF313A
:10F46000FFF71EBF21EAE171FFF71ABF2DE9F04F48
:10F470000C46A5B005465F49204629F039FD98B9EC
:10F480005D49204629F034FD50BB5C49204629F0F7
:10F490002FFD064638BB22465949012023F09AFB2E
:10F4A000304625B0BDE8F08F4FF0720B5549002073
:10F4B00020F06AFE06460028F2D0082200212846E5
:10F4C00029F046FE0DF114080146044640462DF091
:10F4D00047FA1B214B1E18F803203AB10B4608E0EF
:10F4E0004FF0770BE2E74FF0610BDFE71946002B97
:10F4F000F0D124AA02EB03094349224630460125F4
:10F500000CAF09F87C5C0DF1240A2AF072FF039716
:10F510009AE807008DE8070098E80F002CF0CFFF6D
:10F52000BBF1770F044606D118B13046FFF7A0FCB7
:10F53000002427462BE0BBF1610F59D1002CF8D0F5
:10F540000C9B23F07F43234413F8013CFF2B01D095
:10F55000FF2D3DD10027C7F57E68B8F1000F16DDFD
:10F56000B8F1400FA8BF4FF040084246391914A81F
:10F5700031F0F0FF14AA002312F8011BFF2935D047
:10F5800001334345F8D100221F44002AE3D0284626
:10F5900029F0EDF81D49024630462AF02AFF384688
:10F5A00029F0E5F81A49024630462AF022FF2046A3
:10F5B00029F0DDF81749024630462AF01AFF58466E
:10F5C00029F0D5F81449024630462AF012FF67E7C1
:10F5D000013509F87C5C03979AE807008DE807007D
:10F5E00098E80F002CF06BFF0446A7E70122CBE759
:10F5F0000027CCE705BA0600EB610600817E060015
:10F600001A4206002A420600D724060036420600A7
:10F610003C420600434206003D4D0600F1F7FDBAAC
:10F620002DF061B970B5002290B00646084611462B
:10F6300009F0BAF909AC0546314620462DF090F99B
:10F640000023CDE90533CDE9035310AB13E90700DF
:10F650008DE8070094E80F002CF078FF10B070BD23
:10F660002DE9F041804690B008460C4617461E46EC
:10F6700028F074FB60B300222046114609F094F98B
:10F6800000260446374609AD284641462DF068F964
:10F690000023CDE90343CDE9057610AB13E907005C
:10F6A0008DE8070095E80F002CF050FF05465CB18F
:10F6B000E389A3F500739BB2E381E38903F4F0537C
:10F6C00013B9204629F07CF8284610B0BDE8F08137
:10F6D000002CD8D0E28902F5007292B2E281D2E722
:10F6E00030B58FB007AC0146002520462DF038F923
:10F6F000CDE903550EAB13E907008DE8070094E848
:10F700000F002CF0F3FF044690B1294629F0EEFEDD
:10F71000E389A3F500739BB2E381E38903F4F0531B
:10F72000054613B9204629F04BF828460FB030BDE6
:10F730000546FAE770B58EB007AC16460D46014691
:10F7400020462DF00DF9CDE903560EAB13E9070065
:10F750008DE8070094E80F002CF0C8FF0EB070BDD4
:10F7600070B58EB007AC0E46014620462DF0F8F875
:10F770000023CDE903330EAB13E907008DE8070042
:10F7800094E80F002CF0B2FF044600B305F012FE1F
:10F79000E389A3F500739BB2E381E38903F4F0539B
:10F7A000054613B9204629F00BF86EB122F0A4FCEF
:10F7B00050B1C389A3F500739BB2C381C38903F41D
:10F7C000F0530BB928F0FCFF28460EB070BD05467B
:10F7D000FAE74FF4DA202CF0DDBF000013B50C4639
:10F7E0001DF0B6FA8DF807000938062805D80DF186
:10F7F0000702034920462AF09DFF02B010BD00BF5A
:10F8000005F802000B78C1B218461DF0D3B800000D
:10F810002DE9F04389B01F4680460C4691461DF005
:10F8200097FAA0F10903DBB2062B06463AD80F2857
:10F830000FD1374BDB7863B94FF0FF324FF41651DD
:10F84000CDE9041204A8334A06928DF81C30F6F76D
:10F85000D1F8314D8DF80060B9F1000F03D020468A
:10F860002BF0E2FD04466A46294620462AF062FF54
:10F87000B9F1000F0CD05CB1E389A3F500739BB222
:10F88000E381E38903F4F05313B9204628F098FF8D
:10F890002FB169460D20A84769460A20A84709B03C
:10F8A000BDE8F0830028FAD102461C4940462AF000
:10F8B000D9FD324605461A4940462AF0D3FD0DF1DE
:10F8C000100806460246294640461BF05DFE5EB122
:10F8D000F389A3F500739BB2F381F38903F4F0532A
:10F8E00013B9304628F06CFF5DB1EB89A3F50073C6
:10F8F0009BB2EB81EB8903F4F05313B9284628F04F
:10F900005FFF98E80F006D4607C52B70054DA3E714
:10F9100001D300200800010071700400E63B0600DE
:10F92000E83F0600756F040000231A46FFF770BF1A
:10F9300001231A46FFF76CBF00230122FFF768BFBF
:10F94000F0B585B004461DF003FA002205463C4997
:10F9500020462AF087FD064628B93A49012023F0BF
:10F9600039F905B0F0BD0022374920462AF07AFD6A
:10F9700032460146074668461BF006FE39463046C9
:10F980002AF0F0F9304920462BF05EFC2C49204645
:10F990002BF05AFCA5F10903DBB2062B44D9002257
:10F9A0002A4920462AF05EFD08B32BF07BFBC4B247
:10F9B0000021204611F070FF00201BF079FD054664
:10F9C000A8B1214629F0AAF8044618B101462846F4
:10F9D0002BF07CFB284629F0D5F920B91C4B1D499A
:10F9E00058682BF031FC294620462AF0BBF99DF8D7
:10F9F0000600FF2802D0002112F036FB9DF8070018
:10FA0000FF2802D0002112F02FFB9DF80400FF28F0
:10FA100002D0002112F028FB9DF80500FF28A0D09D
:10FA2000002112F021FB9CE7A5F10D03DBB2022BB4
:10FA3000DDD8FF22002128461DF0E8FAD7E700BFF5
:10FA4000E83F060063410600E63B06008A410600E7
:10FA50008C2E00208F410600F0B585B005460F467C
:10FA600014461DF075F90646D4B922465B4928466E
:10FA70002AF0F8FC04462246394668461BF084FD0D
:10FA8000A0B95CB1E389A3F500739BB2E381E3897C
:10FA900003F4F05313B9204628F092FE05B0F0BDF0
:10FAA000E38903F500739BB2E381E4E7009828F053
:10FAB0005EFE4B49024628462AF09BFC7CB122465A
:10FAC000464928462AF095FCA6F10903DBB2062B2D
:10FAD0000AD80F2EE2D16846F5F78CFFDEE73F49E2
:10FAE00028462BF0B1FBEFE7002ED7D19DF805009B
:10FAF000FF2807D0012112F0B7FA01219DF8050077
:10FB00001EF094F89DF80400FF280BD0052112F098
:10FB1000ABFA602028F026FD044660B93149012087
:10FB200023F058F89DF80630FF2BB7D02E4901205E
:10FB300023F050F8B2E702462C4928462AF059FC37
:10FB4000204628F069F9002680F84060044611F04C
:10FB5000D9FF009B9DF80A2084F85860C4E9143648
:10FB60009DF8083013449DF80920B24218BF0133B4
:10FB7000C4E9120184F8593001219DF8040011F004
:10FB80008BFE044610B328F0F2FD194902462846C0
:10FB90002AF02FFC01201BF08BFC06460028C1D068
:10FBA0002A4621462AF090FBF389A3F500739BB205
:10FBB000F381F38903F4F05313B9304628F000FEC3
:10FBC000013C0C4B0C4A43F82420ABE79DF8042081
:10FBD0000A49012022F0FEFFA4E700BFE83F06002B
:10FBE000E63B0600DE4006003B41060004410600FD
:10FBF0008A410600E8D70020CDB404000C4106007D
:10FC000010B50C461DF0A4F8A0F10903DBB2062BD9
:10FC100004D82146BDE810401EF08CBB02490120EB
:10FC2000BDE8104022F0D6BFB34006002DE9F347EF
:10FC30001F46012313600C690646894615460CB120
:10FC40000B68E45C30782E2800F0DE805B282CD135
:10FC500001237B7296F801A0BAF15E0F02D12B68E6
:10FC600001332B604FF000080CE03B4601AA4946E7
:10FC7000FFF7DCFF2B68019A48EA000813445FFA9B
:10FC800088F82B602B68F45CF018002C00F0BE8024
:10FC90005D2CEAD101332B6000237B72BAF15E0F39
:10FCA00014BF444688F001040BE05C2861D10223B4
:10FCB0002B607078642808D1303C092C8CBF00245C
:10FCC0000124204602B0BDE8F087442805D1303C2D
:10FCD000092C94BF00240124F3E766285FD06E2826
:10FCE0005FD072285FD0732805D1204602B0BDE8EE
:10FCF000F04723F045BC532806D1204623F040FCB2
:10FD000080F00100C4B2DCE774284ED076284ED0D3
:10FD100077280DD1A4F13003092B75D9204623F0A3
:10FD200023FC002870D15F2C14BF00240124C8E7F5
:10FD300057280CD1A4F13003092B61D9204623F0B8
:10FD400013FC00285CD15F3C18BF0124B9E7A0F187
:10FD50003003DBB2092B2CD978280AD1B37843B110
:10FD6000F37833B104232B60F178B07823F0EBFB08
:10FD7000C0B27B7AFBB12B68F35C2D2B1BD1788151
:10FD80002868013028603B4601AA49463044FFF705
:10FD90004DFF2B68019A134404462B6091E70C2019
:10FDA000E7E70A20E5E70D20E3E70920E1E70B207C
:10FDB000DFE71846DDE73A7A62B1A4F14103192B77
:10FDC00098BF2034A0F1410398BFE4B2192B9CBF27
:10FDD0002030C0B2B7F90A30B3F5807F12D0DBB261
:10FDE0002AB1A3F14102192A9CBF2033DBB24FF4A0
:10FDF00080729C427A8103D3844201D8984268E79A
:10FE000000245EE784428FE701245AE7024901207B
:10FE100022F0E0FE55E700BF3244060082B02DE933
:10FE2000F047ACB00C4634A9064681E80C0022F03D
:10FE30004BFA30B1002528462CB0BDE8F04702B09F
:10FE4000704733780BB17C2B5BD1582234A90DEB72
:10FE5000020031F07FFBDDE93467DDF8DC8028F05B
:10FE600071FCA26823681A440546D21B3946304605
:10FE700029F06EF900210446024628462AF024FAA9
:10FE80005CB1E389A3F500739BB2E381E38903F4DA
:10FE9000F05313B9204628F093FC0DF1680A4FF097
:10FEA0000009C1450DDB384628F061FC8649024651
:10FEB00028462AF09EFA3246844928462AF078FAE3
:10FEC000B9E75AF8041BDAF820203046521A29F014
:10FED0003FF909F1010904460246494628462AF03D
:10FEE000F3F9002CDDD0E389A3F500739BB2E38125
:10FEF000E38903F4F053002BD3D1204628F060FCB3
:10FF0000CFE75E2B09D12368A268D34292D123F0B8
:10FF10009DF800288ED0013607E0242B1DD1D4E9AE
:10FF200000329A4206F101060CD8502236A96846E2
:10FF300031F010FB34AB0CCB21463046FFF76EFF9F
:10FF4000054678E74C2237A9684631F003FB34AB0D
:10FF50000ECB304600F0B5FAF2E7282B0FD1379BD5
:10FF60002168A26834A80A44191D082B40F82120F2
:10FF700000EB83014A63CADC01333793C7E7292BBF
:10FF80000AD1379B002BC2DD34AA02EB8303216820
:10FF9000A2680A441A63BAE734AB15AA2146304670
:10FFA000FFF744FE159FF35DA3F12A02012A804664
:10FFB00006EB07056ED80137374450B92B2B08D113
:10FFC0004C2237A9684631F0C5FA34AB0ECB38461F
:10FFD000C0E7214616A827F043FC502236A9684600
:10FFE00031F0B8FA34AB0CCB16A93846FFF716FF40
:10FFF0000546199850B1C389A3F500739BB2C3811C
:020000023000CC
:10000000C38903F4F0530BB928F0DAFBD4E90023D9
:100010009A42BFF410AFB8F1000F3FF40CAF204686
:1000200027F0F8FC34AB15AA21463046FFF7FEFD59
:100030002146804616A827F013FC502236A96846B0
:1000400031F088FA34AB0CCB16A93846FFF7E6FE40
:100050008146199850B1C389A3F500739BB2C3813F
:10006000C38903F4F0530BB928F0AAFBB9F1000FD0
:100070000ED05DB1EB89A3F500739BB2EB81EB89E8
:1000800003F4F05313B9284628F09AFB4D46BDE718
:10009000A946FBE7D4E900239A420BD250B120468F
:1000A00027F0B8FC22F0D2FF00283FF4C3AE159B26
:1000B0001E443AE74C2237A9684631F04BFA34AB7C
:1000C0000ECB284646E700BF544406005A440600BB
:1000D0002DE9F047B4B08046084614AF2BF0A4F9E0
:1000E00000226B49054640462AF0BCF92AF0DAFFA7
:1000F00000226849824640462AF0B4F9064627F0B5
:1001000046FF044640B93146284629F02BFE2046DA
:100110008037BD46BDE8F087304629F044F900F14C
:10012000080323F00703ADEB030D0DF15009421C4A
:10013000494630462BF052FB5EB1F389A3F50073BC
:100140009BB2F381F38903F4F05313B9304628F0DE
:1001500037FB69214046FDF749FA4FF480720023CE
:1001600087F830007A8629465246384687F831307B
:100170007B63BD6227F058FE394607F1140027F073
:100180006FFB502207F130016846C7F82CA031F010
:10019000E1F9564607F1280A9AE80C0007F1140124
:1001A0004846FFF73BFE0446386A50B1C389A3F5C1
:1001B00000739BB2C381C38903F4F0530BB928F0D9
:1001C000FFFA384627F026FC1CB9D7E900239A42EB
:1001D00028D3F86850B1C389A3F500739BB2C381DB
:1001E000C38903F4F0530BB928F0EAFA5DB1EB8947
:1001F000A3F500739BB2EB81EB8903F4F05313B9C1
:10020000284628F0DDFADCB9022028F031FA002572
:100210000446284628F0ABFA1D49024640462AF01B
:10022000E8F874E7394607F1140027F019FB0136A6
:10023000502207F130016846FE6231F08BF9ABE7DE
:1002400067214046FDF7D2F900B30021204629F08E
:100250008DFE00221049064620462AF003F92AF0B6
:1002600021FF0546304629F09EF80544002ED0D0E7
:10027000F389A3F500739BB2F381F38903F4F05380
:10028000002BC6D1304628F09BFAC2E70546C0E7EE
:10029000A34006009C400600544406002DE9F84F98
:1002A00005460E4627F073FE20B94FF00008404681
:1002B000BDE8F88F28F046FA80460028F5D01EB930
:1002C000294629F087FFF2E73046F0F76DFD002858
:1002D00000F08180002028F04AFA6A490246304640
:1002E0002AF087F829463046FFF7F2FE0027044639
:1002F00084B1204627F0F8FC814618B3E389A3F5C2
:1003000000739BB2E381E38903F4F05313B92046F1
:1003100028F056FA002028F02AFA5A4902463046B8
:100320002AF067F8284629F03EF8B842BFD339468C
:100330006FF00042284628F00BFF0146404629F0A6
:100340006BFFB4E74946204629F010FE4A464E4965
:10035000824620462AF086F82AF0A4FE81465046BE
:1003600029F021F88346BAF1000F0ED0BAF80E201A
:10037000A2F5007292B2AAF80E20BAF80E2002F48A
:10038000F05212B9504628F01BFAA9EB0702394681
:10039000284628F0DDFE0146404629F03DFFE3896E
:1003A000A3F500739BB2E381E38903F4F05309EBF7
:1003B0000B0713B9204628F003FA384628F0D7F97E
:1003C0003049024630462AF014F829463046FFF7F5
:1003D0007FFE04468CE730462BF026F8064698B19F
:1003E00028F0E1FF8146284628F0DDFF002700F1D4
:1003F000010BABEB090A3C46544531DCB9F1000F67
:100400001CD1C4B90134F7E78146ECE75C461FE034
:100410000146404629F0DEFEFB89A3F500739BB23E
:10042000FB81FB8903F4F05313B9384628F0C8F96F
:1004300004EB0907E6E754450AD111E05445E5D03D
:100440000123224631462846F0F796FA0028D9D1F2
:10045000E21B3946284628F07BFE07460028D7D104
:10046000002E3FF424AFF389A3F500739BB2F38110
:10047000F38903F4F053002B7FF419AF304628F0D2
:100480009FF914E7A34006005444060038B5FFF76F
:100490001FFE054620B127F027FC80F00100C0B206
:1004A00000F001045DB1EB89A3F500739BB2EB8111
:1004B000EB8903F4F05313B9284628F081F920465C
:1004C00038BD84B0F0B59BB021AE054686E80E007D
:1004D00022F0BCFD68B9044620461BB0BDE8F040E0
:1004E00004B070475C2C03D16C78002CF4D03D46EE
:1004F00001352C78002CEFD07C2C05F10107F1D1CF
:10050000DDE9211215A827F08FFC502223A96846A7
:1005100031F020F896E80C0015A93846FFF77EFC6C
:10052000044618980028D7D0C389A3F500739BB25E
:10053000C381C38903F4F053002BCDD128F040F9D7
:10054000CAE70000F7B5064608460D46144627F0F0
:100550001DFC30B92A463349032022F03BFB03B08F
:10056000F0BD6CB300223049304629F0D5FE009032
:10057000C0B129F0D7FC012300906A46002029462B
:100580001CF036FB00980028E9D0C389A3F500735E
:100590009BB2C381C38903F4F053002BDFD128F051
:1005A0000FF9DCE7214F00223946304629F05AFF87
:1005B000044638B92A463946304629F0F9FECEE7D6
:1005C0001B4FF0E727F0C2FB78B12946204629F0FF
:1005D00001FEE389A3F500739BB2E381E38903F491
:1005E000F053002BBBD12046D9E702216846CDE964
:1005F000004529F056FE394605460246304629F0A8
:10060000D7FE002DE5D0EB89A3F500739BB2EB81FB
:10061000EB8903F4F053002BDBD1284628F0D0F807
:10062000D7E700BF943B0600B83B06008A3B0600B4
:100630008F3B060010B500220446FFF783FF2046DB
:10064000BDE81040FDF7D0B838B515460122044684
:10065000FFF778FF25B1002229462046FFF772FFF9
:100660002046BDE83840FDF7BFB8000037B5054665
:1006700001910F4848F2080128F05AF80446A8B141
:100680002A460C4929F094FE012301AA2146284656
:100690001CF0AEFAE389A3F500739BB2E381E38912
:1006A00003F4F05313B9204628F08AF803B030BDA4
:1006B000FB0B0300911D06002DE9F0410F4690460B
:1006C00018490022064629F0CDFE2AF0EBFC002254
:1006D00005461549304629F0C5FE0446F8B14246A4
:1006E0003946013D29F0F0FD284628F040F80D4933
:1006F0000246304629F07DFE1DB921463046FFF7FF
:10070000B5FFE389A3F500739BB2E381E38903F4AA
:10071000F05323B92046BDE8F04128F051B8BDE8B8
:10072000F08100BF594006005F40060037B505461E
:1007300001910F4848F2080127F0FAFF0446A8B1DA
:100740002A460C4929F034FE012301AA21462846F5
:100750001CF04EFAE389A3F500739BB2E381E389B1
:1007600003F4F05313B9204628F02AF803B030BD43
:10077000F50B0300911D060038B500220D460D490A
:10078000044629F06FFEA0B1C389A3F500739BB2A4
:10079000C381C38903F4F0530BB928F011F8204644
:1007A00004492AF051FD29462046BDE83840FFF7AC
:1007B000BDBF38BD5F40060070B51FF069FC06463E
:1007C00080B30022184929F04DFE054627F0DEFAD5
:1007D0000446F8B1F389A3F500739BB2F381F38962
:1007E00003F4F05313B9304627F0EAFFC5B12C6883
:1007F0000E4BE31A5C425C4185B1EB89A3F50073B3
:100800009BB2EB81EB8903F4F0533BB9284627F008
:10081000D7FF03E03146284629F0A4FA204670BDF0
:100820002C46E9E70446F9E732620600552B03003F
:100830002DE9F04F85B0054627F0D4FB044640B9BA
:100840002A464849032022F0C5F9204605B0BDE8F4
:10085000F08F454900201FF097FC04460028F4D093
:1008600048F20801414827F063FF06460028ECD013
:1008700022463F49DFF8F8B029F09AFD27F062FFE1
:100880002946824603A823F087FA4FF0000847461E
:100890000398D8B9A7EB080027F069FF354902464D
:1008A000204629F0A6FD52463349204629F0A1FDF5
:1008B000F389A3F500739BB2F381F38903F4F0533A
:1008C000002BC2D1304627F07BFFBEE729F026FB84
:1008D0000546FFF771FF00283BD048F2600127482A
:1008E00027F026FF8146384627F041FF00210246C7
:1008F000019048462AF00AFB019B5BB1DA89A2F518
:10090000007292B2DA81DA8902F4F05212B9184612
:1009100027F056FF22465946484629F049FD4946E8
:1009200032462846FFF790FE494629F01BFA5DB192
:10093000EB89A3F500739BB2EB81EB8903F4F053D1
:1009400013B9284627F03CFF03A8013723F0E8F944
:100950009EE72A463946504629F0B6FC08F10108C0
:10096000E5E700BF7B3F060064400600790703000F
:10097000911D0600594006005F400600B9060300BD
:100980002DE9FF41064610460191144627F0DEF995
:100990000746002852D0214603A823F0FDF9002481
:1009A000039810BB454930462AF04EFC4449304676
:1009B0002AF04AFC00224349304629F053FD4149C0
:1009C000054630462AF040FC21F096FB8046002880
:1009D0003ED001462846FFF7A9FE2A46214640465A
:1009E00029F094F904B0BDE8F08129F097FA01AB41
:1009F0000122314605461EF07BF9EFB950B1C2899C
:100A0000A2F5007292B2C281C38903F4F0530BB90C
:100A100027F0D6FE5DB1EB89A3F500739BB2EB81A5
:100A2000EB8903F4F05313B9284627F0C9FE03A855
:100A300023F076F90027B3E70446EBE7002CB1D0AA
:100A4000204601AB012231461EF052F90446A9E7C7
:100A50004DB32046FFF7B0FE50B348F208011A48E4
:100A600027F066FE48F208010646184827F060FEA7
:100A70000746A6B198B12A461549304629F098FC98
:100A80002A461349384629F093FC01223146204674
:100A9000FFF758FD424639462046FFF753FD3946D9
:100AA000304629F05FF92946204629F05BF999E79D
:100AB00021462846FFF7DAFDF5E700BF8A3B06002E
:100AC0008F3B06004BB006006D0603002D070300A8
:100AD000911D0600414B2DE9F047B2F100080E468A
:100AE0004FF000023E493F4F054608BF1F4629F020
:100AF000B9FC044668B1C389A3F500739BB2C381F6
:100B0000C38903F4F053002B66D1BDE8F04727F00A
:100B100057BE012027F023FE31490246284629F01E
:100B200068FC22463946284629F09CFC04460028E9
:100B30004ED102462C49DFF8B090284629F092FCAD
:100B40000446CCB9B8F1000F3BD0324627492846BD
:100B500029F02EFC002C3FD0224631462846FFF7D4
:100B60000FFFE389A3F500739BB2E381E38903F4EC
:100B7000F0538BBB2046C8E700223946204629F0B7
:100B800071FC8246024648B131462046FFF7F8FE26
:100B900021465046BDE8F04729F0E4B849462046D2
:100BA00029F060FCE389A3F500739BB2E381E3893C
:100BB00003F4F053824613B9204627F001FE544651
:100BC000BFE732460A490120BDE8F04722F002B8EB
:100BD000B8F1000FC0D0B8E7BDE8F0878F3B060042
:100BE000C13B06008A3B06004BB00600B83B06003E
:100BF000C63B06000022FFF76DBF0122FFF76ABF68
:100C000010B590B00C460146684617F0F3FB40B1B2
:100C1000BDF80530DB0648BF84F001041CB1BDF807
:100C2000090010B010BDBDF80700FAE72DE9F74F35
:100C300021F00045894616461F464FF0FF32414BD2
:100C400029468046044630F00BFA002876D14FF052
:100C5000FF323C4B4046294630F0F8F900286DD170
:100C600032463B463046394630F0FAF9002865D125
:100C7000002200234046494630F0CAF928B309F162
:100C80000045002200233046394630F0C1F910B14A
:100C900007F100431F46002200233046394630F05A
:100CA000ADF978B94FF0FF32264B3046394630F077
:100CB000B9F938B14FF0FF32224B2046294630F0C7
:100CC000B1F9E8B90024002522E04D46D9E7002219
:100CD0001D4B204629462FF029FFCDE90001B246E1
:100CE000BB4652465B46DDE9000130F0A5F95246AD
:100CF0005B46E0B9204629462FF060FD04460D46CC
:100D000022462B463046394630F08CF90028DED199
:100D1000002200234046494630F07AF910B105F12F
:100D200000431D462046294603B0BDE8F08F10461B
:100D300019462FF045FD82468B46D2E70024034D2D
:100D4000F0E700BFFFFFEF7F0000E03F0000F87F0B
:100D50002DE9F84355EC114B11EE100A294657ECDA
:100D6000106B30F093F90928804619D82FF074FEE3
:100D700022462B4630F042F990B1B8F1000F63D013
:100D800030463946B8F1010F03D141EC100BBDE8F4
:100D9000F88332463B462FF0C9FE08F1FF38F1E7F1
:100DA000002200233046394630F032F90022D8B311
:100DB000284B20462946FFF739FF0022002330F058
:100DC0001DF9F0B300224FF0804320462946FFF77B
:100DD0002DFF0022002330F011F9B04607F1004941
:100DE00049EC108B68B12DF0EFFE22462B4651ECFA
:100DF000100B2FF09BFEBDE8F84341EC100B2DF0DB
:100E00005FBE2DF0E1FE22462B4651EC100B2FF079
:100E10008DFE41EC100B2DF053FE53EC102B10EE19
:100E2000100A03F10041B0E700233046394630F0A4
:100E3000E5F830B1002200232046294630F0F2F8D0
:100E400028B147EC106BCEE7002002499DE7002057
:100E500000219AE70000F03F37B50D46014668468D
:100E60001446FCF751FF98B1019890F82532013BE8
:100E7000022B0DD874B18168294419F0E8FE0146AF
:100E800030B10548054B002C08BF1846FCF73AFB6B
:100E900003B030BD2146EFE7963D0600A53D0600B4
:100EA00070B50E4E34783CB917F044FC054628B9AD
:100EB0000B49012021F08EFE204670BD09490A48E9
:100EC00001221AF0AFFA014618B10848FCF71AFBE4
:100ED000F2E7012333702C46EEE700BFB0D50020C7
